:020000040800F2
:1000000000000220D99705087199000839570208A5
:100010008998050889980508899805080000000056
:10002000000000000000000000000000A1B0000877
:10003000A3B0000800000000A5B000086914010882
:1000400089980508899805088998050889980508F8
:100050008998050889980508E7FD0008EBFD000868
:1000600089980508EFFD0008F3FD000861A000086D
:1000700075A0000889A000089DA00008B1A0000894
:10008000C5A00008D9A00008899805080000000054
:10009000000000000000000000000000F7FD000864
:1000A000999F0008C19F0008E99F0008839F0008EE
:1000B00011A0000825A0000839A0000889980508AB
:1000C0008998050889980508899805088998050878
:1000D00089980508B59A0008C19A00080000000038
:1000E000FBFD000889980508A7B000080000000083
:1000F000000000000000000000000000EDA000086B
:1001000000000000899805084DA00008899805089E
:1001100000000000000000000000000000000000DF
:1001200001A1000815A1000829A100083DA10008AF
:1001300051A10008000000000000000000000000C5
:10014000000000000000000000000000F9B00008FE
:1001500065A1000879A100088DA10008899805080B
:100160008998050889980508000000000000000033
:10017000000000000000000000000000000000007F
:100180000000000089980508000000000000000041
:0801900089980508899805080B
:1001980081C90181008408B10000000080C9018183
:1001A800008408B10000000080C90181B0AB08B12B
:1001B80000000000C9010181B0B0AC80000000005F
:1001C800C9060181B0B0AF85000000003F1A018167
:1001D800B0AF81C90000000008B10181B0B000844F
:1001E8000000000008B10181B0B0008400000000E8
:1001F800309F050000840280989F050001000000E0
:1002080000A10500008402806CA105000100000027
:100218006CA105007CFFFF7F20A2050080FFFF7F07
:1002280060A2050084FFFF7F48A30500B0B0AE8040
:10023800ECA40500B0A8018034A6050078FFFF7F74
:1002480054AC0500B0AA0580B0AE0500010000005E
:10025800B0AE05006CFFFF7F1CBA0500010000006E
:10026800B0BC050068FFFF7F1CC30500010000004B
:10027800A4C30500B0A80180B4C3050001000000B4
:10028800E4C30500B00D8480F4C30500010000003C
:1002980018C4050044FFFF7F24C4050048FFFF7F02
:1002A80030C40500AF08B18068C705000100000030
:1002B80074C70500A908B18020C905000100000025
:1002C800F4FE0500A908B1801CFF0500010000002C
:1002D800E8FF0500B0A902807C000600B0B0A88045
:1002E800CC00060001000000D4000600B0B0AA80CF
:1002F80008010600AE71B280CC010600AB3F388021
:100308002C0206000100000034020600B0B0AA80EA
:10031800700206000100000010030600AA0DB2805A
:100328008C030600B0AF08802C0606000100000010
:100338003C060600AD3F0280B80806000100000038
:10034800E8080600B0AD04808C0B06000100000030
:10035800C02201200201000002001400E022012056
:10036800020200000200140000230120020A00001B
:1003780002001400202301200206000002001400DD
:10038800402301200207000002001400602301201E
:10039800020300000400140080230120020800006A
:1003A80004001400A0230120010B000000007700C6
:1003B800C0230120010C000000007600E02301208A
:1003C800011000000000760000240120010D01004A
:1003D80000007700202401200112000000007600B0
:1003E800402401200114000000001E0060240120A8
:1003F800011A000000000D0080240120011B0000EC
:1004080000000E00A0240120011C000000001E00B6
:10041800C02401200117000000000C00E024012086
:100428000118000000000E0000250120012801002D
:1004380000001800202501200120000000004800CD
:10044800402501200121000000004900602501200D
:100458000122000000004A0080250120012300003D
:1004680000004B00A02501200124000000004C00E2
:10047800C02501200125000000004D00E0250120D5
:100488000126000000004E00002601200127000080
:1004980000004F0020260120012B00000000290049
:1004A80040260120012C01000000290060260120BF
:1004B800012D01000000700080260120012E01009E
:1004C80000005200A0260120012F01000000280092
:1004D800C02601200130010000002800E02601208C
:1004E8000234040000012C00002701200133000021
:1004F80000003C00202701200136000000002000F9
:10800000D0E907239A422FBFD01AC0688018C01A3F
:108010007047D0E9092300699A4238BF1218D31A71
:108020000138C01A7047D0E90902131A5842584162
:108030007047036A41690246C85CD16801338B42CC
:1080400028BF002313627047436A8269D154436A90
:1080500002690133934228BF0023426B4362D36815
:1080600043F08003D3607047436B188810F0100012
:108070001EBF1A889B8801207047436B99891A8814
:10808000890610B592B2044607D5900605D5E26A76
:1080900022B39888216B80B29047636B99891A88C4
:1080A000090692B20FD510060DD5D4E909128A42FD
:1080B00022D0A169895C998021690132B2FBF1F07B
:1080C00001FB1022A262998A1A88C90592B204D5CE
:1080D000D20744BF4FF6F7721A8010BD9B88E26941
:1080E0006169DBB28B54E369E2680133B3FBF2F1FF
:1080F00002FB1133E361D0E7DA6822F08002DA6034
:10810000E1E7036941681F2B30B54FF0200285BFBE
:10811000A3F120054C680C68AA4098BF9A402242FF
:108120001ED0826900201074D0688468206820F016
:10813000010020605468206865790A4C828934F80F
:10814000154092B21F2B22EA0402828188BF203B95
:108150004FF020028BBF9A4002FA03F3CA608B6093
:1081600030BD00BFD41106080E4BDA68D20310D41C
:10817000DA68D1060FD4DA68D2050ED4DA6812F0C4
:10818000E00F0CD1DB6813F0020F14BF08200920A8
:108190007047012070470620704702207047072073
:1081A000704700BF003C024007B509238DF8073037
:1081B000FFF7DAFF8DF807009DF80730012BF7D0A5
:1081C0009DF8070003B05DF804FB838A028B9BB225
:1081D00043EA024331EA03030CBF01200020704749
:1081E00082B0002301930093012300900193019B2F
:1081F00063B1009A21F07F4314320092009A126812
:108200001A4214BF0120002002B07047009A1832B1
:10821000F3E77047704701207047044BD3E9000330
:10822000984288BF03F50063181A70473818002079
:10823000054AD2E900318B42FDD0D1180133C3F396
:108240000A03087A1360704738180020044BD3F8EB
:10825000080820B1D3F80808431F58425841704716
:1082600038180020012380F84930704710B5D0F845
:10827000E83504461B699847032384F8123100202F
:1082800010BD08B590F8123180F81331042380F83E
:108290001231D0F8E835DB689847002008BD08B5F2
:1082A000D0F8E435DB6903B19847002008BD08B574
:1082B000D0F8E4351B6A9847002008BD08B5D0F80F
:1082C000E4355B6A9847002008BD30B501380024CA
:1082D00023460134055D002DFAD1DBB201335B008A
:1082E00013800B7003234B70022310F8014F04B965
:1082F00030BD5A1CD2B2CC5402338D54DBB2F4E7F9
:1083000010B5074C2068FF2808D00649D1F80C2882
:1083100001F5016100F070F8FF232360002010BD1B
:108320000000002038180020432301480B807047CC
:1083300004000020122301480B80704747000020F2
:10834000042301480B8070475900002008B50A46F5
:1083500002490348FFF7B9FF084608BD5020002036
:10836000E8AD060808B50A4602490348FFF7ADFF25
:10837000084608BD50200020FBAD060808B50A4697
:1083800002490348FFF7A1FF084608BD502000201E
:1083900000AE060808B50A4602490348FFF795FFF4
:1083A000084608BD502000200AAE060808B50A4657
:1083B00002490348FFF789FF084608BD5020002006
:1083C00015AE060870477047704770477047704792
:1083D000044B00200522C3F80828C3F81809C3F885
:1083E0001C09704738180020024B0020C3F8080809
:1083F000704700BF38180020212838B50C461BD024
:1084000022282BD0202815D1A1B1072A12D11A4D2C
:10841000D5F81C3913B10968002098472368C5F8BE
:108420002039237985F82439637985F82539A379AA
:1084300085F82639002038BD0029FBD0072AF9D15C
:108440000D4BD3F820290A6093F824290A7193F878
:1084500025294A7193F826398B71EBE70029E9D079
:10846000022AE7D1044BD3F81839002BE2D009884F
:1084700000209847DEE700BF38180020074AD2F8EE
:108480002839D2F82C29934203F1FF338CBF002006
:1084900001209B1A03EBC020704700BF3818002052
:1084A000ECE730B50F4CD4E900239A4286BF03F5C0
:1084B0000065AA1A9A1A0A44B2F5006F10D801444E
:1084C0000022814203D102B16360002030BDE21876
:1084D00010F8015B15720133C3F30A030122F0E7C0
:1084E0000220F3E738180020034BD3F8300908B115
:1084F00003691847704700BF38180020034B93F8F2
:108500005809003818BF0120704700BF38180020F4
:10851000034B93F85809032894BF002001207047AB
:10852000381800200048704794210020837B042BDA
:108530000DD0074BD3F898200132C3F89820426041
:1085400004228273D3F89C200132C3F89C20704728
:10855000045F0020202301480B8070475D0000204D
:10856000122301480B8070477D000020042301483E
:108570000B8070478F0000200A4608B5044920B9D7
:108580000448FFF7A2FE024808BD0348F9E700BF10
:10859000C421002023AE06083BAE060808B50A46F3
:1085A00002490348FFF791FE084608BDC421002098
:1085B00053AE060808B50A4602490348FFF785FE90
:1085C000084608BDC421002066AE060808B50A4664
:1085D00002490348FFF779FE084608BDC421002080
:1085E00071AE0608002370B54D1C1E46040FB0F195
:1085F000204F34BF3034373401F8134005F813608E
:108600000133DCB2A2424FEA0010EFD870BD1A234A
:1086100010B50B80094BD3F8E807D3F8EC27801886
:108620000AD0D3F8EA4706490822FFF7DBFF042205
:1086300010312046FFF7D6FF024810BD00F0FF1FA3
:10864000950000209300002008B5FFF74DFF80F053
:108650000100404240B208BD002070470020704732
:1086600070477047D0ED007AD0ED036A30EE677A3C
:10867000E6EE877AB0EE670AC0ED007A7047D0ED7B
:10868000017AF5EE407AF1EE10FA09D1DFED0F7ABA
:1086900060EEA70AB7EE007AC7EE207AC0ED017A45
:1086A000D0ED017A80ED021A71EE277AC1EE276AC9
:1086B000D0ED007AC0ED036A30EE677AE6EE877A95
:1086C000B0EE670AC0ED007A704700BFDB0FC9400B
:1086D000D0ED017AD0ED036A30EE670AE6EE807ADB
:1086E00090ED000AC0ED017AB0EE677AD0ED027A23
:1086F00037EE677AE6EE877AC0ED027A77EEC07AD7
:10870000A6EEA70A80ED000A704790ED056AD0ED4D
:10871000017AD0ED006AD0ED025A90ED045A66EE6F
:10872000277AB0EE407AE6EE807AD0ED066A80EDE8
:10873000057AE5EEA67AD0ED076AD0ED035A80ED12
:10874000066AE5EEE67AD0ED085AC0ED086AE5EE75
:10875000657AB0EE670AC0ED077A7047D0ED006A1F
:10876000D0ED057AE6EE807AB0EE407AB0EE670A98
:10877000D0ED037AD0ED016A67EEC07AE6EE877A33
:10878000D0ED066A76EEA77AD0ED026AC0ED057AE2
:10879000D0ED047A67EEC07AE6EE877AC0ED067A0D
:1087A000704703685A1C02601970704703690133EF
:1087B000012B036106D1002380ED010A80ED000A40
:1087C0008360704790ED006A07EE903A70EE466A5B
:1087D000F8EEE77A86EEA77A77EE067A90ED027ADF
:1087E000C0ED017A30EE670AC0ED007AA6EE807A1D
:1087F00080ED037A80ED027A704703685A1C0260AC
:1088000019707047007970470079C0F340107047C5
:108810000079400970472DE9F041476906468846CE
:10882000002F59D10368C3F30D0515B3D8F80080A4
:108830003568FFF7B9FC092840F08780444C23696C
:1088400023F440732361236943F400732361236994
:1088500043F001032361C5F80080FFF7A5FC2369FD
:10886000092823F0010323616FD133680433336097
:1088700032E0384A934229D302F58042934224D30E
:1088800002F5804293422AD3334A934229D902F512
:108890008032934227D902F50032934225D902F55E
:1088A0000032934223D902F50032934221D902F5D6
:1088B000003293421FD902F5802293421DD9B3F1B1
:1088C000016F1CD305200BF00DF80825FFF76CFC99
:1088D000092816D04FF0FF373846BDE8F081102543
:1088E000F4E71825F2E72025F0E72825EEE7302504
:1088F000ECE73825EAE74025E8E74825E6E758258C
:10890000E4E7134C236923F440732361236943F4A0
:1089100000732361236923F0F803236123691D4356
:1089200045F002052561236943F480332361FFF795
:108930003BFC236923F0020323612369092823F008
:10894000F80323613FF472AFC4E76FF00107C3E798
:10895000003C024000400008FFFF000803682DE9CA
:10896000F04104464068134483421AD80D468E18DD
:1089700004F10C074FF00008B54202D16069BDE870
:10898000F08123695A1C2261234415F8011B1973D5
:10899000042AF1D139462046FFF73DFFC4E904809F
:1089A000EAE74FF0FF30EAE72DE9F347038A8689CB
:1089B000B6B205460C461E404FF0004901F14C0787
:1089C00001F1340816B902B0BDE8F087B6FA86F3B3
:1089D00029FA03F2D24391B2298216401B3B002CA4
:1089E00040D0042BEED8DFE803F039342E28030002
:1089F000E368D5F82CA02BB19B681BB11FFA8AF154
:108A0000201D9847636A33B19B6823B11FFA8AF12E
:108A100004F11C009847E36B2BB19B681BB11FFA54
:108A20008AF140469847636D002BCBD09B68002BA2
:108A3000C8D01FFA8AF1384603E0E368696B5B68C7
:108A4000201D9847BEE7636AA96B5B6804F11C00B0
:108A5000F7E7E36BE96B5B684046F2E7636D296C0F
:108A60005B68E8E7042B06D8DFE803F00D0B090785
:108A70000300EB6A0193019BA4E76B6BFAE7AB6B16
:108A8000F8E7EB6BF6E72B6CF4E790F84820531C03
:108A90000244DBB280F8483082F8341090F8492064
:108AA0000AB1132B01D94FF008BD7047002280F89E
:108AB00049204FF002BD70B50F4E96F88B3A002B4F
:108AC000FBD104464518AC4201D1002070BDD6F858
:108AD0002C3914F8011BF2180133C3F30A0382F88E
:108AE0008C1AC6F82C39FFF7C9FC0028EBD10120FD
:108AF0000AF0BAFBF7E700BF3818002038B50C467B
:108B00001146FFF7A3FB48B1054D002AD5F8943173
:108B100004DD2046FFF7CFFFD5F8943138BD00BF04
:108B200030290020F0B590F8CF5590F8CE1590F888
:108B3000D12590F8D03590F8CC7590F8CDC501EBE3
:108B400005218DB203EB022390F8D31590F8D225BE
:108B500085B002EB012207F01F06012192B29BB201
:108B60008E4204468DF808708DF809C0ADF80A50A1
:108B7000ADF80C30ADF80E20C0F8402180F811118E
:108B800000F00C81022E00F01D81002E40F09B8130
:108B9000BCF1090F5ED8DFE81CF0B600F4005D0000
:108BA000C8005D0057000A005D00A90076002E0A8B
:108BB000022EADF806200BD0032E25D0012E49D170
:108BC000D0F8EC351B68A0780DF10601984709E054
:108BD000D0F8E43580789B6A0DF10601984746701D
:108BE000C4F8F005BDF80620002A47D0BDF80E30C5
:108BF000002B43D09A4228BF1A46ADF80620014602
:108C000020464EF06FFF39E0E9B2052922D8DFE8AF
:108C100001F003070B0F1317D0F8EC355B68D2E7B0
:108C2000D0F8EC359B68CEE7D0F8EC35DB68CAE7C6
:108C3000D0F8EC351B69C6E7D0F8EC355B69C2E7C4
:108C4000D0F8EC359B69BEE71A4303D190F8123196
:108C5000032B03D120464EF071FE0FE0016905F0B1
:108C60007F0680F814610B6865F30A121A430A60E4
:108C70004EF04CFF2EB1022384F81231002005B0D3
:108C8000F0BD0123F8E7E9B2904D012985F898116C
:108C9000E0D890F81231022B0FD0032BDAD1C1B9F2
:108CA000022380F81231D0F8E43580F810115B68A7
:108CB000984720464EF02AFFE0E70029F9D001212D
:108CC000032380F8101180F8123120464EF0F8FD91
:108CD000EFE790F810110129EBD0D0F8E4355B688C
:108CE000984795F8981184F81011EEE7012AB1D150
:108CF00090F81231022B04D0032BABD100F5887110
:108D00007EE773497CE790F81231023B012BA1D832
:108D10006E4B0022C3F8A021D0F8182112B1022214
:108D2000C3F8A0216B4902226AE7012D08D1C0F8DF
:108D30001851D4F8E43502A99B6820469847B8E753
:108D4000022D9BD1DAB2002A98D102691B0A023B9C
:108D50005268032B03D8DFE803F00C0E1012012336
:108D600063F30612594BC3F8A421012384F816318A
:108D70009FE70223F4E70323F2E70423F0E7052348
:108D8000EEE790F81231023B012B3FF663AF012D65
:108D90007FF474AF0023C0F81831CAE790F81221AD
:108DA000032A7FF457AFDBB2012B3FF653AFD0F865
:108DB000E43502A99B689847BDF80E30002B7FF47C
:108DC0005DAF76E707F06007202FD9B205D1D0F864
:108DD000E43502A99B68984750E7BCF1010F31D0F8
:108DE000BCF1030F1ED0BCF1000F7FF447AF90F829
:108DF0001221022A5AD0032A7FF42CAF13F0800FDD
:108E00004FF02802314B59D001F07F0102FB0101E4
:108E100091F81E21002A4FD00122C3F8A8212E4923
:108E20000222EDE690F81231022B3FD0032B7FF4A3
:108E300011AF002D7FF47DAF4A063FF47AAF4EF0BC
:108E40004BFD76E790F81221022A2FD0032A7FF4F7
:108E500001AF002D7FF412AF11F07F003FF429AF76
:108E60005BB2002B4FF02802B5BF02FB004102FBB2
:108E7000014101F58E7101F55D710022DB0F087073
:108E80008A704B7004EB8000C9786BB182691368FB
:108E900002396FF3555301298CBFC3F300710121CF
:108EA00061F31C73136044E7426DF0E74B063FF437
:108EB000E5AE4EF011FDE1E60022AEE702FB010156
:108EC00091F87623A6E707F08001F2E73029002029
:108ED000CC2A0020D02A0020D82A002010B5044631
:108EE00071BB90F81131032B1BD1D0F89023D0F82F
:108EF0007C339A4217D9C178012908BFD0F8801372
:108F0000A2EB030204BFC918C0F88013934228BF24
:108F10001346C0F890239BB2D0F8802300214EF076
:108F2000A5FE002010BDD0F8E4351B6923B190F8F0
:108F30001221032A00D1984720464EF0E7FDF0E7C2
:108F4000D0F8E4359B69002BEBD090F81221032A6E
:108F5000E7D19847E5E770B50A7812F06004064655
:108F60000D462AD0202C2FD1CC884B78FCB112068C
:108F70000CD51F4922461846FFF73EFAEA881C49DD
:108F800030464EF0AFFD0024204670BD194A1360F4
:108F9000194A0323C2F80C4880F81131C0E9E444AF
:108FA000234602F5016200214EF060FEEBE702224B
:108FB00011441846FFF720FAE6E74B780A2B08D051
:108FC0000B2B0BD0062BDFD130464EF0B7FC022422
:108FD000DAE70A4901224EF085FDD5E78B781BB907
:108FE000074BC3F8AC41CFE74EF0A8FCCCE700BF7D
:108FF000482000200000002038180020DC2A002033
:109000003029002010B5282303FB0101074AB1F8DD
:109010008C1304461046FFF744FA2046034A4023C7
:1090200001214EF023FE002010BD00BFE02A0020E9
:1090300070B50F4DD5F8F831044643B195F8FC21D1
:1090400095F81032134302D101214EF045FC8121E5
:1090500020464EF041FC95F81032022B07D12046F5
:10906000044ABDE870401F2301214EF0FFBD70BDD2
:1090700030290020202B0020002310B5194604467B
:1090800040224EF092FC40228021204600234EF0E8
:109090008CFC012384F81231D4F8E835A0785B68A1
:1090A0009847002010BD38B5402204460223812194
:1090B0004EF07BFC20460223402201214EF075FC3D
:1090C00020460323082282214EF06FFC084B022227
:1090D000002583F84B2083F84C50FFF779F90121E4
:1090E0002046044A40234EF0C1FD284638BD00BF4B
:1090F00000000020E02A002010B5812104464EF037
:109100002BFC204601214EF027FC204682214EF008
:1091100023FCFFF769F9002010BD10B5812104463A
:109120004EF01AFC204601214EF016FC024B0020A6
:1091300083F8110210BD00BF3029002038B5264C3D
:1091400094F88B2A012A034633D12448D0F81422FC
:109150001AB984F88B2A002038BD402AD4F828197F
:1091600019D9403A01F14005C0F81422C4F8285931
:1091700040221B4810FA81F1C3E9541140F201105A
:109180000021C3E95621A3F8440103F5A271184652
:109190004EF0D3FCDFE702EB0105C4F828594FF08D
:1091A0000005C0F814520ABF022092B284F88B0A5C
:1091B000DFE7022ACFD1002540F20112C0E9545561
:1091C000C0E95655A0F8442100F5A2714EF0B5FC57
:1091D00084F88B5ABFE700BF3818002030290020E0
:1091E000C422002038B52A4CD4F818320F2B03F1D2
:1091F000010203D0C4F81822002038BD254A0023FC
:10920000C4F8183292F88B3A002BF5D1D2F828190D
:10921000B1F5006F08BFC2F82839D2F82819D2F882
:109220002C39994203D1002382F88B3AE4E78CBFB2
:10923000C1F500635B1A402B1BD9403B01F140058F
:10924000C4F81432012382F88B3AC2F8285940231B
:10925000114A12FA81F140F20112A0F844210022D1
:10926000C0E95411C0E9563200F5A2714EF065FC18
:10927000C2E701EB0305C2F828594FF00005C4F816
:1092800014520EBF022401249BB282F88B4ADFE7FE
:109290003029002038180020C4220020064BD3F8C3
:1092A00088391A79022A05D19A68920702D5586935
:1092B0004EF05CB8704700BF3818002010B50A4C5B
:1092C000D4F8880906F06AFC58B9D4F888090379FB
:1092D000022B08D183689B0705D5BDE8104008F034
:1092E000F1B800BFECE710BD3818002073B50A4E86
:1092F000441C0025D6F88809012300220DF107013E
:109300004FF01FF99DF80700FF2802D10135A54253
:10931000F0D102B070BD00BF3818002037B5044648
:1093200008200191FFF7E2FFFF2813D0FE2813D198
:109330000A4D019BD5F88809002221464FF001F91A
:109340000022D5F88809022311464FF0FAF80020D0
:1093500003B030BD0120FBE70220F9E738180020F8
:1093600037B5124D4FF6FF530024D5F88809ADF8F4
:10937000043001AA02232146C5F854494FF0E1F810
:109380000120FFF7B3FFFF2805D1042385F85839E2
:10939000022003B030BD092385F85839044BD3F8B7
:1093A0009431C5F848392046F3E700BF381800204B
:1093B0003029002013B540F040038DF800300B0E2B
:1093C0008DF801300B0C8DF802300B0A8DF803304C
:1093D000952304468DF804108DF805304FF0D6F82B
:1093E00000B964B907480623D0F888096A46002105
:1093F0004FF0A7F80820FFF779FF02B010BDFF205B
:10940000FBE700BF381800202DE9F041194C1E463B
:1094100094F85839042B0546884617461CD1FFF7A7
:109420003DFF94F84E3903BB69021120FFF7C2FFDC
:10943000E8B9052384F858390F4BC4F83489D3F8B8
:109440009431C4F83859C4F84079C4F84469C4F870
:1094500048390120BDE8F081082B01D00020F9E750
:10946000FFF77EFF0228F9D1D9E72946DDE7FFF7AC
:1094700025FFF3E7381800203029002038B50022F6
:109480000D233421022006F0E5FE234CC4F88809A0
:1094900010B984F8580938BD002106F005FA0120FA
:1094A00009F0E2FED4F888391C4D586906F0B0FC8A
:1094B000D4F888391A4893F91030142202FB0300BB
:1094C0000022D0F8B0000A2311464FF00FF8D4F86C
:1094D000880906F063FB50B9124B84F84C09D3F8A5
:1094E0009431C4F84839012384F85839D3E7013D51
:1094F000EDD1D4F88809022106F0D6F9D4F888090C
:1095000006F0A5F994F84C39C4F88859013384F869
:10951000585984F84C39BEE738180020A18601005C
:10952000000000203029002038B5134C0023A07B18
:10953000E0B125688D4219D1104C03F581751AB937
:1095400004EB0514A27138BD04F1180101EB4323AB
:109550009A4209D1831E5842584104EB05144EF03B
:10956000BDF80123A371EEE70020F6E70133082BD5
:1095700004F11004DBD1E6E71C5F0020044F00205B
:10958000174838B5002380F8A03000F1180425688A
:109590008D421ED1A57B032D1BD1124C03F5817585
:1095A0004AB904EB05140423A371D0F89C300133AD
:1095B000C0F89C3038BD04F1180000EB4320131AAA
:1095C0005842584104EB05144EF088F80123A3716A
:1095D000F0E70133082B04F11004D8D1EAE700BF0B
:1095E000045F0020044F002070B50446144EFFF7BE
:1095F00094FD20460223402281214EF0D6F94022DC
:109600000121204602234EF0D0F90025D6F81C3265
:1096100086F811521B6886F8105228469847E06871
:109620004EF06EFDE06801214EF080FD20461F23C4
:1096300006F5F87201214EF019FB284670BD00BFF7
:10964000302900202DE9F84F0E4601210846174623
:109650001D4606F081FFDFF844800024A54206DCA9
:109660000021012006F078FF0020BDE8F88F06EB0E
:10967000442A04EB0709D8F8303903B9FEE7D3F8D8
:1096800004B000231A4651464846D8470028F2D075
:10969000FEF72AFF0028FBD00134DFE7381800204E
:1096A0002DE9F84F0E460121084615461F4606F0E3
:1096B00053FFDFF848A00024A74218DD06EB442939
:1096C00005EB040801E0FEF70FFFDAF8303943B18B
:1096D000D3F80CB000231A4649464046D847002824
:1096E000F1D1FEF701FF0028FBD00134E4E70021AF
:1096F000012006F031FF0020BDE8F88F3818002067
:10970000024BD3F8200207F004BE00BF302900202E
:109710000068F022FF2107F003BFCA4341EA0212AA
:109720000068D2B2D22107F0FBBE0068B422FF214C
:1097300007F0F6BE0A460068A52107F0F1BE5521E4
:10974000F8E700689622FF2107F0EABE0A460068A3
:10975000872107F0E5BEC90101F080020068782189
:1097600007F0DEBE38B50446154600680A46E1211A
:1097700007F0D6FE30B120682A46FF21BDE8384008
:1097800008F0CABD38BD0A46E121EBE70A46C3210D
:10979000E8E738B5021D0D46F0210446FFF7E2FF69
:1097A00008B123792B7038BDF8B504460E4615462E
:1097B000071D20683A46FF2108F0AEFD30B116B112
:1097C0002379DB07F5D40DB123792B70F8BD002286
:1097D0000121E9E710B50446FFF7A7FF18B12046BD
:1097E000BDE81040F3E710BD10B50446FFF7A2FF37
:1097F00018B12046BDE81040E9E710BD70B5064637
:109800000C468D18AC4201D1012006E014F8011B72
:109810003046FFF7E9FF0028F4D170BDCC21E3E723
:1098200038B504460D46FFF78CFF40B12046FFF7E0
:10983000CEFF20B129462046BDE83840A3E70020EE
:1098400038BD70B506460C468D18AC4201D10120DA
:1098500006E021463046FFF7E3FF01340028F4D14B
:1098600070BD38B505461446FFF770FF2846FFF770
:10987000AEFF20B11CB12B79C3F34013237038BD68
:1098800010B50446FFF7A6FF38B12046FFF7C6FF24
:1098900018B12046BDE8104099E7002010BD73B50F
:1098A0000546CDE90023FFF795FFA8B12846FFF74D
:1098B00046FF88B12846FFF78AFF68B16E46082444
:1098C00016F8011B2846FFF78FFF28B1013C14F062
:1098D000FF04F5D102B070BD0020FBE7C90138B527
:1098E00001F0800104461546FFF735FF08B9002056
:1098F00038BD002201212046FFF756FF0028F6D090
:1099000023795B092B70F3E710B5021D0446FF2194
:10991000006808F001FD18B12079C04300F0010093
:1099200010BD0F49D1F8883043F47003C1F8883076
:109930000C4B1A68002042F001021A6098601A6805
:1099400022F0847222F480321A60074A5A601A6840
:1099500022F480221A60D860044B8B60704700BFED
:1099600000ED00E000380240103000240000000844
:1099700070470028ACBF00F16040074B4FEA01116F
:10998000ACBF00F5614000F00F00C9B2B4BF19547C
:1099900080F80013704700BF14ED00E02DE9F04798
:1099A0009846414B914603EB800205469468002C93
:1099B00078D02833636004F13E03A36104F59F73FC
:1099C000E3614FF48073C4E90433236894F83D00E5
:1099D000E160A36306F090FA064694F8440294F816
:1099E0003CA0271D08B14BF071FA94F8450208B16C
:1099F0004BF06CFAD4F840321BB12C4A116B0B437C
:109A0000136318F0080F2CD00135EDB21EB140F2EF
:109A10000673F380357218F0100F94F846221AD0AE
:109A20000221304606F028FAD4F8481294F9470289
:109A3000FFF79FFF94F9473294F84722002B07DB8A
:109A400002F01F0101228A405B09194941F82320D5
:109A50003846BDE8F08718F0200F14BF12213221DC
:109A6000DFE719F0020F0CD06B1CDBB21EB140F225
:109A70000652F280337294F846220221304606F0F4
:109A8000FBF919F0010FCFD0504606F035FA013539
:109A9000EDB218B140F20663C380057294F8462215
:109AA0000221BFE72746D3E7D41106080038024059
:109AB00000E100E00148FEF7E0BA00BF0401002029
:109AC0000148FEF7DABA00BF50030020024B586F7E
:109AD000C0F30070704700BF003802407047064A6C
:109AE000002352F83310814201D1D8B270470133BC
:109AF0000E2BF6D1FE2070472C120608704770B569
:109B0000002828D04C684CB9426815685679AB8952
:109B100002229BB2B24023EA0203AB818A683AB9BF
:109B200043681D68AB8923F001031B041B0CAB8148
:109B3000816044B14468216864798D890223A3401F
:109B40002B439BB28B8132B143681A6893899BB2D5
:109B500043F00103938170BD0B4B30B51A460024CE
:109B60001D79854208D1DD68294203D0142000FB0D
:109B7000042030BD0029F9D001340A2C03F114036C
:109B8000EED10020F5E700BF9805002038B5036846
:109B90001B681C68254B03F5CC6393ED007A07EE38
:109BA000902AB8EE477AF8EE677A013987EE270AED
:109BB0008DB2DFED1F7A30EE270A50F033FB1D4ADD
:109BC00023880138944280B29BB212D002F58062A1
:109BD00094420ED0B4F1804F0BD0A2F58032944263
:109BE00007D002F58062944203D002F5806294426D
:109BF00002D123F070039BB20F4A944206D002F5C3
:109C0000806294421CBF23F440739BB22380094BB3
:109C1000E5629C42208503D003F580639C4201D11C
:109C2000002323860123A38238BD00BF000000204B
:109C30000AD7233C00000140001000402DE9F0430A
:109C40004568A87910F0040300F002020BD0002050
:109C500017468046042406466B79032B49D8DFE873
:109C600003F0094A89C990464FF480701F461C468C
:109C70000126F1E72D682B8C23F001031B041B0C3C
:109C80002B84B5F820C0B5F804902B8B23F0730318
:109C90001B041B0C43F0600E2CF0020C6E4B4FEAC1
:109CA0000C4C4FEA1C4C48EA06069D421FFA89F903
:109CB0004CEA060C03D003F580639D420AD14FF6AF
:109CC000F3730CEA03033B4329F4407943EA040CA1
:109CD00040EA0909A5F80490A5F818E06963A5F819
:109CE00020C02B8B23F008031B041B0C43F008033C
:109CF0002B83BDE8F0832D682B8C23F010031B040D
:109D00001B0C2B842A8CB5F804E0B5F818C0524B14
:109D10002CF4E64C22F020024FEA0C4C12044FEADD
:109D20001C4C120C48EA06069D421FFA8EFE4CF4AB
:109D3000C04C42EA061203D003F580639D420BD16A
:109D400022F0800242EA071222F040022EF4406E16
:109D500042EA04124EEA800EA5F804E0A5F818C005
:109D6000A9632A842B8B23F400631B041B0C43F48C
:109D70000063BDE72D682B8C23F480731B041B0C40
:109D80002B842A8CB5F804E0B5F81CC022F40073CB
:109D90002CF0730C304A4FEA0C4C1B044FEA1C4C5D
:109DA0001B0C48EA060695421FFA8EFE4CF0600C2A
:109DB00043EA062303D002F5806295420BD123F4D7
:109DC000006343EA072323F480632EF4405E43EAF2
:109DD00004234EEA001EA5F804E0A5F81CC0E963C0
:109DE0002B84AB8B23F008031B041B0C43F00803EC
:109DF000AB837EE72C68238C23F480531B041B0C5D
:109E00002384258CA288A38B25F400552D0448EAD1
:109E100006062D0C23F4E64345EA06350E4E1B04D8
:109E20001B0CB44292B243F4C04303D006F58066E3
:109E3000B44203D122F4804242EA8012A280A3837A
:109E400021642584A38B23F400631B041B0C43F4BF
:109E50000063A3834DE700BF0000014043685A79C7
:109E6000032A0FD8DFE802F00205080B1868343027
:109E7000704718683830704718683C307047186869
:109E8000403070470020704710B543681A68587911
:109E9000084B0344012093F8C840138CA0409BB2A8
:109EA00023EA00031384138CA140194389B211845F
:109EB00010BD00BFD4110608F0B5EFF311841023D4
:109EC00083F31288C5684668AA68136823F0010303
:109ED000136032687779104E938936F817609BB219
:109EE00023EA060393812A696D681F2A4FF0200335
:109EF00085BF203A93409340EB6098BFAB60E3B2DC
:109F000083F31188C3689B6859601A6842F00102A4
:109F10001A6001230374F0BDD41106080268137D92
:109F2000012B04BF0223137592F82C100CBF4FF4C1
:109F300000730023012904BF022182F82C1092F83B
:109F4000441008BF43F48063012904BF022182F852
:109F5000441092F85C1008BF43F4006301290DD14E
:109F6000022182F85C1043F4805342681168002299
:109F70004A628A8992B213438B8101E0002BF4D1AB
:109F80007047034B0348D3F82412FEF70DBD00BF02
:109F9000302900200000014010B5064C0648D4F8D6
:109FA0002412FEF701FDD4F844120448BDE8104025
:109FB000FEF7FABC302900200000014000400140BB
:109FC00010B5064C0648D4F82412FEF7EDFCD4F880
:109FD00048120448BDE81040FEF7E6BC30290020D6
:109FE000000001400044014010B5064C0648D4F87A
:109FF0002412FEF7D9FCD4F84C120448BDE81040F6
:10A00000FEF7D2BC3029002000000140004801408A
:10A01000034B4FF08040D3F82812FEF7C5BC00BFB9
:10A0200030290020024B0348D3F82C12FEF7BCBCA9
:10A030003029002000040040024B0348D3F83012BE
:10A04000FEF7B2BC3029002000080040024B034854
:10A05000D3F83412FEF7A8BC30290020000C0040D1
:10A060000348D0F8703613B100F2646018477047A7
:10A07000000000200348D0F8903613B100F284604D
:10A0800018477047000000200348D0F8B03613B1DD
:10A0900000F2A46018477047000000200348D0F881
:10A0A000D03613B100F2C46018477047000000209A
:10A0B0000348D0F8F03613B100F2E4601847704757
:10A0C000000000200348D0F8103713B100F20470EC
:10A0D00018477047000000200348D0F8303713B10C
:10A0E00000F2247018477047000000200348D0F8A1
:10A0F000503713B100F24470184770470000002039
:10A100000348D0F8703713B100F2647018477047F5
:10A11000000000200348D0F8903713B100F284709B
:10A1200018477047000000200348D0F8B03713B13B
:10A1300000F2A47018477047000000200348D0F8D0
:10A14000D03713B100F2C4701847704700000020E8
:10A150000348D0F8F03713B100F2E47018477047A5
:10A16000000000200348D0F8103813B100F60400B6
:10A1700018477047000000200348D0F8303813B16A
:10A1800000F6240018477047000000200348D0F86C
:10A19000503813B100F64400184770470000002003
:10A1A000036823F0010303600023036043608360BE
:10A1B000C3600361212343612A4B984203D13D22AE
:10A1C00043F8082C7047284B984204D14FF474622E
:10A1D00043F8202C7047254B984204D14FF4741259
:10A1E00043F8382C7047224B984204D14FF07462E8
:10A1F00043F8502C70471F4B984203D11E4A43F836
:10A20000642C70471D4B984203D11D4A43F87C2CA7
:10A2100070471C4B984203D11B4A43F8942C70475B
:10A220001A4B984204D14FF03D5243F8AC2C17E042
:10A23000174B9842C3D0174B9842C7D0164B984241
:10A24000CCD0164B9842D1D0154B9842D6D0154B56
:10A250009842DAD0144B9842DED0144B9842E2D0A8
:10A26000704700BF1060024028600240406002401A
:10A2700058600240706002403D000020886002404B
:10A28000400F0020A060024000003D20B860024066
:10A290001064024028640240406402405864024056
:10A2A0007064024088640240A0640240B8640240C6
:10A2B0002DE9F0410022012603250B6806FA02FC75
:10A2C0003CEA030331D10368540005FA04FE23EA93
:10A2D0000E0303600B79D0F800806FEA0E0703FAD3
:10A2E00004FE013B4EEA080E012BC0F800E011D835
:10A2F00083681F4087604B798768A3403B43836036
:10A30000436823EA0C0343608B79476893409BB210
:10A310003B434360C36805FA04F723EA0703C360BD
:10A32000CB79C768A3403B43C3600132102AC4D134
:10A33000BDE8F081204A936803F00C03042B10B5AC
:10A3400020D0082B20D01D4B1B4C0360A3681C4A57
:10A35000C3F30313134493F864180368CB404360BA
:10A36000A168C1F38221114491F8641823FA01F124
:10A370008160A168C1F342310A4492F86428D34055
:10A38000C36010BD0F4BDFE75368516813F4800FB3
:10A3900001F03F01536814BF0A4A084AB2FBF1F1C9
:10A3A000054A5268C2F30142C3F3881301324B439A
:10A3B0005200B3FBF2F3C7E7003802400024F40078
:10A3C0000000002040787D01F0B5446B8668A389C9
:10A3D00023F400531B041B0CA3818279278A0546B2
:10A3E000BFB2100312F0040F4FEA022100F4005034
:10A3F0006A7927F4405740EA0700208214BF4FF4DF
:10A40000805C4FF0000C12F0010F0CBF00230423FE
:10A410009207A28922F4B05201F4806122F00C026A
:10A4200048BF43F0080341EA0C0112040B43120C2D
:10A430001A43A281A38A23F440731B041B0C85B02A
:10A44000A3826846FFF776FF214B9C4203D003F5B9
:10A4500080639C423AD1039BA2891921170401FB16
:10A4600003F34FF064014CBF7600B600B3FBF6F384
:10A47000B3FBF1F001FB10330201A08900044BBFD4
:10A48000DB001B01323332334BBFB3FBF1F3B3FBC1
:10A49000F1F303F0070303F00F0313439BB223818F
:10A4A0006A6BAB7913F0080F938A0BBF23F0080394
:10A4B0009BB21B0443F0080308BF1B0C93829389D3
:10A4C0009BB243F40053938105B0F0BD029BC3E7F8
:10A4D000001001402DE9F8431E46204B9DF8205006
:10A4E0009DF824709842894690462CD13B462A46D6
:10A4F00031460020FFF752FA04460020C4E9070065
:10A50000C4E90900C4E90B986571A660A7712046EB
:10A51000FFF75AFFEA0707D5636B4FF6DF721A8021
:10A52000DA6842F02002DA60626BAB0742BFD368A0
:10A5300043F08003D36093899BB243F4005393812B
:10A540002046BDE8F883064B984204D13B462A4694
:10A5500031460120CEE70024F2E700BF00100140A1
:10A560000044004081602FE741712DE72DE9F04361
:10A57000654F07EBC00985B005464FEAC00899F85A
:10A58000780805F0B9FC064699F8790805F0B4FC9E
:10A59000044699F87A084AF099FC6B1CDBB21EB1AC
:10A5A00040F60C12F28033721CB140F60C22E280AD
:10A5B000237204223A21304605F05EFC2046042234
:10A5C0003A2105F059FC07EB0803D3F874484F4BC8
:10A5D0009C4263D103F5F2331A6A42F400121A6204
:10A5E0001A6A22F400121A62474497F87B38022B49
:10A5F0006ED0032B6ED0464E464A012B08BF16463E
:10A60000A78827F03F0768463F04FFF793FE3F0CFB
:10A61000029A414BB2FBF3F398B20743A78021881B
:10A6200021F001010904090C21803C498E4253D1DB
:10A630003B4BB2FBF3F2013092B2042A80B238BF36
:10A6400004222084A28323889BB243F00103238049
:10A65000238823F4816323F002031B041B0C43F4BF
:10A66000806323804FF480432381238823F0800379
:10A670001B041B0C238023889BB243F0010323801F
:10A68000284B03EB4513012283F86122002283F853
:10A69000605283F8622205B0BDE8F083224B9C42F1
:10A6A00009D103F5F0331A6A42F480021A621A6A79
:10A6B00022F4800297E71D4B9C4295D103F5EE33BF
:10A6C0001A6A42F400021A621A6A22F400028AE745
:10A6D000124E95E7124E93E706EB4606B2FBF6F2F2
:10A6E00091B2C2F30B020AB941F0010141F40042F8
:10A6F0004FF496714B434FF47A71B3FBF1F301338E
:10A700009BB223849EE700BF00000020005400405D
:10A71000801A060000350C0040420F00A0860100A0
:10A72000400D03003029002000580040005C00402C
:10A730002DE9F047B74D460105EB401908F0B8FC8C
:10A7400099F96022B44B8846D10003EBC202074658
:10A75000D2F8744899F86222013A142A00F28380F0
:10A76000DFE812F0790089009F00B700C200CC003A
:10A77000D500EA00F5000A01150164017D01A3017D
:10A7800006021702290232024302670215005F180F
:10A790004FF0090A97F8780805F0AEFB044697F8E1
:10A7A000790805F0A9FBB5F8C03201339BB2074622
:10A7B0002046A5F8C03205F02BFB384605F028FBF3
:10A7C0001121204605F02EFB1121384605F02AFB09
:10A7D0004FF0650803E00520002108F0A9FC2046A1
:10A7E00005F00DFB10B9B8F10108F4D1204605F0D1
:10A7F00014FB0021052008F09BFC204605F008FB17
:10A800000520002108F094FCBAF1010AE0D12046AD
:10A8100005F003FB0021052008F08AFC384605F00E
:10A82000FCFA0021052008F083FC204605F0F0FA30
:10A830000520002108F07CFC384605F0E9FAAB1948
:10A8400093F96002431C01D0FFF790FEAB19002280
:10A8500083F8622207E0238813F4007340F0238119
:10A86000AA1982F86232AB1993F86232002B7FF496
:10A8700065AFBDE8F087238823F400631B041B0C3D
:10A88000238023889BB243F48063238023889BB278
:10A8900043F480732380AB19C3E99A78032283F8C9
:10A8A00062225E492046FDF790FCAB19002855D086
:10A8B00093F872225AB993F87322FF2A04D193F8BD
:10A8C00070220AB10A22C3E7AB190422C0E70F22A3
:10A8D000BEE7AB1993F8712202F0FE022282C3E9AF
:10A8E0009A78052283F862224D492046FDF76DFCD7
:10A8F000002800F07081AB190622A9E7AB1993F884
:10A9000073222282C3E99A78072283F8622245499A
:10A910002046FDF75AFC002800F05D81AB19D3F802
:10A9200074223AB9228892B242F400722280C3E9BA
:10A930009A780EE108228BE723889BB243F4807358
:10A940002380AB19C3E99A78092283F8622233493C
:10A950002046FDF73AFCAB190028B3D1D3E99A01A0
:10A9600042F21072381A68EB0101904271F1000254
:10A97000FFF479AF15226BE7AB1993F8712242F01F
:10A9800001022282C3E99A780B2283F862222649C7
:10A990002046FDF71AFC002800F01D81AA19D2F804
:10A9A0007432012B1AD1238823F480631B041B0CFF
:10A9B0002380EFF31181102383F31288238B2388E4
:10A9C0009BB243F400732380CBB283F311880C2332
:10A9D00082F86232AB19C3E99A7844E7022B15D1A9
:10A9E00023889BB243F400632380EFF3118110238B
:10A9F00083F31288238B238823F480631B041B0CAE
:10AA00002380CBB283F311880D23E1E7238B0E2340
:10AA1000DEE700BF30290020000000200100030015
:10AA200082000700840007000200030086492046D8
:10AA3000FDF7D6FBAB19002890D0D3F87822511C33
:10AA4000C3F87812218A1170D3F87422013AC3F83E
:10AA500074220122C3E99A7883F87C22F8E67B49C4
:10AA60002046FDF7BDFBF0B1EFF31182102383F315
:10AA7000128823889BB243F400732380AB19D2B2AF
:10AA8000D3F87812481CC3F87802208A087082F341
:10AA90001188D3F87822511CC3F87812218A1170DA
:10AAA0006FF00102D3E7AB1958E768492046FDF77C
:10AAB00097FBAB1900283FF451AFD3F87422032A57
:10AAC00003F51A7130D1228822F480621204120C2C
:10AAD0002280EFF31180102282F31288D3F87822BB
:10AAE00002F1010CC3F878C2B4F810C082F800C0BB
:10AAF000228892B242F400722280C2B282F311889C
:10AB0000D3F87822501CC3F87802208A1070D3F84A
:10AB10007422023AC3F874220C2283F86222C3F82A
:10AB20006872C1F804809EE6022A14D8228822F4B2
:10AB300080621204120C2280228892B242F40072C7
:10AB40002280228AC3F86872002283F87C22C1F82E
:10AB5000048001227CE6D3F87822501CC3F87802E6
:10AB6000208A1070D3F87422013AC3F87422D6E711
:10AB7000238823F480631B041B0C2380AB1993F8F8
:10AB8000712202F0FE022282C3E99A78102283F831
:10AB900062222F492046FDF718FBE0B1AB1993F86C
:10ABA0007322FF2A04D193F870220AB113224FE6D0
:10ABB000AB1911224CE6AB1993F873222282C3E938
:10ABC0009A78122283F8622222492046FDF7FDFA84
:10ABD00008B1AB19EAE720492046FDF701FBAB19A4
:10ABE00000283FF4BBAE142232E6AB1903F51A700D
:10ABF000D3F8742282B1D3F87812013A11F801CB5C
:10AC0000A4F810C0C3F87422C3F86872C3F87812AD
:10AC1000C0F8048012221BE6228892B242F400722D
:10AC200022800122C3F8687283F87C22C0F8048075
:10AC30000EE623889BB243F4007323804FF6FF3364
:10AC4000A382AB1973E600BF40000010040000109F
:10AC500082000700840007000004001038B5114C82
:10AC600004EB401494F86152D5B1C4F87432049BDB
:10AC7000C4F87832002384F87C320223490084F837
:10AC8000732284F8623201229DF8143084F8711224
:10AC900084F8722284F87032FFF74AFD94F87C52EF
:10ACA000284638BD3029002038B5114C04EB40143B
:10ACB00094F86152CDB1C4F87432049BC4F8783270
:10ACC0000223490084F8732284F8623200229DF83E
:10ACD000143084F8711284F8722284F87C2284F88B
:10ACE0007032FFF725FD94F87C52284638BD00BF2E
:10ACF00030290020F0B587B0002300930193744BF6
:10AD00001A6842F480321A601A6802F40032019222
:10AD1000009A01320092019A1AB9009AB2F5A04F36
:10AD2000F2D11B6813F4003318BF01230193019B78
:10AD3000012B40F0B180664B66491A6C42F080529C
:10AD40001A640A6842F440420A609A689A609A68F3
:10AD50009A609A6842F480529A605F4A5A601A6810
:10AD600042F080721A601A689201FCD55B4A40F288
:10AD7000027111609A6822F003029A609A6842F0A8
:10AD800002029A60524A936803F00C03082BFAD12E
:10AD90009368534C03F00C03042B7FD0082B7FD017
:10ADA000504BC4F860364A4B4F4D9A684F48C2F337
:10ADB00003122244002692F88C18D4F86026CA4068
:10ADC000C4F860264A4AEA605A6F4A4AAA605A6B37
:10ADD00022F080025A635A6F42F080725A67196BF0
:10ADE000454A0A431A635A6B5A631A6C42F08752F7
:10ADF00042F4F61242F41F6242F00F021A64596CD8
:10AE00003E4A0A435A6402A948F2FF73CDE902366A
:10AE10004FF6FF77FFF74CFA00F580600297FFF7D7
:10AE200047FA00F580600297FFF742FA00F580606C
:10AE3000FFF73EFA00F58060FFF73AFA0846FFF7A1
:10AE400079FA029B2E4AB3FBF2F32E4AC2F8C432BF
:10AE5000D5F8FC302C4A43F08073C5F8FC302B4BFE
:10AE6000C3F8B02F5E601A6842F001021A60D4F88D
:10AE700060364FF47A72B3FBF2F3013BB3F1807F9B
:10AE800008D24FF0E0225361F02385F823300723E6
:10AE90009661136107B0F0BD00BFFDE71C4B80E772
:10AEA0005368516813F4800F01F03F01536814BFD9
:10AEB000174A0C4AB2FBF1F1054A5268C2F301424B
:10AEC000C3F3881301324B435200B3FBF2F368E73C
:10AED000003802400070004019304004003C02403D
:10AEE000000000200024F40000ED00E0000002401B
:10AEF0000003FA05000000081F90670033570700A1
:10AF000040420F003029002055CEACC5001000E0B3
:10AF100040787D0182B000230193054B0193019B92
:10AF200003EB80000190019B196002B0704700BFE5
:10AF30005028004082B000230193054B0193019BF0
:10AF400003EB80000190019B186802B0704700BFBE
:10AF50005028004010B51C2004F0CEFF11210446FB
:10AF600004F060FF204604F058FFC82008F07CF988
:10AF70002046BDE8104004F04BBF436D064A1A61FD
:10AF8000C278012A06D100F2CC5058611A684FF0FD
:10AF900080221A60704700BF1800086038B5044668
:10AFA00000296FD190F81131022B2AD1D0F8382125
:10AFB000D0F824118A4232D9C378012B04BFD0F8CB
:10AFC00028315B18A2EB010208BFC0F828314FF40A
:10AFD0008071D0F82831C0F83821002592B2A0F84D
:10AFE0001C11C0F82C31C0F83451C0F8302100F5E4
:10AFF0008E714CF025FD2B462A46294620464CF002
:10B0000035FE94F81631012B07D1244A2369D2F872
:10B01000A4215A60002384F81631002038BDD0F8EE
:10B020003C31B3FBF1F501FB1535A5B9994212D8B6
:10B03000D0F8402193420ED24FF48073C0E94A55B4
:10B04000C0E94C55A0F81C3100F58E714CF0F8FCAD
:10B05000C4F84051CFE7D4F8E435DB682BB194F85D
:10B060001221032A01D120469847052384F8113183
:10B07000002320461A4619464CF0F8FD2046FFF7FB
:10B080007CFFBEE7D0F8E4355B69002BC5D090F8B3
:10B090001221032AC1D19847BFE700BF3029002001
:10B0A00070477047704710B5114C94F8D232CBB14D
:10B0B0004FF0E022D2F8103D23F00603C2F8103D15
:10B0C000FEF72FFC94F8D23263B1D4F8D8329B68E3
:10B0D000DB0707D5D4F8D423136823F0030161F309
:10B0E00007031360034B4FF480225A6110BD00BF69
:10B0F00030290020003C01402DE9F04F974CD4F856
:10B10000D4325A69D0078DB000F1A4825A699B6984
:10B110001340019300F09E82C3F307430293019B07
:10B12000190311D5D4F8D832DFF83C929E69DB6957
:10B1300004F5327B1E40360C04F547774FF00008CB
:10B14000DA46002E40F01681029B5A070FD5D4F83C
:10B15000D832834E9F69DB691F40BFB2A6F1180544
:10B160004FF00009A6F53878002F40F04881019B88
:10B170009DF80470980741BF784BD3F8D43202226F
:10B180005A61019B002B1BDA744D95F8D2323BB10A
:10B19000D5F8D423136823F0030161F30703136088
:10B1A000D5F8D8226F48536823F0010353606E4BE3
:10B1B000D3F8B4389847D5F8D4324FF000425A61EA
:10B1C000019B1905C3F3072631D5644D00238DF883
:10B1D0001F3095F8DA338DF81F30634B05F5327068
:10B1E000D3F8B0389847D5F8D422D5F8D8324FF4F0
:10B1F00000619B68516195F8D222C2B1DA0716D579
:10B2000095F8DD33012B12D19DF81F30032B0ED1A1
:10B21000D5F8D4331A6842F001021A601A6842F075
:10B2200003021A60514A136943F0060313613B0796
:10B230000AD54A4D4C4B05F53270D3F8A8389847DB
:10B24000D5F8D43208225A61FD0615D5434BD3F800
:10B25000D402826922F010028261026AC2F3434181
:10B26000022902F00F0500F08681062900F0AA816C
:10B27000836943F010038361F00637D5374DD5F865
:10B28000D822D5F8D4025368002723F00103536075
:10B2900039464CF04BFFB84695F8C9023B4605F5D8
:10B2A0003875FF218342C0F09B81D4F8D8322D48F5
:10B2B0004FF0FF329A614FF00112DA610B2262F314
:10B2C000070762F307085F61C3F810801A686FF31D
:10B2D0000A121A60FFF751FED4F8D43221484FF415
:10B2E00080525A61204BD3F8AC389847B10640F1F0
:10B2F00093811A4CD4F8D832D4F8E00299680268E5
:10B30000C1F34101022906BF032161F30A026FF371
:10B310000A0202605A6842F480725A6008A8FFF775
:10B3200009F8D4F8D412D4F8D802CB68099A6FF38C
:10B330008D23CB6085680E48C5F34105284490F8FD
:10B34000CC00032840F05381002284F8CA224FF435
:10B350000072A4F8CC22092258E100BF3029002055
:10B36000102C0020F82B00200000002000ED00E051
:10B37000D4110608F2073BD55FFA88F104EB81038C
:10B38000D3F81C339D68D4F8D8325B691D40EB07B5
:10B3900020D594F8CB023B680125A8429D6007D1D7
:10B3A0001869DBF87C33C0F312001B1ACBF88C331E
:10B3B000D9F89C385046984794F8CB32012B09D1E4
:10B3C000B8F1000F06D194F8D933052B02D15046BD
:10B3D000FFF7D3FDA80742BF3B6802259D60290700
:10B3E00006D5D9F8A438504698473B6808229A6099
:10B3F00008F10108760804370BF1280BA1E6FB07DA
:10B4000079D5D8F8D8325FFA89FA1969586B08EB00
:10B410008A0220FA0AFBD2F8E0224FEACB1B92689C
:10B420005FFA8BFB4BEA010B0BEA020B1BF0010FDF
:10B430001ED05A6BA8484FF0010B0BFA09F122EA13
:10B4400001025A633368C3F808B0A44B5146D3F8DD
:10B45000A038984798F8CB325B4509D1B9F1000F75
:10B4600006D198F8D933042B02D19B48FFF785FD0C
:10B470001BF0080F1EBF33684FF0080BC3F808B06D
:10B480001BF0100F1EBF33684FF0100BC3F808B04D
:10B490001BF0400F1EBF33684FF0400BC3F808B0DD
:10B4A0001BF0020F1EBF33684FF0020BC3F808B049
:10B4B0001BF0800F1FD0D5E94C329B1AD5F8242100
:10B4C000D6F800E098F8CBB2DEF81800934228BF17
:10B4D00013460333D8F8D82203929B080AF1320AA4
:10B4E000049308EB8A0A049B80B2984203D9D5E9F9
:10B4F0004C03984205D809F101097F080436283524
:10B5000032E6C01AD5F82431984228BF1846C31C29
:10B510009B080493BBF1000F1BD0D5F82811D5F878
:10B5200034210144C5F82811D5F8301102448A426B
:10B53000DEF81800C5F83421D5D1039B95F81C110D
:10B540005A6B012303FA01F1039B22EA01025A63B9
:10B55000C9E782B2DAF8D012D5F828C103329310C5
:10B5600005930A465946059B8B42D6D05CF821309C
:10B5700013600131F7E747F6F07111423FF478AEFE
:10B58000282101FB0531C2F30A12D71CD3F898E336
:10B59000D1F848C6BF1000218F420DD1282101FBF0
:10B5A0000533D3F848161144C3F84816D3F8541697
:10B5B0000A44C3F854265BE6DEF800804CF821808C
:10B5C0000131E9E7D3F898130F68C3F89478096854
:10B5D000C3F89818282101FB0533C2F30A12E5E7E6
:10B5E00055F8042B9160AA6B013391605AE6012053
:10B5F00084F8CA024020A4F8CC02A0F56400384CBC
:10B60000A0F562401044A04227D80E2262F38D2399
:10B61000CB604FF400534B61029BDA060BD5314CE3
:10B620002E4B04F53270D3F8B8389847D4F8D4329A
:10B630004FF480125A61029B9B060BD5294C274B75
:10B6400004F53270D3F8BC389847D4F8D4324FF4AC
:10B6500000125A610DB0BDE8F08F234CA2F57400C2
:10B66000A0F51050A04201D80D22CFE71F48204C72
:10B670001044A04201D20C22C8E71E4CA2F18C70EB
:10B68000A0F54340A04201D80B22BFE71A481B4C4B
:10B690001044A04201D20A22B8E71948194C1044BC
:10B6A000A042FFF458AE184CA2F1B770A0F5585064
:10B6B000A04201D20822A9E71448154C1044A04228
:10B6C00001D20722A2E713481044134A904234BF24
:10B6D000062205229AE700BFF82B00200000002078
:10B6E0003F420F0030290020DFC810002013FBFE6E
:10B6F00020D61300FF69180000D3CEFE40771B0050
:10B70000C05BB3FEC091210040AC2700C01D6AFEA3
:10B7100040E13300803C36FEE09C4100034BD3F80F
:10B72000840908B104F06BBB012070473818002071
:10B7300008B5FFF7F3FF0A4A18B9002382F8583911
:10B7400008BD92F84C390133DBB2072B82F84C3933
:10B75000F3D8044BD3F89431C2F848390123EDE70C
:10B7600038180020302900202DE9FF47CC4CD4F8B0
:10B770008809002867D0CB4DCB4E04F6741794F897
:10B780005839013B082B46D8DFE813F00900600068
:10B79000EC004500C4014B01A0014500FF01FDF78D
:10B7A0007DFD00210846FDF705FE8046FDF786FD7C
:10B7B000B8F1010F2AD14FF0000984F84D99FDF737
:10B7C0006DFD40F2AB110820FDF7F4FD05280AD10C
:10B7D00084F84D89FDF772FD94F84D39A3B1022329
:10B7E00084F85839CBE70128F4D10423D4F8880928
:10B7F0004A4669464CF0A5FE9DF80330AB2B04BFCA
:10B80000022384F84D39E5E784F85839D4F88809DB
:10B81000022104F049F894F85839013B022B09D869
:10B82000A04BD4F84829D3F894319B1AC82B01D9DE
:10B83000FFF77EFF94F85809042800F0B681A0F1C4
:10B8400008035842584104B0BDE8F087FDF726FDD3
:10B8500094F84D39022B0CBF4FF080484FF0000890
:10B8600000213720FDF7A6FD41462920FDF7A2FD66
:10B870008046FDF723FDB8F1000FC7D194F84D398C
:10B88000022B39D1FDF70AFD41463A20FDF792FD22
:10B89000042381464246D4F8880969464CF051FE9B
:10B8A000FDF70CFDB9F1000F02D0FFF741FF66E78D
:10B8B000009B1BBAC3F3807384F84E39FDF7EEFC8E
:10B8C00000210920FDF776FD98B910213846FDF7D3
:10B8D00025FD814668B901217F2049F05FF90128E3
:10B8E000804606D10221484649F058F938B101286E
:10B8F0002CD0FDF7E3FC89E784F84E89DEE70421CC
:10B900002C2049F04BF9032182464E2049F046F99C
:10B910000C218146362049F041F909F10202411C0F
:10B9200001FA02F208FA0AF3A2FB03385B0A43EABF
:10B93000C853C4F85C39FDF7C1FCFDF7AFFC00212A
:10B940000A20FDF737FD50B9032349E716213A20B5
:10B9500049F024F901308002C4F85C09EBE7FDF7F7
:10B96000ADFCA2E710216846FDF7D8FC00287FF463
:10B970004DAF9DF8003084F86239BDF801305BBAF4
:10B98000A4F860399DF8033084F863399DF80430D9
:10B9900084F864399DF8053084F865399DF80630DF
:10B9A00084F866399DF8073084F867399DF80830C7
:10B9B0001A0903F00F0384F86D39DDF8093084F8B3
:10B9C0006C291BBAC4F868399DF80D309DF80E201B
:10B9D0001B01DBB243EA121303F5FA6302F00F0214
:10B9E000A4F86E3984F87029FDF768FC94F84E3994
:10B9F0004BB1D4F88809022103F056FF0023C4F8A4
:10BA000054390423ECE6FDF749FC4FF40071102093
:10BA1000FDF7D0FC8046FDF751FCB8F1000FE8D0EF
:10BA200043E794F83C19D4F83429D4F888098023E2
:10BA300002EBC11200214CF084FD94F83C39013333
:10BA4000DBB2042B84F83C397FF4E5AED4F88809E6
:10BA50000223324600214CF074FD0123D4F88809FA
:10BA6000002269464CF06DFD9DF8003003F01F0385
:10BA7000052B1BD1072384F858390A4BD4F84059B9
:10BA8000D3F89431C4F84839002D3FF4C4AED4F84B
:10BA90004439D4F83429D4F838190120A847BAE633
:10BAA0003818002030290020A4120608FFF740FEB5
:10BAB000D4F84089B8F1000F3FF461AED4F84439AE
:10BAC000D4F8381900220120C04758E64CF05EFD3A
:10BAD000002861D0002384F84C39D4F85439012B64
:10BAE0000BD9013BC4F85439D4F850390133C4F8A8
:10BAF0005039082384F858398DE607D1FDF730FC1A
:10BB000002287FF488AEFDF7D9FB84E6042384F88D
:10BB10005839F8E7D4F834094FF40071FDF7FEFB0B
:10BB20000128804618D002281ED000287FF473AE6A
:10BB3000FDF7C4FBD4F8405984F84C89042384F8F9
:10BB40005839002D3FF467AED4F84439D4F834297D
:10BB5000D4F838194046A1E7D4F84839D5F89421EB
:10BB600064339342BFF457AEFDF7A8FBFFF7E0FD47
:10BB7000D4F84089B8F1000F3FF401AE0022D4F8A8
:10BB80004439D4F8381910469EE74CF0FFFC18B140
:10BB9000FDF794FB0423ADE7D4F84839D5F8942198
:10BBA000FA339342FFF481AE35E601204BE62DE9EE
:10BBB000F341294C05460E4690461F4694F85839E5
:10BBC000042B0BD0082B07D1D4F85039AB4219D035
:10BBD000FDF7C6FB0228F1D001200EE0FDF75EFB69
:10BBE00094F84E3963B969021820FDF7E3FB48B1B8
:10BBF000FDF764FBFFF79CFD032002B0BDE8F08178
:10BC00002946F1E794F85839D4F88809082B0CBF75
:10BC1000FC23FE23FF228DF804208DF8053001AAB5
:10BC2000022300214CF08DFCD4F888098023324691
:10BC300000214CF086FC012384F83C390623C4F82B
:10BC40003469C4F83859C4F84089C4F8447984F890
:10BC500058390020D1E700BF3818002070B51C4CBF
:10BC600094F85839042B05460E4610D1FDF716FB03
:10BC700000213720FDF79EFB31461720FDF79AFB88
:10BC800090B1FDF71BFBFFF753FD032002E0082BEB
:10BC900001D0012070BDD4F85039834214D0FDF793
:10BCA0005FFB0228F5D1E1E794F84E3973B96902D8
:10BCB0001920FDF77FFB0028E3D1082384F85839C9
:10BCC000C4F85469C4F850590220E3E72946EFE765
:10BCD00038180020044B054A03F6C801D3F8C838C9
:10BCE000C2F83019184700BF0000002038180020A3
:10BCF000002108B5084604F02FFCFFF7EBFFFCF726
:10BD0000F3FB0028FBD00121002004F025FC0020DB
:10BD100008BD034BD3F8300908B143691847704791
:10BD200038180020034BD3F8300908B1836918474D
:10BD3000704700BF38180020034BD3F8300908B112
:10BD4000C3691847704700BF3818002038B50D4642
:10BD50001446FFF7F1FF03682B604FF40073236074
:10BD6000002038BD034B1B78032B0CBF80204FF401
:10BD700080707047044F002008B50B4A68B1816895
:10BD800011B10723937008BDFFF7ECFFC2E903115F
:10BD9000C2E9010011750423F4E702F58051012383
:10BDA00081F8B4315370EEE7044F002010B50278EB
:10BDB0004368022A0B4A06D1D2E9800100EB410018
:10BDC00000EB532010BD0169D2F81802D2F81042DE
:10BDD00018400239D2F80C32400A04FB0100184422
:10BDE000F0E700BF045F0020074B1B78022B0BBF5E
:10BDF000030AC0F3D413C0B200F07F000CBF0B6085
:10BE00000B601060704700BF044F002090F91A309B
:10BE10005A1C0AD003F58172124B03EB0213DA7934
:10BE20006FF30002DA71FF23837690F91B104B1C2D
:10BE300016D00C4A01F5817102EB011302EB0112DD
:10BE4000DB79D179C3F34503012B86BF03F1FF33BF
:10BE500003F03F03002363F34601FF23D171C37650
:10BE6000704700BF044F002008B5FFF77BFF034B6E
:10BE7000D3F810325843400208BD00BF045F0020D1
:10BE80000378022B09D10D4BD3F820224368B3EB82
:10BE9000422F2CBF012000207047006960B1084B81
:10BEA0001B78032B0EBF074B80B24FF6F7739842F7
:10BEB00094BF00200120704701207047045F0020DC
:10BEC000044F0020F7FFFF0FF7B50D464168C1F39F
:10BED00008032B44B3F5007F044603D22944616074
:10BEE00001202EE0FFF792FF0378022B01D1616859
:10BEF000F4E7164BD3F81022B5EB422F4FEA422756
:10BF000021DCD3F8183246681E407342AB421ADC7B
:10BF1000AB19BB4210D30169007E01AA4BF0B2FC01
:10BF2000012810D123696361019B236163683B444D
:10BF30009B1BED1B636035442046FFF7A1FF0028E3
:10BF4000D5D003B0F0BD0020FBE700BF045F0020A8
:10BF500070B504460E461546FFF7B6FF20B10DB189
:10BF60002046A847012007E094F82800022320B9C2
:10BF7000C4E90B5684F8283070BD1846FCE7054A22
:10BF800092F8B411012309B982F8B431024A53700E
:10BF9000704700BF045F0020044F002008B5074B26
:10BFA000C31A48BF03F2FF13B3F5805F4FEA632063
:10BFB00003D3FFF7E4FF4FF0FF3008BD1C4F002014
:10BFC0002DE9F74F12F0020B0191174600F0D180D6
:10BFD000002840F0CE80FFF7D2FF02266EE04FF03F
:10BFE000FF36DFF8C4C1DFF8ACA1B6463446B1462F
:10BFF0000025DCF800109CF80E8088421BD1B8F1B7
:10C00000000F00F09880D2F89840624E0134C2F8D8
:10C01000984005F581721201B4502C465D4D04F52F
:10C02000817805EB08129679042ED4D8DFE806F063
:10C03000315DB05D6700B8F1000F26D0B8F1010F97
:10C0400014D105F581780AEB081898F8078018F0E4
:10C05000010F0BD118F07E0F08D15FEAD81116D16D
:10C06000DCF80880C14501D9AE46C1460135082D2E
:10C070000CF1100CBDD1751C79D1611C5CD1BEF1E5
:10C08000FF3F00F08580744656E02E46EEE72C46D2
:10C09000ECE717F0010215D03F4BD3F83039002BF5
:10C0A00076D03E495F683E4A002301EB4421B84701
:10C0B00000286DD005EB08150223AB71304603B0A4
:10C0C000BDE8F08F05EB0810FE1090F807C0032BB9
:10C0D00066F3C71C80F807C02BD94FF6FF72934256
:10C0E00028BF134605EB08129380BBF1000F06D062
:10C0F00005EB041000F580501830FCF717FA7A07AA
:10C1000041BF05EB0812D37943F00103D371FB065D
:10C1100008D505EB0815EB79C3F34502013262F34C
:10C120004603EB711D4B019A03EB44231360012678
:10C13000C4E71346D6E72C46164E41F2180506EB27
:10C14000041C4CF80500D2F898500135C2F89850FC
:10C1500041F21C024CF8025004F581724FEA021CB5
:10C1600006EB021246F80C500025556056E734469F
:10C17000E2E70C4AD2F80862002E3FF430AFD2E971
:10C18000834505FB0644A042FFF429AFFFF7F7FE05
:10C19000002693E7044F0020381800201C4F002091
:10C1A00029950008045F00201C5F00207FB50F4D1B
:10C1B00001AA0C4602A9FFF717FE05F58053029E5F
:10C1C000D3F800020322002303A93044FFF7F8FE4E
:10C1D000012808D12978039B019A02290CBF23F872
:10C1E000124043F8224004B070BD00BF044F00204D
:10C1F0002DE9F0470D4686B0164604A903AA074666
:10C200002868FFF7F1FD364A0499D2F8003201EBB5
:10C210000308039B013B9C19FFF7A4FD2B68E41A5C
:10C220000444A2F5805AB4FBF0F408EB0409296831
:10C23000B142A9EB080303D3012006B0BDE8F087A3
:10C24000039A0193FFF78EFD9419641A8442019BAF
:10C2500028BF0446002A35D1A04294BF0A220B22EF
:10C2600005A94046FFF7ACFE0128E6D19AF8000088
:10C270002A680599039B022802F101022DD1A342ED
:10C2800022D32B68039A9B1A2344012F2B6014D1CD
:10C29000B34212D102280BBF04F1004404F18043E1
:10C2A00004F1FF3403F1FF330BBF4FF6FF734FF080
:10C2B000FF3221F8143041F82320002308F101084F
:10C2C0000393B4E70B22CBE721F8132001330132AB
:10C2D000D5E741F8232001330132A342F9D3D0E757
:10C2E000045F00202DE9F04F85B08346FFF73AFD4B
:10C2F0000C461646814601AA206802A9FFF774FD84
:10C300000BF1FF33012B68D9019B63B94D46DFF870
:10C31000D080BBF1010F8CBF4FF0000B4FF0010B31
:10C32000A8F5805A1BE0FFF72AFE02202AE0D8F881
:10C330007821C2B1D8F89401884214D1D8F81032CB
:10C34000013A590202EB4323B3FBF1F30344B3FB7D
:10C35000F5F205FB12320AB12B449B1A23602168C7
:10C36000B142E4D329E0D8F80002029F0023092259
:10C3700003A93844FFF724FE012806D00228D4D0B0
:10C380000028ECD105B0BDE8F08F9AF800200399A1
:10C39000022A07D0032AC8D1019B51F8233023F089
:10C3A000704302E0019B31F813302768B3FA83F33E
:10C3B0005B095B4504D1BE42E4D826600320E1E777
:10C3C000019B2B442F444B4527600193E0D3029BF4
:10C3D0000133029300230193C1E7012597E700BFD2
:10C3E000045F002037B50446C0690D4698B10023AC
:10C3F000032201A9FFF7E4FD012806D1B4F920309A
:10C40000002B0ADAFFF7BBFD022003B030BDE525A3
:10C410005554A2680BE00120F7E7019A012D4FEA7D
:10C42000431102EB4313F4D0022DF0D0E268DA613D
:10C430002278032A04D100221A775A779A77DA777A
:10C44000626A5A83110C9982DFE770B5304D044659
:10C45000042694F83430052B2CD8DFE803F00324AD
:10C460003139424BD5F8082204F130010232012063
:10C47000FFF738FF012807D00238C0B2012819D8C9
:10C48000052384F83430E4E7D5F81012E268236B12
:10C49000C5F8143202EB4122E260E26A236102B97C
:10C4A00063620123EDE7206B4FF0FF31FFF77EFE63
:10C4B000012801D0002070BDE36A3BB10223E0E710
:10C4C000D4E90B01FFF772FE0128F3D10323D8E76B
:10C4D00000212046FFF786FF0128EBD184F8346065
:10C4E000B7E794F82830082B02D1002384F82830CD
:10C4F0000120E0E794F82830082B04BF002384F8DB
:10C500002830034B012283F8B5210220D3E700BF76
:10C51000045F00202DE9F743DFF81891044694F8F2
:10C520003850032D00F28180DFE805F002106E77AD
:10C530002046FFF78AFF012802D184F83800EEE791
:10C54000022873D1032384F83830E8E7237866683B
:10C55000022B18BFD9F81832204618BF1E40FFF72B
:10C5600025FCC6F34F260746361A0023022201A9EE
:10C570003846FFF725FD06EB070801281FFA88F863
:10C58000054653D101984FF40072002152F0F6FD98
:10C59000E369FBB16368EBB9019B4FF020322E21B8
:10C5A0001A605A601970C3F80720606A5883050C36
:10C5B00010201A625A6283F8201083F82110D87272
:10C5C000C3F82720E26B9D8222FA00F199865A87F0
:10C5D00083F82B00D9F810124B1E984508D24FF45F
:10C5E00000712046FFF770FC4BF078F80137BCE78C
:10C5F000C1EBC151490201F500712046FFF764FC0F
:10C600004BF06CF802239EE7002384F82830236C5B
:10C610000BB120469847012508E0236C002084F8E0
:10C62000280003B19847022500E00025284603B002
:10C63000BDE8F083045F0020F8B52E4E044600F1FB
:10C640003007A6F5B87594F83830032B50D8DFE8DA
:10C6500003F0022E363FD5F894212261FFF704FC47
:10C66000E3681844E060FFF77DFB1044C5F89401CF
:10C67000FFF7FAFBD5F87831181AC5F87801FFF7FB
:10C68000F3FBD5F87C31181AC5F87C012263FFF75B
:10C6900069FBE36A1044606323B96262012384F892
:10C6A0003830D0E7FFF75EFB101A2063F6E7002171
:10C6B0003046FFF797FE01280ED10223EFE7626BA9
:10C6C00039460120FFF794FD012805D10323E6E751
:10C6D00000212046FFF786FE431EDBB2012B06D861
:10C6E00094F82830062B04BF002384F82830F8BDC6
:10C6F0000220F1E7746000202DE9F743454D002941
:10C70000044614BF0226002605F5805794F83C30F5
:10C71000042B71D8DFE803F0290336406300DFF80B
:10C72000FC802B78206B032B53D1404594BF4FF0F6
:10C7300000094FF00109B9F1000F48D101A948F0F3
:10C7400009FA012863D1206B4946FFF72FFD012824
:10C750005DD1019B2363D7F81422013B934294BF20
:10C76000C7F81432C7F81422DBE731462046FFF73A
:10C7700039FE0128034648D1626B02B1022384F8D6
:10C780003C30C3E7626B04F130010020FFF730FD5D
:10C7900001283AD10323F2E7E26AD7F89431C7F8C7
:10C7A00094219B1AD7F810221B485343D7F87821BD
:10C7B00002EB4322C7F87821D7F87C21002102EB55
:10C7C0004323C7F87C31FFF70DFE01281DD1042358
:10C7D000D5E71FFA80F94FF6F7739945A6E794F865
:10C7E0002830042B04BF002384F82830A36B0BB13E
:10C7F0002046984701200AE0022094F82830042BB4
:10C8000005D1002384F8283001E00228F5D003B0D8
:10C81000BDE8F083044F002074600020F7FFFF0F95
:10C8200070B50378023B012B04461CD8237E990681
:10C8300023D42046FFF7EAFA237E1A070AD51F4DB4
:10C8400095F89801C31F584258414AF047FF00230A
:10C8500085F898310023237084F82830E36A5BB1AF
:10C86000BDE870401847037E13F0060FDED00121AB
:10C87000FFF7B8FD0128D9D070BDE2691049002347
:10C8800018014058824211D10E4903F5817201EB23
:10C890000213DB79C3F34503012B0BD8002301EB13
:10C8A0000212D17963F34601D171C2E70133082B3B
:10C8B000E6D1BEE7013B03F03F03F0E7045F002051
:10C8C0001C5F0020044F002010B580B1027872B1C7
:10C8D00090F828206AB9D0E9012494422CBF8460E2
:10C8E0008260032280F82820C162FFF799FF0120AF
:10C8F00010BD0020FCE7B1F904300F2B2DE9F34106
:10C9000004460D4616460BD14FF40071FFF7DCFAD2
:10C9100018B9002002B0BDE8F0814FF6FF73AB807C
:10C920002046FFF743FA94F91B20531C074611D009
:10C930001E4B41F2180103EB021041588F4230D0D8
:10C94000FFF71DFB2046FFF79BFA0028E1D00023EC
:10C95000336024E02046FFF793FA80460028F1D1A7
:10C96000381E18BF01204AF0B9FE4346112201A922
:10C970003846FFF725FB0128E4D10198FFF70EFBAD
:10C98000E076019A002ADDD0AB8801331BB2AB8080
:10C9900002EB431333602046FFF708FA28600120BA
:10C9A000B8E7183303EB42230193EAE7044F002072
:10C9B0002DE9F0414FF0FF31304A314C0D46002354
:10C9C000107804280ED103F5817004EB0010C079B3
:10C9D000C70707D46E1C52F80A0C01D0884201D256
:10C9E0001D4601460133082B02F11002E8D16B1CF1
:10C9F00042D0234C234E05F5817704EB0713998829
:10CA000049B1D6F8303933B104EB051041F21802C0
:10CA10009B6880589847D6F830399BB11A4ED3F8A6
:10CA20000C801A4A04EB051C41F2180000235CF844
:10CA3000000006EB4521C04720B1022810D000209D
:10CA4000BDE8F081124BD3F89C2004EB0714013AA7
:10CA5000C3F89C200322A271012283F8A020EEE7F4
:10CA600006F6E87604EB0714D6F89C30013BC6F8CE
:10CA70009C300123A371E2E70120E1E72A5F002057
:10CA8000044F0020381800201C4F0020819500081A
:10CA9000045F002008B500214422104852F06EFBCC
:10CAA0000F4B03F580501B784FF6FF72A0F8D22190
:10CAB000022B4FF0030218BF134680F8B831D0F8AC
:10CAC0001C32C0F8DC31102380F8D02180F8D1313D
:10CAD00000F5DC7048F02CFA012008BDBC60002095
:10CAE000044F002070B5124D124BC5F8BC3840F20F
:10CAF0000112002385F81132A0F84421C0F85C31FE
:10CB000005F6BC020D23C0E95422044685F8C81876
:10CB1000C0F8583100F5A2714BF00FF805F5F87226
:10CB200020461F23BDE8704001214BF09FB800BF95
:10CB3000302900205553425310B5074B93F8FD118F
:10CB400004464BF0B1F8002804DA20460121BDE884
:10CB50001040C7E710BD00BF30290020F8B50B78A2
:10CB600013F0600506460C4638D0202D74D14A7863
:10CB7000FE2A05D0FF2A1CD04AF0E0FE02252BE059
:10CB80004D88A5B9CF88012F11D11A060FD5334C86
:10CB9000D4F81C329B699847C0B284F8CC0830B1F5
:10CBA0003A4604F6CC0130464AF09CFF14E0304689
:10CBB000E2E74A88002AFAD1CD88002DF7D11B067A
:10CBC000F5D4264A012182F8115282F810121F234F
:10CBD00002F5F8724BF04AF82846F8BD4B780A2B5C
:10CBE00024D00B2B25D0012BF6D194F90430898861
:10CBF000C068002B22DA01F07F014BF097FA21790F
:10CC0000164F30464AF0A8FE0223217940223046D2
:10CC10004AF0CBFE97F81032022B12D18121304618
:10CC20004AF05AFE002387F81032D5E70C4901225A
:10CC3000BAE70A4B4A8883F8CD28CDE74BF060FA73
:10CC4000DDE794F90420002AC6DA012BC4D00121C3
:10CC50003046FFF747FFBFE70025BDE7302900203A
:10CC6000FD31002008B5084B93F81132022B07D094
:10CC7000033B012B02D80021FFF734FF002008BD41
:10CC8000FFF75AFFFAE700BF3029002070B52F4C9C
:10CC900094F8116205461EB1012E54D0002070BDDB
:10CCA000D4F8F431C4F8C038D4F8F831C4F8C43832
:10CCB000B0F8B4331F2B0DD1D4F8F021244B9A4295
:10CCC00008D194F8FD11012904D894F8FE31013BF4
:10CCD0000F2B0AD92021052047F08AFE022384F871
:10CCE00010322846FCF7A4F9D8E74AF0DDFF002807
:10CCF000F7DB94F81132013B022BCFD9B4F8CE18F0
:10CD0000E9B1D4F8F83184F8C868994228BF1946C7
:10CD1000D4F8C4385B1AC4F8C438042384F8113238
:10CD200040F20113A5F844310A4BC5E95616C5E98E
:10CD3000543305F5A27128464AF0FFFEAEE72846B7
:10CD4000FFF7D0FEAAE7FFF7F7FEA7E7302900209C
:10CD500055534243043F0020F0B59C0827010E467E
:10CD6000154600EB0414A04206F1100605F110056B
:10CD700008D103F0030339443A4404EB83039C4293
:10CD800023D1F0BD84469CED006A16ED045AD0ED27
:10CD9000016A56ED037A90ED027A56ED025A26EEBC
:10CDA000056A66EEA76AD0ED037A05ED046A16ED12
:10CDB000016A45ED036A27EE257A67EE867A103020
:10CDC00005ED027A45ED017ACDE7F4EC017AB1EC9C
:10CDD000017A67EE877AE2EC017AD0E74A0901230B
:10CDE00001F01F0103FA01F150F82230194214BF7B
:10CDF0000120002070474A09012301F01F0103FAB6
:10CE000001F150F822300B4340F8223070474A09B4
:10CE1000012301F01F0103FA01F150F8223023EA47
:10CE2000010340F82230704780EA0120082341F2D4
:10CE3000210210F4004F4FEA400018BF5040013B60
:10CE400080B2F6D1704738B50C468D18AC4200D18F
:10CE500038BD14F8011BFFF7E7FFF7E74840082348
:10CE600010F0800F4FEA400018BF80F0D500013B62
:10CE7000C0B2F5D1704710B50A440C46944200D1B7
:10CE800010BD14F8011BFFF7E9FFF7E738B50A46B4
:10CE9000056804460020AA4203D36B1C2360287057
:10CEA00038BD12F8011BFFF7D9FFF4E7DFED0A7A6E
:10CEB000C0ED020A20EE270AB7EE007AC7EE007A2C
:10CEC00000230360C0ED017A70EEA77A80EEA77AA6
:10CED00080ED037A704700BFDB0FC94090ED017A07
:10CEE000D0ED007AC0ED020A30EE877AC0EE876A94
:10CEF00030EE677AE6EE877AB0EE670AC0ED007A28
:10CF00007047012303700023C364836403650364D3
:10CF100043644365836283657047DFED157A80ED76
:10CF2000010AF4EEE70AF1EE10FAC0ED020A80ED14
:10CF3000031AC0ED051A18DDB4EEE70AF1EE10FA97
:10CF400010DD81EE007AC0EE207AF0EE006A77EE16
:10CF5000877A86EEA77A80ED047A80ED0F2AC0EDFD
:10CF60000E2ACEE700230361F7E700238360FAE788
:10CF7000BD378635FDEEC07A17EE903A2033402B50
:10CF800043D8DFED237A9FED237AB4EEE70AF1EE82
:10CF900010FA28DCDFED207A9FED1E7AB4EEE70A66
:10CFA000F1EE10FA22D4DFED1D7AB4EEE70AF1EECD
:10CFB00010FA1EDD30EE670A37EEC00A60EE007A26
:10CFC000DFED176A9FED177AA7EEA67ADFED166AF6
:10CFD000E7EE876A9FED157AA7EEA67A20EE276A1C
:10CFE000A6EE070A704730EE470ACEE730EE070A92
:10CFF000D4E79FED0F7AB4EEC70AF1EE10FA44BF02
:10D0000030EE270A37EE400AD8E79FED0A0A70474C
:10D01000DB0F4940DB0FC940DB0F49C0DB0FC93FC5
:10D020009A7C2E36FAAF4FB93587083CA4AA2ABE9F
:10D03000DB0FC9BF00000000DFED027A30EE270AE7
:10D0400098E700BFDB0FC93F38B51D46304BB3FB37
:10D05000F2F39942B0EE405AF7EE005A4FF0000456
:10D060004FD207EE901A9FED2B7ADFED2B6AF8EE88
:10D07000677A67EE877A07EE102AB8EE477A27EECE
:10D08000267AC5EE876A87EEA64AB0EE440AFFF715
:10D0900071FFF0EE404AB0EE440AFFF7CDFF35EEE7
:10D0A000055A012D84EE854AF0EE407A1CBF35EE1C
:10D0B000E76AF6EE006AB8EE000A34EE257A12BF8F
:10D0C00066EE266A27EE806AF0EE656A86EE875A7B
:10D0D000C6EE076A67EE807A75EEC45AC0ED016A43
:10D0E000C7EE876AC5EE877A80ED005A80ED025A56
:10D0F000C0ED036AC0ED047A846144610462C461D6
:10D1000038BDC0ED005A44608460C4600461F3E738
:10D1100020A10700DB0FC940BD3786359FED010A0E
:10D12000002391E7F304353F2DE9F041FCEEC07A8E
:10D1300013460A4617EE901AD0F814808769C6691C
:10D14000056AB0EE600A89B2FFF77EFFC0F814806E
:10D150008761C6610562BDE8F081F0EEE06AB0EE7D
:10D16000C07AF4EEC76AF1EE10FAD4BFB0EE476AA7
:10D17000B0EE666AB5EE406AF1EE10FAF0EE405A93
:10D1800046D0F4EEC76AF1EE10FA54BFB0EE475A3B
:10D19000B0EE665AC5EE067A9FED1F6A9FED1F5AE4
:10D1A000DFED1F4AA7EE865A9FED1E6AA5EE276A9D
:10D1B0009FED1D5AA6EE275A9FED1C6AA5EE276A21
:10D1C0009FED1B5AE7EE854AB7EE005AA4EEA75A28
:10D1D000F1EE467A87EE850AF4EEC76AF1EE10FAB0
:10D1E00048BFDFED147AF5EEC00A48BF37EEC00A3B
:10D1F000F1EE10FA48BFDFED107AF5EEC05A48BFE5
:10D2000037EEC00AF1EE10FA48BFB1EE400A70479F
:10D21000DFED0A7AC0E700BF39094E3DE3B59EBE97
:10D2200069A2163E88FA16BE45FE7FBFA7DFA8B4E6
:10D2300099FB243FDB0FC93FDB0F49400000000092
:10D2400044F25063984203DDA0F50C40A0387047CB
:10D25000034B9842BCBF00F50C40A030704700BFA4
:10D26000B0B9FFFF48F69F43984203DDA0F50C409C
:10D27000A03870470028BCBF00F50C40A0307047B4
:10D2800091ED005A08B5B0EE450AFFF7D5FEF0EE75
:10D29000405AB0EE450AFFF76DFE91ED015AF0EEEF
:10D2A000404AB0EE450AFFF7C7FEF0EE403AB0EE56
:10D2B000450AFFF75FFE91ED023AB0EE405AB0EE3C
:10D2C000430AFFF7B9FEB0EE404AB0EE430AFFF75B
:10D2D00051FE25EE806A63EEC07A24EE847AC0EDBA
:10D2E000017AF0EE467AE5EE077A25EE843A64EEAE
:10D2F000806AC0ED037AF0EE437AE5EE667AA5EE39
:10D30000067AE5EE436A23EE844A64EEE34A65EE6C
:10D31000A35A80ED004A80ED025AC0ED047AC0EDB8
:10D32000054AC0ED066A80ED077AC0ED085A08BDCF
:10D33000034600F1400100221A615A619A61DA61E4
:10D3400010339942F8D11022002151F017BF91ED0E
:10D35000007AD0ED047AE7EE077AC0ED047AD1EDD9
:10D36000006A91ED017AD0ED057AE6EE877AC0ED9C
:10D37000057AD1ED006A91ED027AD0ED067AE6EEFB
:10D38000877AC0ED067A91ED007AD0ED077A77EED4
:10D39000877AC0ED077AD1ED016A91ED007AD0ED80
:10D3A000087AE6EE877AC0ED087A91ED017AD0ED41
:10D3B000097AE7EE077AC0ED097AD1ED016A91EDBD
:10D3C000027AD0ED0A7AE6EE877AC0ED0A7A91ED1C
:10D3D000017AD0ED0B7A77EE877AC0ED0B7A91ED7A
:10D3E000007AD1ED026AD0ED0C7AE6EE877AC0EDD4
:10D3F0000C7AD1ED026A91ED017AD0ED0D7AE6EE6C
:10D40000877AC0ED0D7A91ED027AD0ED0E7AE7EED3
:10D41000077AC0ED0E7A91ED027AD0ED0F7A77EEB1
:10D42000877AC0ED0F7A91ED007AD0ED107A77EE21
:10D43000877AC0ED107A91ED017AD0ED117A77EE0E
:10D44000877AC0ED117A91ED027AD0ED127A77EEFB
:10D45000877AB7EE007AC0ED127AD0ED137A77EEC4
:10D46000877AC0ED137AD1ED017AD1ED006A91EDA2
:10D47000027A67EEA77AE6EEA67AE7EE077A90EDF3
:10D48000007AA6EEA77A80ED007AD1ED016A90EDE0
:10D49000017AA6EEA77A80ED017AD1ED026A90EDCD
:10D4A000027AA6EEA77A80ED027A90ED037A77EE03
:10D4B000277AC0ED037A70472DE9F043034685B023
:10D4C00000F11007054600261C46AC4612E0F8ECB9
:10D4D000016A1EED047AD4ED007AE6EEC77AC4ED57
:10D4E000007A98450EF1100EF1D10434BC420CF1D3
:10D4F000040C03D0A7F11008E646F2E701361C46FB
:10D50000B646BEF1040F1FD000EB0E1CA84604F176
:10D51000100909E0FCEC016A18ED047AD4ED047AF4
:10D52000E6EEC77AC4ED047ACC4508F11008F1D1D3
:10D53000D4ED046A93ED007AC6EE877A0EF1010EFF
:10D54000C4ED047A6446DCE7042E03F1140305F10C
:10D55000040507F11007B7D100230093019302934C
:10D5600003936C460023142752F8045B44F8045BD1
:10D5700007FB030C00EB03156E4665451FD1013315
:10D58000042BF1D104AD103100F1400255F8044DE7
:10D590000E4600EB031741F8044D1446A742D1EDA7
:10D5A000007A17D152ED016A87EEA67A013BA2F10B
:10D5B000140281ED007AE9D105B0BDE8F083B6EC44
:10D5C000017A54ED017AF5EC016AE6EEC77A44ED92
:10D5D000017AD2E7F4EC016AB6EC017AE6EEC77A9A
:10D5E000C1ED007ADAE79FED0C7A00F10C03F0EC64
:10D5F000017AF4EE677AF1EE10FA06D7F0EEE77AE8
:10D60000F4EE477AF1EE10FA03DC9842EFD10120F4
:10D6100070470020704700BFFFFF7F7F1FB50C469B
:10D62000024669461030FFF747FFDDED007AB6EE9F
:10D63000007A67EE877A2046C4ED007ADDED017A44
:10D6400067EE877AC4ED017ADDED027A67EE877ABC
:10D65000C4ED027AFFF7C7FF04B010BD60EEA00A68
:10D6600020EE400A70EEA00AC0EE200A9FED010AEB
:10D670004CF088BE54F82D40B5EEC00AF1EE10FA19
:10D6800008B506DB4CF0DCFEB4EE400AF1EE10FA11
:10D6900001D79FED010A08BD00000000F8B52DED8F
:10D6A000028B044625461C3004F1640250ED017AD9
:10D6B000B1EC010A77EE807A40ED017AFBF776F85B
:10D6C00018309042F2D123692D4E626801332361F4
:10D6D000D6F894319B1AA26893422DD99FED298ADE
:10D6E00004F13007EB6A012BC1BF03F1FF3307EEF2
:10D6F000903A95ED0A7AF8EEE77AD4BFB0EE480A90
:10D7000087EE270AFFF7B8FFBD42D4ED057A16D0A1
:10D71000F4EEC07AF1EE10FA05F11805E2D5237B9C
:10D7200053BBD6F89421626000222361A261E362B8
:10D7300022636364A264E365BDEC028BF8BDF4EE82
:10D74000C07AF1EE10FAEAD4D4ED047AD4ED066A88
:10D75000F8EE677A022386EEA77AD4ED0C6A84EDA0
:10D76000067A86EEA77AD4ED126A84ED0C7A86EEFC
:10D77000A77A84ED127A00E003232370DCE700BF70
:10D78000302900200000000038B50378012B044642
:10D790003CD10369254D23B9426812B9D5F89421CB
:10D7A0004260D4ED067A77EE807A01332361C4EDCE
:10D7B000067A04F11C00FAF7F9FF6268D5F8943193
:10D7C0009B1AA268934221D9E36A012BC3BF03F1DC
:10D7D000FF3307EE903A94ED0A7A9FED150AC4BF25
:10D7E000F8EEE77A87EE270AFFF746FFD4ED057AD1
:10D7F000F4EEC07AF1EE10FA0CD5237B3BB9D5F8E4
:10D800009421626000222361A261E36238BD032398
:10D810002370FBE7D4ED047AD4ED066AF8EE677A5C
:10D82000022386EEA77A84ED067AF1E730290020FC
:10D830000000000008B52DED028BF0EEC08AB0EEBE
:10D84000408AB7EE000A30EE680AFFF715FF9FED39
:10D850000E7ADFED0E7AE8EE877A9FED0D7AA7EE6D
:10D86000A87ADFED0C7AE7EE287AB5EEC08ABDEC37
:10D87000028BF1EE10FA20EE270A44BFDFED067AA4
:10D8800037EEC00A08BD00BF306E99BC2716983D20
:10D89000843459BEA40DC93FDB0F494060EEA00A95
:10D8A000E0EE000AB0EE600AE6E660EEA00AE0EE06
:10D8B000000AE1EE010AB0EE600ADDE62DE9F74F5D
:10D8C00090469DF83020002A14BF4FF030094FF0E9
:10D8D00020090D9A1C1E05460F46BABF644201235B
:10D8E000002312F8011B01B12CB9A24663B1002438
:10D8F0000D9EA41B12E0013CF3E7BD4204D2494651
:10D9000028460193C047019BBAF1010AF5D2EFE71F
:10D91000BD4203D228460193C047019B06EB040B8E
:10D9200016F8011B0029F3D133B15446002C07DC53
:10D93000BAF1000FA8BFD344584603B0BDE8F08F3A
:10D94000BD4202D249462846C047013CEEE70FB42B
:10D9500037B50C4D06ABD5F8D41853F8042BD5F8D1
:10D96000D00801934AF043FE0446D5F8200203F0A4
:10D97000FAFC0028F9D0204603B0BDE8304004B0DE
:10D98000704700BF302900200EB403B503AB08492F
:10D9900053F8042BCDE9003001A84AF028FE019B82
:10D9A00000221A7002B05DF804EB03B0704700BFAC
:10D9B000FB8700080CB430B52C4CD4F8D838A5B08F
:10D9C0001BB9D4F8DC38002B39D094F8E0389942F0
:10D9D00006D9012303FA00F0D4F8E43818422ED017
:10D9E000D4F894114FF47A7304A8B1FBF3F203FB5B
:10D9F00012131F49FFF7C8FF04AB0344289A1D49BF
:10DA00000393054629AB03A802934AF0F0FD039B5C
:10DA1000591C03910A211970039B0246591CD4F822
:10DA2000D80803910021197090B103681B6A03B1F3
:10DA30009847D4F8D85804AC14F8011B21B925B084
:10DA4000BDE8304002B07047284603F062FCF3E7BF
:10DA5000D4F8DC38002BF2D002212A4400910A4489
:10DA6000FD2004A927F0EAF9E9E700BF30290020EA
:10DA70007FAE0608A387000810B54FF4004086B0BB
:10DA800025F064FB044690B34FF4004125F0C0FC40
:10DA900002281AD1226848F201039A4227D14FF492
:10DAA000004046F0B9FB10B31F4BD3F8E828824280
:10DAB0001FD0D3F8C429904230D0D3F8A02A904286
:10DAC0002FD00022C3F8DC2811E00023022294F9B1
:10DAD0000400CDE901234FF4612200924FF400418C
:10DAE0001A4625F0E5FC104BC3F8D80828B906B053
:10DAF00010BD03F6E802C3F8DC280C4B04930C4B72
:10DB000003930C4B02930C4B01930C4B00930C4A68
:10DB10000C4B02210020FFF74DFFE8E703F6C4128B
:10DB2000E9E703F52A62E6E7302900208BAE060814
:10DB300094AE06089DAE0608A9AE0608E8AD060834
:10DB400038B90608FBAD0608174A38B5D2F87C4B41
:10DB5000033004EB9003B3F5007F19D802F5386564
:10DB6000C2F87C3B114A02EB810120F00300D1F89E
:10DB70008822C3F500731044C1F888020C4A9B0048
:10DB80000421002005EB8404FFF714FF204638BD74
:10DB90000021084A0846FFF70DFF074A136843F0C3
:10DBA000007313600024F1E730290020283A002098
:10DBB000AFAE0608D3AE0608582701202DE9F0477E
:10DBC00006460068FBF78BFF0D28054608DD1F4A57
:10DBD00000210520FFF7EEFE00242046BDE8F08777
:10DBE0001B4F07EB80094FEA8008D9F824A2BAF14D
:10DBF000000F1CD107216420FFF7A6FF0446C9F8D7
:10DC0000240228B90146134A0520FFF7D3FEE4E7B2
:10DC10006422514651F0B2FA0F48D9F824322DB29D
:10DC200000EBC505C3E90053DB615B63DB6447447C
:10DC30007179D7F82442182000FB014300221C46CA
:10DC4000C3E903229E601A750434C6E7E1AE0608F4
:10DC50003029002006AF06082C12060803685A1C5B
:10DC6000026019700368090A5A1C02601970704733
:10DC700003685A1C0260197003685A1C02600A0A81
:10DC80001A7003685A1C02600A0C1A700368090EA5
:10DC90005A1C02601970704703685A1C02600A0A15
:10DCA0001A7003685A1C02601970704738B5044630
:10DCB000006815464FF0C4F823682B44236038BD34
:10DCC00003685A1C02601878704703685A1C026087
:10DCD0001A4612F8021B0260587841EA0020704789
:10DCE00010B502681146531C036011F8024B016025
:10DCF000D31C5178036093781B0443EA0123111D60
:10DD00000160D078234343EA006010BDD1E90032BE
:10DD10009A4206D05A1C0A6008B11B780370012091
:10DD2000704700207047D1E900239B1A012B10B5E2
:10DD30000446084604DDFFF7C8FF2080012010BD1F
:10DD40000020FCE730B50A440446914201D100208E
:10DD500011E014F8013BA3F14100192811F8010B5F
:10DD6000A0F1410598BF2033192D98BF20301B1A10
:10DD700002D10028E9D130BD1846FCE76FF000421F
:10DD8000E0E710B50288C378A2F5FA62910840F284
:10DD9000B554013B04FB013381780C24013902F0B6
:10DDA000030204FB02120D49847901EB420218219F
:10DDB000B2F8D2201344027901FB0322437900898F
:10DDC0003C2101FB0233064A224401FB03224FF4AB
:10DDD0007A730021C2FB030110BD00BFD4110608F5
:10DDE00080436D382DE9F04190461F4605464FF4BB
:10DDF0007A720023404639464BF084FC284B3C2184
:10DE0000034493FBF1F201FB1233AB7192FBF1F38C
:10DE100001FB13226A7140F2B551182293FBF2F410
:10DE200002FB143394FBF1F201FB1244B4F5896F49
:10DE30002B714FEA82032EDA40F2DA2294422CDC74
:10DE4000B4F5B77FB4BF00210121164A182000FBAA
:10DE500001220B2632F81600A04201DD013EF9D165
:10DE600003F5FA630B442B80731CAB700C2303FB8C
:10DE700001660D4B03EB46060134B6F8D230E41AC6
:10DE8000EC704FF47A720023404639464BF03AFC6E
:10DE90002A81BDE8F0810321D7E70221D5E700BF41
:10DEA00080BC92C7A6120608D4110608F0B5274D0B
:10DEB00006460F460FCD8DB06C460FC40FCD0FC474
:10DEC00095E80F0084E80F0016F003033AD16421AF
:10DED00096FBF1F201FB126242B94FF4C87296FB55
:10DEE000F2F302FB1363003B18BF0123721EC3F160
:10DEF0001D03002A019340F26D13104606FB03F345
:10DF0000B8BFB01C03EBA0006FF0630392FBF3F308
:10DF100018444FF4C87392FBF3F21044063069467C
:10DF200000240725013F51F8042BA74202EB000310
:10DF300093FBF5F0C0EBC000A3EB000004D1101A76
:10DF40000DB0F0BD0123D1E70134ECE7081306085A
:10DF5000084BD3E9C41251EA020309D0064BD3F8A7
:10DF600094315B1842F10002C0E900320120704791
:10DF700000207047283A00203029002037B5054698
:10DF80006846FFF7E5FF044638B1DDE9002328467F
:10DF9000FFF728FF204603B030BD40F20113288070
:10DFA0006B80A880A8712881F4E71FB50190FFF766
:10DFB000E5FF0199044648B1064B0DF10E02B3F896
:10DFC0001833ADF80E30084646F028FD204604B060
:10DFD00010BD00BF283A00202DE9F043994E87B0CC
:10DFE0000446A6F5DC7594F83030042B11D8DFE830
:10DFF00013F0130005005E00DE00250104F11C098A
:10E0000001AA49463046FEF776FC01280ED00228C8
:10E010002FD007B0BDE8F083304646F089FF4FF6B9
:10E02000FF732384012384F83030DCE7019F0FB1B4
:10E030003B7863B93046FDF7E9FE237EDF061BD54A
:10E0400046F076FF4FF6FF7323840223EBE797F841
:10E050000B8018F0080FD3D10B2204F131013846A0
:10E0600051F026F80028CBD1637E88EA0303D90655
:10E0700004D53046FDF7CAFE0423D4E7BA8A7B8B69
:10E0800043EA02436362D5F81022FB69A36052029F
:10E09000B3FBF2F102FB113109B113445B1AE360E7
:10E0A00084F819803046FDF7B1FE0323BBE795F8ED
:10E0B000E031002BADD104F11C08092701AA41462B
:10E0C0003046FEF718FC012850D1019888B3037838
:10E0D000E52B01D0002BF1D1FDF760FF5A4901EB90
:10E0E0000010FAF723FA01F5D070FDF78FFE202219
:10E0F0000021019851F042F8019BD4F831201A60B8
:10E10000D4F835205A60B4F839201A8194F83B20AD
:10E110009A72019B627EDA7203A8FFF746FF019BA9
:10E1200038BB6FF07E021A7447225A749873D87302
:10E1300038E095F8B831022B9ED095F8E031002BED
:10E140009AD1C5E97D33D5F8CC2185F8F03185F831
:10E15000EC31D5F8143285F8E071C5F8E421C5F842
:10E16000E8313046FEF7D6F90128A7D0022883D03F
:10E170004FE79DF80E109DF80F2042EA4112BDF8BE
:10E180000C10A1F2BC7142EA41221A829DF81020C3
:10E190009DF81110D20242EA41129DF8121042EA93
:10E1A0005102DA811A8A1A83DA89DA827DE7237EBC
:10E1B0009A0608D5E0690023112202A9FDF700FFA5
:10E1C00001287FF426AF204646F0B2FE2269237E66
:10E1D0008AB91B0708D51D4B93F89821002A7FF4B4
:10E1E00018AF072283F89821002384F82830E36AC7
:10E1F000204698470DE703F0F70213F00403227658
:10E2000008D00023E26AA16884F828302046FDF790
:10E210009FFEFEE6122AE7D1E26AA263626A84F8F0
:10E220003C300421C4E90B22C4E9023384F82810ED
:10E2300063636362204646F07BFEEAE60020E36A01
:10E240002070D6E7BC6000201C5F0020045F002027
:10E250002DE9F34103780446002B76D090F828305E
:10E26000013B082B71D8DFE803F00509475B4C61DF
:10E2700070666B0002B0BDE8F041ADE6344B456816
:10E28000D3F81072D3F818327F021D40216B20465C
:10E29000FDF7F6FD05EB01084745064626D880B197
:10E2A000D4E901329A422CBFA260A360002384F813
:10E2B0002830E36A002B48D0204602B0BDE8F04188
:10E2C00018472169207E01AA49F0DCFA01283CD1D7
:10E2D00023696361019B236163683B445B1B63604B
:10E2E000236BDB1B1D4425633546CFE7636800289D
:10E2F000D6D119446160D3E702B0BDE8F041FEF722
:10E300008FBA0121FEF7F8F901281ED1216C0023F4
:10E31000204684F8283002B0BDE8F041FEF7D4BAB8
:10E32000002102B0BDE8F041FEF7E6B902B0BDE859
:10E33000F041FEF781B902B0BDE8F041FEF785B8C3
:10E3400002B0BDE8F041FEF7E5B802B0BDE8F081EB
:10E35000045F0020F0B50124B0FBF4F58D4203D238
:10E3600000261CB91C70F0BD4C43F5E7B0FBF4F57A
:10E37000B4FBF1F704FB15002EB9002D03DC8C4231
:10E380000CD33C46EDE7092D08DD002A14BF3724E5
:10E3900057242C4403F8014B0136F2E73024F8E708
:10E3A000A0F13003DAB2092A01D818467047A0F16B
:10E3B0006103052B01D857387047A0F14103052BA5
:10E3C00094BF37384FF0FF30704770B50446944221
:10E3D00008461546B4FBF2F602D33046FFF7F5FFC8
:10E3E00005FB1644024B1B5D00F8013B70BD00BFEE
:10E3F0002BAF0608B5EEC00ADFED2D7AF1EE10FA6C
:10E40000CCBF30EE270A30EE670ADFED2A7A20EE25
:10E41000270A30B5FDEEC07A87B017EE904A054660
:10E4200084EAE470002303A9A0EBE470CDE9003393
:10E43000029346F06DFD002CACBF20232D2303A8D2
:10E440008DF800304AF096FA012822D130238DF859
:10E4500001308DF802308DF8033003A9684651F081
:10E46000DDFD68464AF086FA0338C4B222466946A2
:10E4700028464EF0E5FC00232B550F49284651F065
:10E48000CDFD0DEB0401284651F0C8FD284607B02C
:10E4900030BD022805D130238DF801308DF80230CF
:10E4A000DBE7032804BF30238DF80130D5E700BF38
:10E4B0006F12033A00007A442BE7060830B5027861
:10E4C000202A034600F10100F9D0092AF7D02D2AAD
:10E4D0004BD10346BFEE000A9FED3C7A1A46F2EE9E
:10E4E000046A134612F8010BA0F13001CCB2092CDA
:10E4F00041D92E280BD1F2EE046A1146B0EE666ABD
:10E500000B4611F8012B303AD0B209283CD91A78C1
:10E5100002F0DF02452A53D15A782D2A3FD1023327
:10E520000120013B00220A2513F8011F3039CCB22B
:10E53000092C3AD9B2F59A7F1346DFED256A28BF38
:10E540004FF49A731A46F7EE007A072A30D8DA08A1
:10E550006FF0070101FB0233F2EE046A63BB88B37C
:10E56000C7EE276A20EE260A30BD2B2A08BF0346D5
:10E57000B7EE000AB0E707EE901AF8EEE77AE7EE9A
:10E58000267AB0EE677AACE707EE902AF8EEE77AE3
:10E59000C7EEA65A66EE866A37EE257AB0E72B2AD2
:10E5A00014BF013302330020BBE705FB0212BBE7B7
:10E5B00067EEA67A083AC8E767EEA67A013BCDE790
:10E5C000F7EE007A67EE276ACCE700BF0000000094
:10E5D00020BCBE4C70B5034610F8012B202AFAD09F
:10E5E000092AF8D02D2A0ABF034601254FF0FF352E
:10E5F000591E00240A2611F8010FFFF7D1FE092841
:10E6000002D905FB04F070BD06FB0404F3E710B566
:10E610000023802804D893420AD2C854581C10BD45
:10E62000934205D060F07F04CC54C0090133F0E779
:10E630004FF0FF30F3E770B51249134C134E01222F
:10E640000020FEF700FC228862B1A31DB34217D25E
:10E65000A518B54214D2052A12D92146FEF7F3FBBC
:10E660002C46F0E721460222FEF7EDFB63880849BD
:10E67000084AC31A641A5842A2F8B444584170BDFB
:10E680000020FCE70040000801400008008000086E
:10E69000FC3F0008283A00202DE9F04F794BDFF8C5
:10E6A000F4818FB0A3EB0802CDE901234FF00309F9
:10E6B000102200210AA850F061FD019B0993029BE2
:10E6C0000893714BCDF81C801A69002ABFBF6F4AAE
:10E6D0005A6002F188325A600124F322DA604FF066
:10E6E000000A7E23224604A907A88DF83440CDF8FD
:10E6F00030A08DF81030FAF731F9504513DA0023C5
:10E70000B9F1010900F0B780002BD1D098F80030A2
:10E710007E2B40F0B380FFF78EFF002800F0AE8024
:10E720000FB0BDE8F08F224604A95046FEF78BFBE0
:10E73000574CDFF864B1ADF812005C453CD30024BF
:10E74000022205A907A8ADF81440FAF707F9A0427C
:10E75000D5DBBDF81200022205A9FEF774FB0222E8
:10E76000ADF812000DF1120107A8FAF7F7F8A04270
:10E77000C5DB0B9888B1079B089A03449342BED827
:10E780000AABC0F104022146184450F0F7FC0AA974
:10E7900007A8FAF740F8CDE90B400C9B002BAEDB45
:10E7A0009DF8342022B138490A6942F000420A61DA
:10E7B000B3FA83F35B09A3E762888DF819A0C2F36B
:10E7C0000B06B31DADF814302388C3F30B011B0BEC
:10E7D0008DF818301304ADF8161020D4062205A9C0
:10E7E00007A8FAF7BBF8002889DBBDF8120006225B
:10E7F00005A9FEF728FB6168ADF81200324607A8AC
:10E80000FAF7ACF80028FFF67AAFBDF8120061689D
:10E810003246FEF718FBADF8120014348DE70027DE
:10E820003D460135EDB2062205A907A88DF819501D
:10E83000FAF794F80028FFF662AFBDF8120006223E
:10E8400005A9FEF700FB6168ADF8120039443246B5
:10E8500007A80391FAF782F80028FFF650AFBDF839
:10E86000120003993246FEF7EEFA032DADF81200BE
:10E870003744D6D1D1E7002B7FF448AF052005F00F
:10E8800031F800BF00800008003C024023016745CA
:10E89000F816070800400008E41B0708034AD2F8EE
:10E8A000B83423EA0000C2F8B8047047283A0020C0
:10E8B000034606490648884201D300207047028873
:10E8C000C2F30B029342F9D01430F4E7E41B0708BB
:10E8D000F816070813B542880B460446C2F30B022C
:10E8E00000211846019250F049FC216903460A486C
:10E8F000814209D30948019A814205D2184602B0E3
:10E90000BDE810404EF09CBA21B1184602B0BDE8F7
:10E910001040084702B010BDE41B07088920070813
:10E9200010B4B0F902404288002C0B4641685DF8F3
:10E93000044BBEBFC2F30B02DBB203FB0211C9E7FB
:10E9400030B5094B094CA34200D330BDB3F90220C6
:10E950005988002A06DA5A68DD68C1F30B0100FB0A
:10E9600001222A601433EEE7F8160708E41B0708B3
:10E9700030B502460144002012F8015B082480EA09
:10E98000050313F0010F4FEA50001CBF80F08C0309
:10E99000D8B2631E13F0FF044FEA5505EFD18A4247
:10E9A000EAD130BD2DE9F04F87B0CDE90212002544
:10E9B000804604930195039B404603EBC50AFAF792
:10E9C00009FFEC00024600286DD0002201214046DC
:10E9D000FAF7EAFE0246002865D098F80430990755
:10E9E00061D5F0214046FAF7FFFE024600285AD0D2
:10E9F000039BA4F108024FF0000B012713443C468F
:10EA00005E460593029B002B55D0082C53D804F189
:10EA1000FF3943FA09F909F0010949464046FAF776
:10EA20009AFE024600283ED0002201214046FAF715
:10EA3000BBFE0246002836D098F8041001F0600CA6
:10EA4000BCF1600F4FEAD11016D0029B1BB1082C0D
:10EA500001D8814527D1002841D01AF80610394342
:10EA60007F00013417F0FF070AF80610E4B2C9D19D
:10EA70000136F6B2082E1CD1402C10D90721504681
:10EA80000592FFF775FF9AF80710059A814206D1A3
:10EA90000135EDB2BBF1000F05D0CDF804B0049BF9
:10EAA0001B78AB4287D8049B10461D7007B0BDE8A9
:10EAB000F08F0127A6E75DB1019BA34208D9059B12
:10EAC0009A5D174214BF4FF001094FF00009A4E707
:10EAD000019B1B1BD3F1000949EB03099DE7880942
:10EAE00040EA511111F0010F1AF8061008BFA346B1
:10EAF00021EA0701B4E700BF90F83C20034602F08A
:10EB0000FF0012B1002283F83C2070474FF480537D
:10EB1000838170474FF40063838170474FF4006333
:10EB2000838170474FF40063838170474FF4006323
:10EB3000838170474FF40063838170474FF4006313
:10EB40008381704710B5064A0423002152F8044B14
:10EB5000844208BF42F8041C013BF7D110BD00BF3E
:10EB6000286100203248F0B5C38B058AB0F92840EF
:10EB7000B0F91660B0F922C0B0F93070ED1A838B8D
:10EB80006B43B0F9265004EBE334ED0295FBF4F54A
:10EB900005EBE335A5F57A6E0EFB0EF42313B0F901
:10EBA0001840C5620EFB06F60EFB04FEB0F92040CD
:10EBB0005C4303FB0CFCF612241406EBEC2C04EB78
:10EBC0006E34B0F91460438B02340CEB860CA41045
:10EBD000466B04F500440CFA07FC63430CF1020C8D
:10EBE0004CF25030DC0BA6EBAC0640FA07F3734353
:10EBF00055BF5B00B3FBF4F3B3FBF4F35B0071B1FF
:10EC0000181240F6DE34404360430A4C00145C4363
:10EC100000EB244000F6CF6003EB20130B6022B121
:10EC20000A235D4308352D1115600120F0BD00BF9A
:10EC30002861002043E3FFFF012070470120704757
:10EC40002DE9F8435E4F1546BC6BBA8FB7F842907A
:10EC5000C2EB24135200C2EBE402B7F93E40624318
:10EC600003FB03F4B7F9403024135C43A41304EB13
:10EC7000E224B7F946307C650E46A4F5FA3181FBF3
:10EC800001CE4FEAE37803FB0EF20CFB0822A3FB54
:10EC90000C389044B7F9442082FB01021B0A12038E
:10ECA00043EA086342EA105200031B1842EB282291
:10ECB00002F50042A3FB093809FB02884FEAE8731A
:10ECC0004FEA680253EA68084FF000006CD0B7F9C9
:10ECD0004C904FEAE97809FB0EFE0CFB08EEA9FB0D
:10ECE0000C9CE644B7F94AC08CFB01814FEA414CC9
:10ECF0004FEA484111EB0909B96D4CEAD83C4EEB9B
:10ED00000C0CC1F5801E0EF00048B7F9481048EA17
:10ED10005E0810EB09004FEACE7EBEEB00000CEB64
:10ED2000C10168EB010C40F63548A0FB080108FB67
:10ED30000C114AF0E7FCB7F952304FEA613E4FEA56
:10ED4000503C4CEAC14C03FB0EF24FEAE3790CFB5A
:10ED50000929A3FB0C324A4403FB0EFE0CFB02EE16
:10ED6000A3FB0C3CB7F95020E6445B0E43EACE13FC
:10ED700013EB000C804602FB01F34FEAE27941EB12
:10ED80006E6EA2FB082809FB00314144D00C40EA1A
:10ED900041301CEB0000B7F94E304EEBE141000A68
:10EDA00040EA016000EB03100EB1000A306025B1AB
:10EDB00004EB8404803424122C600120BDE8F88325
:10EDC0002861002031B10A4BD3ED1D7AFDEEE77AC0
:10EDD000C1ED007A52B1064B9FED067AD3ED1E7A53
:10EDE00067EE877AFDEEE77AC2ED007A0120704780
:10EDF000286100200000C8422DE9F74FCDE900123C
:10EE0000554AB2F88A30D16FB2F88660B2F88C7089
:10EE10001B02C91AB2F888306EEB0E0EA3FB010478
:10EE200003FB0E44B2F88430C00940EA44601B047E
:10EE3000C018A6FB013506FB0E55B2F882604FEAFA
:10EE4000132343EA05634FEAC6364FEAE41444F15C
:10EE500000049B19A7FB012607FB0E664FEAD2525E
:10EE600042EA46224FEA252545F10005F61512F53E
:10EE7000FA6C46F1000BBCF5FA6F7BF100074CDA37
:10EE8000A2FB02784FF0050A02FB06F908EB4909DC
:10EE9000A7FB0A780AFB09884FEA570949EAC879AB
:10EEA000BF08B0EB090047EA887764EB6804DB1B16
:10EEB0002A4F65EBA805BC454FF0FF377BEB0707F2
:10EEC00020DA40F6AC57D21946F100065643A2FBB1
:10EED000027202EB46064FEAC608FA00BA1A48EA7E
:10EEE000577866EB0808101844EB08044FF00B083D
:10EEF000A7FB087208FB06267F0847EAC677DB1BDC
:10EF000065EB660501FB0EFEA1FB011202EB4E0E46
:10EF1000C90F41EA4E01BCEB010C009A9AB10E4AAE
:10EF2000D2F89010A1FB032301FB0535520D42EAF4
:10EF3000C522121A4FEA6555009B65EB0404D20BFB
:10EF400042EA44421A60019B0BB1C3F800C00120A1
:10EF500003B0BDE8F08F00BF2861002024FAFFFF56
:10EF600001207047B0F90000084B4143994208DB8B
:10EF7000B1F5000F07DA0029B8BFFF31081200B25F
:10EF800070470348FBE747F6FF70F8E701FF7FFF94
:10EF90000080FFFF064B0022C3F89420C3F898209E
:10EFA000C3F89C200022C3F8A0200120704700BFB6
:10EFB00028610020104B1A68104BD3F8A010521A89
:10EFC000FA2A16D8D3ED257AFDEEE77A17EE902AC5
:10EFD000D3ED267AC286FDEEE77A17EE902AD3EDBE
:10EFE000277A0287FDEEE77A17EE903A43870120F1
:10EFF00070470020704700BFC42A0020286100200D
:10F0000090F85F3230B53BB990F85D1290F85E32FF
:10F010000124DAB2914200D830BDB0F8665204FA49
:10F0200003F22A43A0F866220133F2E7437913F092
:10F0300001031FBFD0E90732C0689B1A00F1FF30FF
:10F0400014BF184018467047437913F002031FBFDE
:10F05000D0E9093200699B1A00F1FF3014BF9843D0
:10F060001846704710B5437913F0010301460DD0DF
:10F07000FFF7DCFF60B10A6A4B69C8689B5C01322C
:10F08000B2FBF0F400FB1422DBB20A62184610BD9A
:10F090000346FBE743799B070AD5436A8269D1544B
:10F0A000436A02690133B3FBF2F102FB113343629D
:10F0B000704741717047D0E90920131A58425841EE
:10F0C0007047024BD3F8A4305B68184728610020D2
:10F0D000024BD3F8A43008309B6818472861002001
:10F0E00001207047012070470120704701207047C0
:10F0F0000120704731B10C4BD3ED2A7AF8EEE77A54
:10F10000C1ED007A7AB1084BDFED086AD3F8AC3074
:10F11000A3F5D543333B07EE903AF8EEE77A87EE56
:10F12000A67A82ED007A7047286100200000C8426C
:10F1300001207047012070477047044B03EB8000AB
:10F14000D0F8B0300BB19B6819607047286100207F
:10F1500008B50246FFF7F1FFBDE8084010461FF072
:10F16000C9BD054B03EBC00040F2FF739942A8BF35
:10F1700019468180704700BF903D00200C4A1378EB
:10F180007BB10C4B93F8F01059B193F8F11059B1D1
:10F1900050680021FA2883F8F110A8BF4FF0FF3023
:10F1A00070476FF0010070476FF00200704700BFBA
:10F1B00038100020286100200B4B93F8F2206AB130
:10F1C00093F8F3206AB1002283F8F320074B986884
:10F1D000B0F5967FA8BF4FF0FF3070476FF0010089
:10F1E00070476FF00200704728610020381000203F
:10F1F000024BD3F8F4305B68184700BF2861002049
:10F20000024BD3F8F4309B68184700BF28610020F8
:10F21000024BD3F8F430DB68184700BF28610020A8
:10F22000014BD868704700BF38100020044B93F89A
:10F23000F83013B1034B186970476FF00100704745
:10F2400028610020381000202DE9F043062592F9AE
:10F25000007087B06B43144612F80580A0EB080ECF
:10F26000A0EB070CBEF1000FB8BFCEF1000EBCF151
:10F27000000FB8BFCCF1000CE64502EB050905F123
:10F280000605BCBF4FFA88F74C46AB421646E3D1A1
:10F290001A443378BB420CD1658873884D1BCB1A56
:10F2A000002DB8BF6D42002BB8BF5B429D42C8BF66
:10F2B00034460636B242ECD1637904932379039342
:10F2C000638802932378064ACDE90013034603219D
:10F2D0000120FEF76FFB204607B0BDE8F08300BFBA
:10F2E000D5AF060808B5006848F057F8014BD86755
:10F2F000012008BD2861002008B5006848F04DF8DD
:10F30000024BC3F89000012008BD00BF2861002017
:10F3100038B514460D46002943D0344B9FED346A6E
:10F32000D3ED3F7AB3F91421F8EEE77AC7EE866A97
:10F3300007EE902AB3F9102107EE102AF8EEE77ACB
:10F34000B8EEC77AB3F91221A6EEA77AD3ED427AC6
:10F35000F8EEE77AE6EE877A93ED417AB8EEC70ADF
:10F36000A6EEA70A07EE902AB3F90E2107EE102A9F
:10F37000F8EEE77AB3F90C21B8EEC77AA6EEA77AD1
:10F3800007EE902AF8EEE77AE6EE877A93ED467A72
:10F39000B8EEC77AC7EE066AA6EEA70A4AF042FFA1
:10F3A00028600CB3114BDFED126AD3ED467AB3F946
:10F3B0000021B3F90231F8EEE77A07EE102A87EE62
:10F3C000A60A07EE903AF8EEE77AB8EEC77A60EE52
:10F3D000277AF6EE006AE7EE267A9FED060A27EE18
:10F3E000800A4AF01FFF2060012038BD28610020FC
:10F3F0000000F04A0000C84238B50B4D55F83030D7
:10F4000007EE901A04466BB193ED047A93ED030A6C
:10F41000F8EEE77AA7EE870A4AF004FF55F8343091
:10F420009B68186038BD00BF903D002010B50C4BA4
:10F430000C4C1B68D4F81C011B1AFA2B06D90420AB
:10F4400019F0E8FE002084F8200110BD11B1D4F8B5
:10F4500024310B6012B1D4F8283113600120F4E795
:10F46000C42A0020286100202DE9F0410C4DDFF86E
:10F4700034802C686B6901271C400CB9BDE8F08111
:10F48000B4FA84F3C3F11F0307FA03F608EB83030E
:10F4900024EA0604D3F82C01036898476E61ECE770
:10F4A000003C01402861002010B5114CD4F86C01DB
:10F4B00018B1104A6421FAF769FBD4F86C010021F5
:10F4C000FAF7BCFBD4F86C315B681A68B2F84430C8
:10F4D0006FEA43436FEA53439BB2A2F84430138868
:10F4E0009BB243F001031380012384F8703110BDF7
:10F4F00028610020009F240010B50B4CD4F86C014B
:10F5000018B10A4A0321FAF741FBD4F86C01002133
:10F51000FAF794FBD4F86C010549BDE8104040F2BD
:10F520002B3245F00DBC00BF28610020009F240055
:10F530009C62002037B583681C686379DB0724D59B
:10F54000A57994F85C3205F001010D46FBB1E06B42
:10F5500043681A68D36AC3F34E03536294F86D325A
:10F56000012B07D094F8613223B1B4F8683201332B
:10F57000A4F8683285F0010145F030FB0023A4F8BF
:10F5800066324FF08073C4F85C3203B030BD94F83B
:10F590005F320191012B04BF94F85D3284F85E3232
:10F5A0002046FFF72DFD94F85F32019953B90123EE
:10F5B00084F85F3285EA0301E06B03B0BDE83040B8
:10F5C00045F00CBB002384F85F32F5E7F0B52DED74
:10F5D000028B83B00E46154642F09EF800286BD091
:10F5E000374B384C1B6894F8202E03F00203002A96
:10F5F00047D0002B5BD0344F0DF1060023F066F8A6
:10F60000D7F8EC23BDF806309FED307A9B1A07EE51
:10F61000903AF8EEE77AF0EE408A87EE870A07F52F
:10F62000806704F62464DFED2A7A20EE270AFDF7CE
:10F6300003FD97ED008AA0EE688A3CF091FDD4EDC1
:10F64000020AD0ED057AB0EE480A70EEA70AFEF77E
:10F6500025F97EB1DFED1F7A9FED1F7A20EE000ABB
:10F6600020EE270AC0EE077A9FED1C7A77EE877AA4
:10F67000C6ED007A0DB11A4B2B6003B0BDEC028BC6
:10F68000F0BDA3B1B4F9523E01EE103AB4F9503EC8
:10F6900000EE903AB4F94E3E00EE103AB8EEC11AC0
:10F6A000F8EEE00AB8EEC00AFEF7FFF8D1E7D4F8AA
:10F6B000683E93ED340ACCE79FED0A0AC9E700BF24
:10F6C000F427012028610020849C00200000C8420B
:10F6D00035FA8E3CCDCC9C3F00409C4682E6C54727
:10F6E000331390430000000008B5202150F0A5FC22
:10F6F000034620B11A78202A00F10100F8D01846FC
:10F7000008BD70B50D461446FFF7EEFF0646A0B1E2
:10F71000FEF760FF40F634039842A8BF1846B0F5E4
:10F72000617FB8BF4FF46170A0F561731920B3FB1E
:10F73000F0F32B702378013323703046FFF7D4FFAA
:10F740000646A0B1FEF746FF40F634039842A8BF34
:10F750001846B0F5617FB8BF4FF46170A0F56173D2
:10F760001920B3FBF0F36B7023780133237030461C
:10F7700070BD144951F8200070B500B30C2202FB93
:10F78000001292F96D3E581C1AD092F8750EB0B165
:10F79000C8188C2590F8C06E92F8744E0020142280
:10F7A0006B431D1901EB4505013AB5F8C45E3444BD
:10F7B00010FA85F0F5D11423B0FBF3F080B270BDE0
:10F7C0000020FCE72861002038B503200D461446D0
:10F7D000FFF7CFFF07EE900A8DB19FED0B7AF8EEA1
:10F7E000677AF0EE006A67EE877AB8EE047AA7EEE1
:10F7F000A67ADFED067A67EE277AC5ED007A0CB1BE
:10F80000034B236038BD00BF6740533A00007A4481
:10F810003313904310B5427A044632B10146406832
:10F8200051F80A3B98470023637210BD10B4447A24
:10F83000621C0444D2B24272A172037A934202D88B
:10F840005DF8044BE6E75DF8044B7047EEE710B552
:10F8500003681A79022A044602D1987A47F08EFD8D
:10F8600000232360237110BDF0B50D4B0D4E0446EF
:10F87000B34201D30020F0BD587988420DD11D79E3
:10F88000A54200D04CB9D879904206D118680779C2
:10F89000AF4202D105689D42EDD00C33E8E700BFCE
:10F8A000580300080805000873B50279022A38D108
:10F8B00090F910308DF802200324142673438DF83C
:10F8C00003401A4C1A4EE35800250120B3428DF82C
:10F8D00000508DF8010026D0164DAB4203D01648DB
:10F8E00083421ED1104601F108020DEB02011A8875
:10F8F00011F8085C22F040021204120C14211A8044
:10F9000001FB00401A88C16822F0380231F8251046
:10F910001204120C0A431A801A8892B242F0400272
:10F920001A8002B070BD2846DDE700BFB00000209D
:10F930000030014000380040003C0040C36910B571
:10F94000044623B909211420FEF7FEF8E061E069BE
:10F9500010BD10B504460068FFF7F0FF8378DBB1F7
:10F96000B0F90A3007EE903AF8EEE77AC4ED057A7E
:10F97000B0F90C3007EE903AF8EEE77AF1EE677ADC
:10F98000C4ED047AB0F90E3007EE903AF8EEE77A5B
:10F990000120C4ED067A10BD1846FCE710B50446F8
:10F9A0000068FFF7CBFF8378CBB1B0F9043007EEE6
:10F9B000903AF8EEE77AC4ED047AB0F9063007EE33
:10F9C000903AF8EEE77AC4ED057AB0F9083007EE20
:10F9D000903AF8EEE77A0120C4ED067A10BD184699
:10F9E000FCE710B504460068FFF7A8FF8378CBB1A9
:10F9F0008388DBBA07EE903AF8EEE77AC4ED047A32
:10FA0000C388DBBA07EE903AF8EEE77AC4ED057AE0
:10FA10000389DBBA07EE903AF8EEE77A0120C4EDED
:10FA2000067A10BD1846FCE710B500680C46FFF7D3
:10FA300085FF83784BB143892222DBBA93FBF2F333
:10FA400003F26D132380012010BD1846FCE738B582
:10FA500000680D461446FFF771FFD0F8013007EE3D
:10FA6000103ACDB1D0F80530DFED166A9FED166A79
:10FA700007EE903AF8EE677A77EEE67A77EEA77AB5
:10FA8000C7EE866AF7EE007A76EEE77ADFED0F6A68
:10FA900067EEE67AC5ED007A9CB1DFED0D7ADFED19
:10FAA0000D6AB8EEC77A27EE277AC7EE267A9FED61
:10FAB0000A7A77EEC77A9FED097A77EE877AC4EDF6
:10FAC000007A38BD9AC9CC449AC94C460E76D745BF
:10FAD0000000484300E0FF4400004842339388435D
:10FAE00037B500680D461446FFF728FFD0F80530FB
:10FAF0009FED237A07EE903AF8EE677A77EEC77AB1
:10FB00009FED207A67EE877AB3EE097A67EE877AFF
:10FB1000B2EE047AF4EEC77AF1EE10FA06DCBAEE31
:10FB2000047AF4EEC77AF1EE10FA0CD517EE900ACB
:10FB300049F08CF8144ACDE9000104210320FDF7B7
:10FB400039FF03B030BDD0F8013007EE103A2DB1C7
:10FB5000DFED0E6A67EEA67AC5ED007A002CF0D0D4
:10FB6000B8EE477ADFED0A6ADFED0A7AE7EE267A29
:10FB70009FED097A77EE877AC4ED007AE1E700BF5E
:10FB800000000046000080380EB006080AD778430F
:10FB90000319C83D000048C2339388430379022B00
:10FBA0000DD190F9103014225343064AD3581A89C4
:10FBB000920746BF1889C0F3C0100120704700208B
:10FBC000704700BFB00000200368DB6B13B504462C
:10FBD0002BB923685B6B3BB9FF23E38202E09847B4
:10FBE0000028F6D102B010BD214601A89847002890
:10FBF000F2D0BDF80630013B9BB2EEE710B50368CA
:10FC000004469B68984701236374FF23A37410BDC7
:10FC1000036810B504461B689847236820469B6814
:10FC20009847E37C0133E37410BD036810B50446C4
:10FC30005B689847236820469B689847E37C013BB4
:10FC4000E37410BDF0B585B0044618460D4616465F
:10FC5000039348F08FFE2268E67328440021A073C6
:10FC600000915769039B324629462046B84705B0A4
:10FC7000F0BD30B5046885B0E469089D34B10DB9B4
:10FC80000DF10F050095A04705B030BD2046FBE7FC
:10FC900003685B6A184703689B6A184710B5037BC3
:10FCA00004460BB1437B13B92046FFF7F4FF2368EA
:10FCB0002046DB68BDE81040184703685B6C03B161
:10FCC0001847704738B504468B6801600D46984761
:10FCD0000B4B2361002323752B6B13B120469847F0
:10FCE0002075084B93F814311BB1237D23F00103D9
:10FCF00023750023E3822046BDE8384064E700BF57
:10FD00000001FF002072002003681B6803B1184740
:10FD1000704703685B6803B11847704703681B6A44
:10FD200003B11847704703685B6A03B1184770470F
:10FD300030B40468A46A14B1A44630BC604730BC37
:10FD4000704730B40468E46A14B1A44630BC60471C
:10FD500030BC704703685B6C03B118477047036899
:10FD60009B6C03B11847704703689B6F03B118473A
:10FD700070470368D3F8803003B1184770470368B1
:10FD8000D3F8843003B1184770470368D3F888303C
:10FD900003B11847704721B10B68D3F88C3003B119
:10FDA00018470020704738B5094B052404FB003084
:10FDB000A0F1A00515F8010B013C47F02CF814F058
:10FDC000FF04F7D12046BDE8384047F024B800BF13
:10FDD000C813060810B5441E14F8010F00B910BD71
:10FDE000FFF7E1FFF8E7FFF73FBBFFF73DBBFFF78A
:10FDF0003BBBFFF739BBFFF737BBFFF735BB30B174
:10FE0000036882881B691A4214BF012000207047D2
:10FE100010B1036882881A83704710B10368828822
:10FE20005A83704737B50C46054600B30368114A3C
:10FE300003F13F4303F57E0302EB932393F8A30200
:10FE400045F044F8AB88009304F003038DF80430C8
:10FE5000C4F381038DF805302868C4F300136946A4
:10FE600064098DF806308DF80740FAF721FA03B0DF
:10FE700030BD00BFC8130608F7B50C461546064648
:10FE8000A8B303681B4A03F13F4303F57E0302EB6B
:10FE900093230F2793F8A30245F018F83068B6882B
:10FEA0000096B6FA86F3C3F11F0303F00702C3F30B
:10FEB000CC0300EB83039200196A974021EA070103
:10FEC0001962196A95400D431D6204F003038DF811
:10FED0000430C4F381038DF805306946C4F3001380
:10FEE00064098DF806308DF80740FAF7E1F903B0A0
:10FEF000F0BD00BFC813060838B50409013C032C47
:10FF000000F00F021AD80E4D05EB4403B3F8AA1205
:10FF100041FA02F313F001000FD0012303FA02F2B9
:10FF2000013A02EA01002C4450F0D8FF94F8B232B2
:10FF30001844044B0C2202FB003038BD0020FCE7C3
:10FF4000C8130608387300202DE9F04F54220446E8
:10FF500093B0B84800214FF011F9B74A601E15461A
:10FF60000334134610F8011F4E1E052E88BF0021D2
:10FF7000844245F8041BF5D1AF48002150F8044BEA
:10FF8000012C00F04E8101310429F7D1002152F8F3
:10FF9000040B022800F03C8101310429F7D1032031
:10FFA000FEF7D0FD0420FEF7CDFD0520FEF7CAFDCB
:10FFB0000620A24E9F4CDFF89482FEF7C3FD4FF05F
:10FFC0001A094FF0000A06F52E77207B38B394F912
:10FFD0000D50FFF791FF28B105238371002380F8AE
:10FFE000079003721321FFF71DFF227B002317F8F0
:10FFF0003310914240F0DC8006EBC303D3F8BC32EF
:020000040801F1
:100000002361182303FB0585AB6A23755A1C07235C
:10001000A3750123AA62637585F824309A4409F117
:1000200001095FFA89F9B9F1200F04F10C04CCD170
:10003000BAF1000F00F0B980814CDFF814924FF054
:100040000008237C002B00F0A6806079794D44F0F5
:100050003DFF207944F03AFFA068FAF7A1F80023A9
:10006000CDE90E33CDE91033069308932368A068D9
:10007000CDF814904C330493E3680393636914221E
:10008000534307934FF480624FF40063CDE9092393
:100090004FF400514FF48073CDE90B134FF400334C
:1000A00003A90D9344F022FEA268136843F00103F4
:1000B0001360644A536823F4733323F4477323F0C3
:1000C000030343F440335360226863695168012B92
:1000D00021F04071D4BF0020012021F4807141EA59
:1000E0000021516090685849014041F0020191603F
:1000F000D16A013B21F47001DBB241EA0353D362C0
:100100004FFA88F101239C4601914FF01F0E697D43
:1001100051B395F90D100198814225D1297CAE7D0E
:100120005F1C0929FFB249D9A1F10A00D2F80CA03D
:1001300000EB40004FF0070B0BFA00FB2AEA0B0A1A
:1001400006FA00F040EA0A00D060062B44D8013BD2
:10015000506B03EB83030EFA03F620EA060001FA64
:1001600003F3034353633B460CF1010CBCF1070F4F
:1001700005F10C05CBD1936843F400739360936849
:1001800043F480739360936843F001039360936832
:1001900043F08043936008F10108B8F1030F04F1C4
:1001A000180409F58C797FF44CAF13B0BDE8F08FDB
:1001B0000133102B7FF41BAF002321E7106901EB03
:1001C000410A4FF0070B0BFA0AFB20EA0B0006FA74
:1001D0000AF630431061B8E70C2B0CD8073B106BC4
:1001E00003EB83030EFA03F620EA060001FA03F399
:1001F00003431363B7E70D3BD06A03EB83030EFAA7
:1002000003F620EA060001FA03F30343D362AAE7E8
:10021000212283F8842E93F8C02E013283F8C02E59
:10022000BDE6112183F8781E93F8C01E013183F8D2
:10023000C01EABE6946F002028610020C81306089A
:100240004C10002000230140FDF7FFC038100020B3
:10025000EC6F00202DE9F0479846AB4DAB4B9D422B
:1002600021D26C798C4240F063812C79844202D097
:10027000002840F05D81EC79944240F059812C686F
:10028000DCB11C220021201D4EF078FF25602B7967
:10029000237195F806A0C4F808A02A7AE260012B21
:1002A00003D0022B0CD0002407E0E87AFFF724FEED
:1002B0006B7A2374AB7AA06163742046BDE8F08743
:1002C000E87AFFF719FE95F90960A0612674A87A0B
:1002D000FFF712FE6061002800F0128114238C4D9C
:1002E0007343EF18EB58002B00F00A81BB7C002B06
:1002F00040F0C080387A44F0E9FD3B7A03F01F02F9
:100300005B090121023B01FA02F2032B08D8DFE866
:1003100003F06C6602607F490B6923EA02020A61FE
:10032000142303FB0653771C5879FFF7E5FDFFB252
:10033000814618B140F60A33C3800772142303FBC9
:100340000653D879FFF7D8FD18B140F60A53C38099
:100350000772142303FB06539879FFF7CDFD18B1FC
:1003600040F60A43C3800772142707FB06571AF0AA
:10037000040A7A7A3FD04A214846FFF77DFDF87992
:10038000FFF7BAFD7A7A2A21FFF776FDB879FFF7F1
:10039000B3FD7A7A142707FB06570A21FFF76CFD95
:1003A000387928B1FFF7A8FD7A7A0921FFF764FDB3
:1003B00014237343EA58584B9A4226D103F58433E9
:1003C000596A41F480515962596A21F48051596245
:1003D00028E050494B6923EA02024A61A0E74D49EF
:1003E0000B6A23EA02020A629AE74A494B6A23EA45
:1003F00002024A6294E70A214846FFF73DFDF87978
:10040000FFF77AFD7A7A0A21BEE7444B9A4240D13F
:1004100003F50033196A41F480411962196A21F425
:1004200080411962BAF1000F67D000231846118885
:10043000034301F441510B4343F445731380938B01
:1004400023F400631B041B0C93830723138213887C
:100450009BB243F040031380142303FB0653187927
:1004600018B1FFF749FDFFF7D3FC142303FB065532
:100470000123AB74606928B10E23C371002380F897
:10048000068003720921FFF7CDFC6069FFF7C0FC0D
:1004900013E7234B9A4209D103F5FE33196A41F45D
:1004A00000411962196A21F40041BAE71D4B9A42D2
:1004B00009D103F58233596A41F400515962596AEE
:1004C00021F4005183E7184B9A4209D103F56843A0
:1004D000596A41F480115962596A21F4801176E712
:1004E000124B9A429ED103F56443596A41F40011BC
:1004F0005962596A21F4001169E70123022096E745
:100500002046FFF7A4F9CEE65803000808050008C6
:10051000B0000020003802400030014000380040A8
:10052000003C0040003401400050014000540140B4
:100530000C3594E6074B03EB8000D0F838333BB121
:100540009A881B6859690A4201D05A8370471A83F6
:10055000704700BFC8130608094B03EB8000D0F8B2
:10056000383349B903B970471A689B8813837047B9
:100570001A689B8853837047002BF9D1704700BFDE
:10058000C81306082DE9F74FDFF8AC8198F8700121
:10059000002840F0CE80D8F86C3101931B7C002BF2
:1005A00040F0C780DFF894C19CF866239CF867335D
:1005B0009CF86853ACF864030CF26A3A86463C2611
:1005C0009AF802109AF80370C1F1FF0189B200296C
:1005D00000F0AB80C1F1FF017943BAF80040B4FBF1
:1005E000F6FB0912BBF1050F1FD8DFE80BF0030D76
:1005F000616F808E7B1A6343B3FBF6F353FA81F38A
:10060000CDB2DBB23A460FE0B4FBF6F206FB124283
:1006100092B2C2F13C027C1A6243B2FBF6F252FA89
:1006200081F2CDB2D2B23B460120170247EA03471E
:100630002F4300240121C4F1170B01FA0BFB1BEA25
:10064000070F0EEB040908BF8B4609F12A0189B296
:1006500008EB810104F1010418BF4FF0020B182CC4
:10066000C1F874B1E6D10EF1180E1FFA8EFEBEF578
:10067000407F0AF1040AA3D1ACF8EAE328B18CF870
:1006800066238CF867338CF868532023ACF8643306
:100690009CF8EC33002B4CD0019840F22B31F9F749
:1006A0000BFCD8F86C0103B0BDE8F04FF9F736BC8D
:1006B000B4FBF6F306FB13447D1AA4B2CAB2654339
:1006C000B5FBF6F555FA81F1CDB2ACE7B4FBF6F324
:1006D00006FB13439BB2C3F13C037C1A6343B3FB99
:1006E000F6F353FA81F3CAB2DBB23D469CE7B4FBA2
:1006F000F6F006FB10447A1AA4B26243B2FBF6F29B
:1007000052FA81F2CBB2D2B2EFE7B4FBF6F506FBB8
:100710001545ADB2C5F13C057C1A6543B5FBF6F550
:1007200055FA81F5CBB2EDB26CE73D463B463A4611
:100730007AE703B0BDE8F08F286100202072002026
:10074000F8B500212520F9F707FA064608B3FDF7AA
:1007500035FA214F0446C7F86C01D0B12520FFF7C8
:10076000CBFB1E4DC5F8F00320B140F21523C3802A
:1007700000230372327A4A21FFF77EFB95F8F433A7
:10078000022B07D1FEF790FE2046F9F767FB002306
:100790000360F8BD032B06D1FEF786FE2046F9F76D
:1007A0005DFB6423F4E7FEF7A7FE10B985F8EC03C0
:1007B000EFE70B4840F6AC4200214EF0DFFC95F825
:1007C000F433012B04BFFF23C7F81C3E012385F837
:1007D000EC33BDE8F840D5E6286100202072002007
:1007E0009C620020F8B5134BD3F86C41054604B366
:1007F00093F87011C9B9E06866688268136823F0DD
:1008000001031360326877790B4E938936F81760CD
:100810009BB223EA06039381217413889BB243F0B1
:10082000010313800177FEF73FFE2046F9F716FB20
:100830000560F8BD28610020D411060838B5114BB9
:10084000D3F86C0158B193F8702142B10E4C94F872
:10085000F423032A04D1F9F701FB6423036038BDB4
:10086000022A4FF0000503D1F9F7F8FA0560F6E720
:1008700083F87051FEF740FE0028F0D184F8EC03B5
:10088000EDE700BF28610020207200208379806B93
:10089000DB0748BF81F0010109B1FFF7B9BAFFF7E3
:1008A000BCBA10B5837913F0010F03F0200204469F
:1008B000C36B12D05B68002A1A7A14BF022142214E
:1008C000606BFFF7D9FA0121E06B84F86012A4F89D
:1008D0005C12BDE81040F9F7D7BA5B68002A18BF70
:1008E00002211A7A08BF2221EAE7036C806B23B148
:1008F0005B6801211A7AFFF7BFBA0121FFF792BAAC
:1009000070B583681C6863799A0731D594F8615291
:10091000D5B194F962329BB1B4F864124B08A4F8D3
:100920006432204601F00101FFF7B0FF94F8623213
:10093000A279013B5BB2500684F8623218D5BBB98C
:10094000002384F8613213E0A36A626A94F86012AB
:100950009A4226D161B9A3791B0709D5236CA06BF4
:10096000DBB15B681A7AFFF787FA2046FFF799FF39
:100970006379D90740F1818094F85C32002B7CD1F7
:1009800094F85D320133DBB2092B84F85D3235D146
:100990002046BDE87040FEF733BB1946FFF742FA28
:1009A000E3E75A1CA069A262C35C26695B0043F4BA
:1009B0000073A4F864320A23B24234BF10462846BA
:1009C00084F862320123A06284F8613291B1A37984
:1009D0001E070FD5E06B2946F9F756FAE36B606BFB
:1009E0005B6829461A7AFFF747FA84F86052204676
:1009F000FFF77BFFA3795D068BD4B9E70A2B3CD1C7
:100A000094F85F322BB9B4F8663243F00103A4F8CE
:100A10006632B4F86602820501D4C3071AD4B4F86A
:100A20006A320133A4F86A3294F85F5201239D427E
:100A3000A4F85C3221D1A179E06B002384F85F3205
:100A400001F0010144F0CAF8E06B2946BDE87040AE
:100A5000F9F71ABAE36AC0F3470013B1216B98475C
:100A6000E2E7E3696269D054E369E2680133B3FB0A
:100A7000F2F102FB1133E361D6E770BD234B1A6834
:100A800010B513460446B3FBF1F0B0F5803F03D335
:100A9000012BFAD95B08F6E781B22046F9F776F820
:100AA00023681B68587990B1032140B2F8F761FFC1
:100AB00023681B685A7993F90530002B07DB02F095
:100AC0001F0101228A405B09114941F82320236854
:100AD0001B68987990B1032140B2F8F74AFF236868
:100AE0001B689A7993F90630002B07DB02F01F018F
:100AF00001228A405B09064941F8232063681A688D
:100B000013889BB243F00103138010BD60060020E0
:100B100000E100E08160C06BB0E7002ABCBF801834
:100B20005242002BBCBFC9185B420028BCBF121A3E
:100B30000020F0B584180029A4F11D04BCBF5B1887
:100B40000021002CC8BF121BCC180F3C002CC8BFC2
:100B50001B1B0B4E02440B443C274FF0200C9042D1
:100B60000CDC06EB40050C4604E007FB04FE0134F8
:100B700025F80EC09C42F8DD0130F0E7F0BD00BF63
:100B80001876002008B5114B1A6C42F080521A6496
:100B90000F4A012111620F4AFF215162CA2151629D
:100BA000532151625B6FDB0005D50020FAF7C2F9D3
:100BB000094B984209D000210120FAF7ABF9BDE8B2
:100BC000084005490020FAF7A5B908BD00380240E1
:100BD00000000E420028004076614E6970B5044660
:100BE000012022F01FFC58B103684BB11A4A237947
:100BF00092F83C1092F83D209A422BD08B4229D09B
:100C0000164B5E68710612D500212720F8F7A4FF65
:100C1000002105462620F8F79FFF1DB12A682368AA
:100C20009A4217D018B1026823689A4212D0F20390
:100C300008D500212520F8F78FFF18B12268036836
:100C40009A4207D02079112804D0A0F121035842FC
:100C5000584170BD0120FCE74C030020F42701201F
:100C6000094A30B505460A2400201368AB4205D175
:100C7000D3688B421EBF431CD160D8B2013C02F145
:100C80001402F2D130BD00BF980500202DE9F74FC6
:100C9000384DDFF8E880DFF8E8904FF0000B0646AB
:100CA0002F465C46AA463A68002358F833108A4219
:100CB00043D1DBB24B4493F8B837012B42D0022B1F
:100CC00049D038460192FFF789FF78B9142303FB16
:100CD0000BA3019AD96801F00C03042B06D110462E
:100CE000FFF7BEFF0134E4B20444E4B20BF1010BA0
:100CF000BBF10A0F07F11407D5D11F4F2846FFF7A4
:100D00006DFFA0B9E9684B0711D501F00C03042B66
:100D10000DD0A64227D921F0080141F0040128682E
:100D2000E960FFF79DFF0134E4B20444E4B21435F6
:100D3000AF42E3D103B0BDE8F08F01330E2BB4D145
:100D4000FF23B7E7FB681807BBD523F0080343F080
:100D50000403FB60B5E7FB685907B2D523F0040331
:100D600043F00803F5E721F004012868E960FFF784
:100D700077FFDCE798050020600600202C120608AB
:100D80002072002010B5044608462060194608B1BC
:100D9000F8F7FCFEBDF808102068F8F74FFF206850
:100DA00043681A68B2F844306FEA43436FEA53432A
:100DB0009BB2A2F8443013889BB243F00103138026
:100DC000F9F74CF80023A060036010BD2DE9F04F47
:100DD00085B099469DF83C30039307468A46904675
:100DE000FCF7ECFE054650B1224B93F8C6170729D5
:100DF00009D9214A00210420FCF7DCFD0025284602
:100E000005B0BDE8F08F4A1C5C205FFA82FB83F8D6
:100E1000C6B703F5F96600FB013301FB006600214C
:100E2000C3F8C81783F8CC173879FFF765F804467C
:100E300028B1022380F806A0C37180F808B0039B94
:100E40007BB13A7A02212046FFF716F8BDF8383018
:100E5000009329464B4642463046FFF793FF3546FE
:100E6000CDE720461121FEF7DDFF2046FEF7D5FF36
:100E7000ECE700BF2072002030B006082DE9F347F0
:100E8000394C94F8A83A0746002B6BD094F8A96A1D
:100E900094F8AA3A0136F61A102E0DDD022384F8D2
:100EA000AB3A324A10230093002133460420FCF76A
:100EB00081FD02B0BDE8F08794F8B43A012B11D05F
:100EC000022B13D02A4B94F8B41AC4F8B83A11F094
:100ED000FD010FD0274A0221042002B0BDE8F047EF
:100EE000FCF768BD45F098FB234BECE745F094FB1D
:100EF000224BE8E77B68B34229DBDFF89480DFF818
:100F00008090DFF890A028370D46B542D1DADAF8A4
:100F10000420B4F8AE3AB9FBF3F3C2F300720192C5
:100F2000B4F8AC2A00920321154A57F8040B9BB27F
:100F3000FFF74CFF014688B90523124A84F8AB3A03
:100F400004202B4602B0BDE8F047FCF733BD042077
:100F500000930D4A84F8AB0A3346A8E748F8040B1F
:100F60000135D2E7094AB6E7207200206BB00608C7
:100F70003BF1000897B00608F5EC020851F10008B3
:100F800040420F0009B10608D3B006082EB106088A
:100F9000D8610020F427012030B51E4B2DED028BC7
:100FA0001C68B4FBF1F303F57F4383B0FF331B0CE4
:100FB000B4FBF3F40023B4FBF1F501920093224655
:100FC000ABB20221F0EE408AB0EE608AFFF7FEFE7F
:100FD000E0B107EE904AB5EE408AF1EE10FAF8EE75
:100FE000677A0ABF07EE105A67EE880AF8EE470ADA
:100FF0009FED097AC0EE876A0123037127EE667AB6
:10100000C0ED046AA7EEA87A80ED037A03B0BDECC8
:10101000028B30BD6006002000007A4400230649A0
:1010200010B51C46984200DC10BD51F833200AB1BF
:10103000926814600133F5E7903D002013B50F4C22
:101040008DF80700D4E90423A16853438B4212D0E2
:101050006368E0680DF1070118444BF0F1FE636826
:1010600022691344A268B3FBF2F102FB11336360FF
:1010700063690133636102B010BD00BF683D0020A9
:101080000F4B1B78062B14D8DFE803F01613040768
:101090000A0D10004FF4FA6070470A4B98887047A9
:1010A0004FF47A6070474FF4FA5070474FF47A501B
:1010B00070474FF47A7070474FF4C870704700BFA4
:1010C000443D0020D03E00202DE9F04F2DED028B55
:1010D0006A4B6B4E1F780C2F85B081460FDD0123C4
:1010E00086F8AB3A674A0C2300933B460021042064
:1010F000FCF760FC05B0BDEC028BBDE8F08F624BE5
:101100009C79624B032C1C7013D9231F022B12D91C
:101110005F4BC6F8BC3A5F4B13F81430F3B95E4A24
:101120000221042005B0BDEC028BBDE8F04FFCF7B6
:1011300041BC5A4BEDE7FFF7A3FF594A594B80B228
:10114000B3FBF0F000235360574B10604FF0000AE0
:101150004FF0000BC3E900AB544BDAE7D9F800308D
:10116000BB421ADB524CDFF874B19FED528A09F191
:1011700008094FF00008B845BCDA444BDBF80420FE
:101180001B7859F8045BC2F30072062B6FD8DFE8B6
:1011900003F06429310B3B3B3B00032286F8AB2A6A
:1011A0000093454A3B46A1E70392FFF769FFDFED55
:1011B000430A039A0146B0EE600A2846FFF7ECFEA8
:1011C000206054F8081B002954D105233C4A86F8B6
:1011D000AB3A0420434605B0BDEC028BBDE8F04FAE
:1011E000FCF7E8BB0392FFF74BFFDFED360A039AEB
:1011F0000146E0E70392FFF743FFDFED330A039A6E
:101200009FED320A0146D8E7052B24D030493148FA
:10121000062B08BF01464FF0000A019228460A46F5
:10122000CDF800A014230221FFF7D0FD054680B1C0
:1012300000F11403194600680393122243F080FD65
:10124000039B30B11846482251464DF097FF0123C9
:101250002B712560B5E72049DDE70392FFF710FF0A
:101260009FED140A039A0146F0EE480AA5E7002311
:101270002360A6E708F101087DE700BFF027012001
:101280002072002048B10608D03E0020443D0020D6
:1012900039F100083813060874B10608F9F300089C
:1012A000503D002040420F00583D002063F10008EF
:1012B000903D00206F12833A92B1060800000000B2
:1012C000CBB106086F120339ACC5A737ACC5A7363A
:1012D000C0C62D00001BB700808D5B00F4270120E5
:1012E000034AD2F8B82A12B10F2800D81047704725
:1012F0002072002050B10138002330F0FF019AB273
:1013000003F1010303D140EA022080B27047400894
:10131000F3E703681B68184703685B6818470368AE
:101320009B6818470368DB6970B506460C4615468E
:1013300083B1BDE8704018473046FFF7F0FF002842
:10134000FAD014F8011B3046FFF7E3FF2B1B002BEC
:10135000F2DC70BD0D44F9E7E4E70368DB68184789
:1013600003681B69184703685B69184703689B6A31
:1013700003B1184770470368DB6A03B11847704729
:10138000164B1B6813F0100F154B05D0B3F8C02A8D
:1013900012F0040F18BF002093F8DA2A72B1D3F8C4
:1013A000DC2ACAB1926838B1B3F8E01A0D4BB3FB2E
:1013B000F1F35B101360704710607047D3F8E42AB4
:1013C00093F8E83A0BB980F001002AB113689288CB
:1013D00008B11A8370475A83704700BF582701200D
:1013E0002072002040420F00BFF34F8F0549064B8B
:1013F000CA6802F4E0621343CB60BFF34F8F00BFB3
:10140000FDE700BF00ED00E00400FA0508B572B684
:1014100000224FF0FF31930003F1604303F5614375
:101420000132082AC3F88010C3F88011F3D1FFF706
:10143000DBFF012108B50846F9F76CFDFFF7E6FF71
:1014400008B50120F9F776FD012809D10021F9F747
:1014500061FD044B1A6882F308885B689847FEE7D1
:1014600008BD00BF0000FF1FEFF31183102282F3BD
:10147000128809490A6801320A604FF0E0220749E0
:101480009069C1F8EC0A0020C1F8F00A1269DBB2D9
:1014900083F31188704700BFC42A00202072002007
:1014A000064A074B51681B6858434FF47A73B0FBE8
:1014B000F3F053685B1A8342FBD97047001000E0D9
:1014C000F42B002010B504464FF4FA70FFF7E8FF44
:1014D0006069BDE81040FEF79BBC90F9103073B511
:1014E0001546142253430D4AD65883689A0704467A
:1014F00004D44069019145F039FF0199304647F025
:101500005DF82946304647F059F8A3689B0702D496
:101510002046FFF7D7FF012002B070BDB0000020C9
:101520007FB50379012B0D460AD0022B19D18368B0
:10153000DB0758BF01F07F0104B0BDE87040CCE785
:1015400081688DF80F2001F001010DF10F0200926A
:101550000191417C90F910002A46F9F77FFB04B015
:1015600070BD0020FBE700682E22F421D8E7044B71
:1015700000681A8E9201343202F0FC02F421CFE7A7
:101580002861002008B53122F4210068FFF7C8FF68
:10159000012008BD006801225821C1E7006801222E
:1015A0004821BDE7006802220821B9E7006801224E
:1015B0000821B5E710B50446002221210068FFF795
:1015C000AFFF2068FC222021FFF7AAFF20684022FD
:1015D0002421FFF7A5FF20680C222321FFF7A0FF9D
:1015E000206800222221FFF79BFF012010BD10B5CB
:1015F000012204460B210068FFF792FF20B120680A
:101600001D220921FFF78CFF00F0010010BD044BE3
:101610000246D3F8F40A08B1802181E7704700BF81
:101620002072002010B5B020FFF7F1FF4020FFF737
:10163000EEFF0020FFF7EBFF1020FFF7E8FF4FF46D
:101640008064013C0020A4B245F0E5FB002CF8D1F9
:1016500010BD503910B50446C8B2FFF7D8FF04EBEF
:101660004400400004EB440400F00E00FFF7CFFFFD
:10167000C4F3C3001030BDE81040C8E708B55038C7
:10168000C0B2FFF7C4FF0020FFF7C1FFBDE808406C
:101690001020BCE738B500221F2333210120FEF7BC
:1016A000D9FD3D4BC3F8F40A10B90024204638BDDB
:1016B000AE20FFF7ACFF04460028F6D0D420FFF799
:1016C000A6FF8020FFF7A3FFA820FFF7A0FF3F2081
:1016D000FFF79DFFD320FFF79AFF0020FFF797FF4A
:1016E0004020FFF794FF8D20FFF791FF1420FFF7B4
:1016F0008EFFA120FFF78BFFC820FFF788FFDA20BD
:10170000FFF785FF1220FFF782FF8120FFF77FFFA1
:10171000CF20FFF77CFFD920FFF779FFF120FFF7FB
:1017200076FFDB20FFF773FF4020FFF770FFA42058
:10173000FFF76DFFA620FFF76AFFAF20FFF767FFF7
:10174000A620FFF764FFAE20FFF761FF2020FFF720
:101750005EFF0020FFF75BFFB020FFF758FF40203F
:10176000FFF755FF0020FFF752FF1020FFF74FFF54
:101770004FF48065013D0020ADB245F04CFB002DDB
:10178000F8D18120FFF743FFC820FFF740FFAF20CB
:10179000FFF73DFF8AE700BF2072002008B5FFF782
:1017A000BFFE014B187008BD38100020F7B51E466B
:1017B00090F910301546142253430E4AD7588368C7
:1017C0009A07044604D44069019145F0CFFD019980
:1017D000384646F0F3FE33462A460021384646F0A6
:1017E00085FEA3689B0702D42046FFF76BFE01200D
:1017F00003B0F0BDB0000020F7B50779012F164601
:101800000AD0022F15D18468E40758BF41F0800147
:1018100003B0BDE8F040C9E7826802F00102CDE9FB
:1018200000620A46417C90F91000F9F717FA03B0FC
:10183000F0BD0020FBE707B5130A8DF804308DF8E2
:101840000520022301AAFFF7D7FF024B187003B04F
:101850005DF804FB3810002010B50A4C002384F812
:10186000F83A84F8F91A84F8FA2A032304F6F822DD
:10187000FF21FFF7C1FF00280CBF6FF00C00002014
:1018800010BD00BF2072002010B50B4C002384F85F
:10189000F83A130A84F8F91A84F8FA3A84F8FB2A19
:1018A000042304F6F822FF21FFF7A6FF00280CBF4F
:1018B0006FF00C00002010BD20720020024A00686A
:1018C0000023512198E700BF187E0020F7B51E467F
:1018D00090F910301546142253430E4AD7588368A6
:1018E0009A07044604D44069019145F03FFD0199EF
:1018F000384646F063FE334600222946384646F015
:10190000F5FDA3689B0702D42046FFF7DBFD01200D
:1019100003B0F0BDB0000020F7B50779012F1646DF
:101920000AD0022F15D18468E40758BF41F0800126
:1019300003B0BDE8F040C9E7826802F00102CDE9DA
:1019400000620A46417C90F91000F9F7ADF903B046
:10195000F0BD0020FBE713B5062304466A46006885
:101960000221FFF7D9FFB8B1BDF9003007EE903A78
:10197000BDF90230F8EEE77AC4ED077A07EE903A47
:10198000BDF90430F8EEE77AC4ED087A07EE903A34
:10199000F8EEE77AC4ED097A02B010BD13B5022360
:1019A00004466A4600680321FFF7B6FF10B900201D
:1019B00002B010BD9DF90130002BF8DA2068072332
:1019C0006A461221FFF7A8FF0028F0D09DF90220F7
:1019D0009DF8013043EA022313EB430348BF03336E
:1019E0009B1007EE903A9DF904209DF8033043EADE
:1019F000022313EB4303F8EEE77A48BF03339B104F
:101A00009DF90620C4ED047A07EE903A9DF8053062
:101A100043EA022313EB4303F8EEE77A48BF0333AC
:101A20009B10C4ED057A07EE903AF8EEE77AC4ED24
:101A3000067ABDE738B504460068FDF77FFF0C2342
:101A40000546021D19462068FFF766FFA870B8B169
:101A5000B5F9043007EE903AF8EEE77AC4ED077A6C
:101A6000B5F9063007EE903AF8EEE77AC4ED087A59
:101A7000B5F9083007EE903AF8EEE77AC4ED097A46
:101A800038BD38B504460068FDF758FF0D230546FC
:101A9000C21C0C212068FFF73FFFA870B8B1B5F950
:101AA0000A3007EE903AF8EEE77AC4ED077AB5F916
:101AB0000C3007EE903AF8EEE77AC4ED087AB5F903
:101AC0000E3007EE903AF8EEE77AC4ED097A38BDA9
:101AD00013B503230C46006801AA2221FFF71CFF5F
:101AE00030B1BDF9053003EB83031B12E6332380CD
:101AF00002B010BD13B5062304466A4600681F21D4
:101B0000FFF70AFFD0B1BDF80030DBBA07EE903A1C
:101B1000BDF80230F8EEE77ADBBAC4ED047A07EEDE
:101B2000903ABDF80430F8EEE77ADBBAC4ED057AF6
:101B300007EE903AF8EEE77AC4ED067A02B010BDEF
:101B400013B5062304466A4600682521FFF7E4FE24
:101B5000D0B1BDF80030DBBA07EE903ABDF80230E4
:101B6000F8EEE77ADBBAC4ED077A07EE903ABDF8F3
:101B70000430F8EEE77ADBBAC4ED087A07EE903A63
:101B8000F8EEE77AC4ED097A02B010BD70B50668C8
:101B900005463046FDF7D2FE0E230446021D3B21CA
:101BA0003046FFF7B9FEA070B8B1A389DBBA07EEE3
:101BB000903AF8EEE77AC5ED077AE389DBBA07EEEB
:101BC000903AF8EEE77AC5ED087A238ADBBA07EE99
:101BD000903AF8EEE77AC5ED097A70BD07B50223B1
:101BE000006801AAF621FFF797FE20B1BDF8043086
:101BF000024A5BBA138203B05DF804FB286100203F
:101C000007B50323006801AAF621FFF785FE80B11E
:101C10009DF805309DF8042007491B0243EA024362
:101C20009DF806201343B1F93020C2F10802D340D9
:101C30004B6303B05DF804FB2861002037B5062331
:101C4000F7210068154C6A46FFF766FE1449E8B1B3
:101C50009DF801209DF800309DF80350120142EAE2
:101C600003329DF8023042EA13129DF804308A656F
:101C70001B0143EA05339DF80550C4F8F82B43EAED
:101C800015138B63C4F8FC3B03B030BDD4F8F83BAC
:101C90008B65D4F8FC3B8B63F6E700BF2072002015
:101CA0002861002007B50323006801AA1946FFF741
:101CB00033FEA0B19DF804309DF805109DF9042075
:101CC0001B0443EA01239DF80610002AB4BF4FF01D
:101CD0007F4200220B431343024AC2F8183103B07B
:101CE0005DF804FB2861002007B50323006801AA02
:101CF0000021FFF711FEA0B19DF804309DF80510FA
:101D00009DF904201B0443EA01239DF80610002AD4
:101D1000B4BF4FF07F4200220B431343024AC2F884
:101D2000FC3003B05DF804FB2861002013B50446C5
:101D300000680379022B0CBF4321032106236A4666
:101D4000FFF7EAFD18B9E086A06302B010BDBDF848
:101D500000305BBAE386BDF802305BBA6387BDF83A
:101D600004305BBA2387F0E713B50023C38683638F
:101D70000446062300686A460321FFF7CDFD78B1CB
:101D8000BDF8003003EB4303E386BDF902305B424C
:101D900003EB43032387BDF8043003EB430363875E
:101DA00002B010BD07B5012301AAFF210068FFF7AB
:101DB000B3FD03B05DF804FBF7B505460068FDF719
:101DC000BDFD00230370042304460DEB03022868C5
:101DD000FF21FFF7A1FD10B9002003B0F0BD286876
:101DE00004236A46FF21FFF797FD0028F4D09DF8F1
:101DF00004108A09023A012AEED99DF8053003EB56
:101E0000012343F6FF75C3F30D03AB42E4D0002B6F
:101E1000E2D09DF806109DF8072040F2FF7702EB14
:101E20000122B7EB521F4FEA6211D5D00029D3D05F
:101E30009DF800609DF8012002EB0622C2F30D021E
:101E4000AA42C9D0002AC7D09DF802609DF803506D
:101E500005EB0625B7EB551F4FEA6516BCD0002EE3
:101E6000BAD09D1A002DB8BF6D42FF2DB4DC8D1B7A
:101E7000002DB8BF6D42FF2DAEDC01251344314467
:101E80002B4129412570C4F80530C4F80110A4E79E
:101E900073B505460068FDF751FD0026042304468E
:101EA00006700DEB03022868FF21FFF735FD48B1EE
:101EB0009DF804108B0907D003200D4A0421FBF77D
:101EC00079FD304602B070BD9DF805209DF80730C1
:101ED00002EB01229DF8061003EB012392B25B1185
:101EE00001212170C4F80520C4F80130EAE700BFE1
:101EF000F0B1060807B5022301AAFFF70DFD044B58
:101F00001870BDF8040040BA80B203B05DF804FB5D
:101F10003810002038B515460D4A0B0A82F8F83AF9
:101F200082F8F91A022302F6F822FF210446FFF78D
:101F300063FC10B96FF00C0038BD01232A46FF2165
:101F40002046FFF7E9FC0028F4D00020F4E700BFAA
:101F500020720020F8B5124D164685F8F91A05F6DC
:101F6000F82200240223FF21074685F8F84AFFF7EC
:101F700043FC05F6F82210B96FF00C00F8BD0223FF
:101F8000FF213846FFF7C8FC0028F5D095F8F82A5D
:101F900095F8F93A03EB022333802046EEE700BFC1
:101FA000207200202DE9F341754D0468DFF8DC81D3
:101FB0000023064685F8F2302D27B9B218F8012B18
:101FC00020460137FFF748FC882FF6D140228721B1
:101FD0002046FFF741FC00238DF806300DF1060185
:101FE000204644F07CFE9DF80630002BF6D00122FE
:101FF00086212046FFF730FC002287212046FFF78C
:102000002BFC092208212046FFF726FC00220B2189
:102010002046FFF721FC002853D137680DF1060256
:102020005E213846FFF796FFBDF80630B3F5D77F3F
:1020300000F0A18055D8512B00F09B8049D81D2B72
:102040006CD01E2B00F095803068212144F0B6FD45
:1020500034680DF10602DE212046FFF77BFFBDF854
:1020600006309FED487AC3F309032822ADF8063005
:10207000534307EE903AF8EEE77A434A67EE877AE1
:102080000021FCEEE77A82F8F81A17EE903A6C21FC
:1020900082F8F91A190E82F8FA1A190C82F8FB1A4A
:1020A000190A82F8FC1A82F8FD3AFF2102F6F8229A
:1020B00006232046FFF7A0FB306840228721FFF768
:1020C000CBFBB0FA80F0400985F8F20002B0BDE821
:1020D000F081AD2B4FD0D62B01D0602BB4D1212471
:1020E0001DE040F2E132934247D00CD840F2D922B1
:1020F000934242D040F2E122934202D0B3F5E67F10
:10210000A2D164240BE040F28F42934203D040F20C
:102110009152934298D14FF4FA7400E00F240028B2
:1021200092D10A224B213846FFF796FB0F226021FD
:102130003846FFF791FB0D2263213846FFF78CFBF1
:10214000B82269213846FFF787FB40F60D727821E7
:102150003846FFF799FB40F60E627A213846FFF7C2
:1021600093FB00287FF470AF2146384644F026FDEB
:102170006AE71424D3E73224D1E7C824CFE700BFAD
:10218000286100209A99893F207200200C170608C8
:1021900037B5124D95F8F2300446E3B100680DF101
:1021A000050144F09CFD9DF805307BB10DF1060260
:1021B00020689621FFF7CEFE0A22BDF80630B3FB59
:1021C000F2F3074A9360012385F8F3302068012277
:1021D0008621FFF741FB03B030BD00BF286100201E
:1021E0003810002013B5022301AA044651210068CB
:1021F000FFF792FB114AF0B1BDF804305BBA9BB215
:10220000D360D368B3F5C87F02DD4FF0FF33D360EE
:102210000B4B0C4A1968D2F8003C32338B4208D27F
:10222000C2F8001C2068002302F6F8325121FFF7A3
:10223000E3FA02B010BD6FF00103E8E738100020A8
:10224000C42A00202072002007B50223006801AADA
:102250000021FFF761FB0F4B83F8F800B0B1BDF828
:1022600004300D4A5BBA9BB2B3F5FA6F3FBF0A2147
:10227000B3FBF1F307EE903AF8EEE77A2BBF4FF09D
:10228000FF33FDEEE77A1361C2ED047A03B05DF827
:1022900004FB00BF286100203810002013B5022382
:1022A0000C46006801AA0021FFF736FB60B15CB163
:1022B0009DF805309DF90420DB0903EB830302EB55
:1022C000820203EB4203238002B010BD90F910306C
:1022D00073B51546142253430E4AD65883689A079D
:1022E000044604D44069019145F040F80199304614
:1022F00046F064F9012300222946304646F0F6F8FC
:10230000A3689B0702D42046FFF7DCF8012002B047
:1023100070BD00BFB000002073B50379012B1646D5
:102320000AD0022B15D18368DB0758BF41F080012A
:1023300002B0BDE87040C9E7826802F00102CDE951
:1023400000620A46417C90F91000F8F7ADFC02B03B
:1023500070BD0020FBE7F7B515460DF107021C46DE
:1023600006460F46FFF7D8FF9DF8073005EA03023F
:10237000A24209D023EA050222433946304603B07F
:10238000BDE8F040FFF7CCB803B0F0BD13B504468C
:102390006A4600680821FFF7BFFF9DF8003013F080
:1023A00010037ED0206806236A460021FFF7B4FAA6
:1023B000002874D09DF801309DF800209FED3A6A06
:1023C0009DF804101B0203EB02439DF802201C023F
:1023D0001A4448BF02F17F4207EE902AF8EEE77AEE
:1023E0009DF80330C7EE866A090201EB03419DF8B0
:1023F00005300B44090248BF03F17F4307EE903AD2
:102400002A4BB3F97020B8EEE77A07EE902AB3F9B9
:102410006C20C7EE065A06EE102AF8EEE77AB8EE00
:10242000C66AB3F96820A6EEA76AD3ED197AB8EEAA
:10243000E77AD3ED187AA6EE867AF8EEE77A26EEFA
:10244000A55AE6EE877A07EE102AB3F96E20B8EEA9
:10245000C77A06EE102AB3F96A20E5EE877A07EE0E
:10246000102AB8EEC66AB8EEC77AB3F95C20A6EEB9
:10247000867AF6EE006AE5EE077A07EE102AB3F9DF
:102480005E20C3ED1D7A07EE902AF8EEE77AB8EEEB
:10249000C77A67EEA57AE7EE267AC3ED1E7A02B018
:1024A00010BD1846FBE700BF0000784828610020F7
:1024B0001FB50446002300688DF807300DF10702B0
:1024C0002721FFF729FF68B19DF8073013F00803B3
:1024D00020D02068062302AA2821FFF71DFA18B988
:1024E000E086A06304B010BDBDF90830002BB8BF72
:1024F00003339B10E386BDF90A30002BB8BF0333CA
:102500009B102387BDF90C30002BB8BF03339B1001
:102510006387E7E71846E5E71FB500210446C18653
:1025200081630DF107020068FFF7F6FEC0B19DF868
:10253000073013F0080315D02068062302AA0121F2
:10254000FFF7EAF960B1BDF808305BBAE386BDF881
:102550000A305BBA2387BDF80C305BBA5B426387F5
:1025600004B010BD1846FBE730B5002585B0044621
:10257000C58685630DF1070200680621FFF7CCFED2
:10258000A0B19DF8073013F0040311D02068062392
:1025900002AA2946FFF7C0F940B1BDF80830E3862A
:1025A000BDF80A302387BDF80C30638705B030BD15
:1025B0001846FBE707B50DF10702FFF7ADFE034B29
:1025C00018709DF8070003B05DF804FB3810002078
:1025D000F8B5144E144F41F0010200210446FFF7F4
:1025E000DDF83568C7F8045C13212046FFF7E2FFE9
:1025F00010F007000BD001220B212046FFF7CEF888
:10260000002220461146FFF7C9F8012008E0D7F85C
:10261000082C002AE8D033689BB25B1B9A42E3D2B5
:10262000F8BD00BFC42A00202072002010B50C465F
:102630000121FFF7BFFFC0F300132370C0F3C003F5
:10264000A370C0F380036370C0F38013C0F3C010A5
:10265000E370207110BD2DE9F047884650211446E3
:102660000646FFF7A7FF01304000C0B22080462198
:102670003046FFF79FFF2D4F2378013080B27B4318
:102680004FF47A79A08003F5FA734FF4FA6AB3FB3A
:10269000F9F25121B3FBFAF300FB02333046B3FBEE
:1026A000F9F3E360FFF726FCC3B2C0F30F222578ED
:1026B00003FA02F2013293B27D43E38005F5FA7228
:1026C0003046B2FBF9F1B2FBFAF203FB01227021B2
:1026D000B2FBF9F22282FFF76DFF01304000C0B279
:1026E000608071213046FFF705FCC3B2C0F30F20B4
:1026F0008340013398F803209BB2238112B1E28812
:102700009B1A2381A37820897B4303F5FA734FF446
:102710007A724FF4FA65B3FBF2F1B3FBF5F300FB09
:102720000133B3FBF2F36382BDE8F087002F3A0078
:102730002DE9F047DB4FDFF87483DFF874934FF433
:10274000FA738CB00446002689210068C7F8083C5B
:1027500088F8F060FFF72EFF40F00100C2B2892137
:102760002068FFF71BF8324620688821FFF716F82B
:10277000206801228021FFF711F820680122FF2143
:10278000FFF70CF8324631462068FFF707F8912131
:102790002068FFF70FFF314687F80C0C01222068F4
:1027A000FEF7FCFF32462068FF21FEF7F7FF3246B6
:1027B00020688021FEF7F2FF60212068FFF7FAFE13
:1027C00040F01200C2B260212068FEF7E7FF2068E7
:1027D00020224421FFF72FF82068FF220121FEF775
:1027E000DDFF2568012280212846FEF7D7FF012260
:1027F000FF212846FEF7D2FF324631462846FEF733
:10280000CDFF0622FF212846FEF7C8FF8321284678
:10281000FFF7D0FE40F00400C2B283212846FEF745
:10282000BDFF0722FF212846FEF7B8FF01228121C4
:102830002846FEF7B3FF012280212846FEF7AEFFAF
:102840006B2294212846FEF7A9FF324683212846B1
:10285000FEF7A4FFD9F80060C7F8046C832128466E
:10286000FFF7A8FE002800F05283012228468321AA
:10287000FEF794FF92212846FFF79CFE0022C0F34A
:10288000C716814681212846FEF788FF0622284682
:10289000FF21FEF783FF83212846FFF78BFE83216C
:1028A00000F0FB022846FEF779FF28460122FF21AF
:1028B000FEF774FF284601220021FEF76FFF28462D
:1028C0000022FF21FEF76AFF284600228021FEF742
:1028D00065FF062305AAB0212068FFF71DF82068D0
:1028E0000122FF21FEF75AFF206800224F21FEF748
:1028F00055FF20682C224E21FEF750FF2068002251
:10290000FF21FEF74BFFB4222068B621FEF746FFF9
:102910000025002E18BF0C2609F07F092A464FF02B
:10292000010CC5F3C40000F130035FFA85FE0DEB26
:102930000300764510F81C3C05F0070102D89145CC
:1029400040F0F0820CFA01F123EA010300F81C3C8C
:102950000135302DE5D1062305AAB0212068FEF708
:102960004BFF514B01221870FF212068FEF716FF24
:10297000002211462068FEF711FF20680022FF2187
:10298000FEF70CFF206800220921FEF707FF2068F0
:1029900000221021FEF702FF206800221121FEF71D
:1029A000FDFE206801222421FEF7F8FE2068FF22A8
:1029B0002521FEF7F3FE206800227521FEF7EEFECA
:1029C00020680122FF21FEF7E9FE20682C224E211B
:1029D000FEF7E4FE206800224821FEF7DFFE2946CC
:1029E00020682022FEF7DAFE20680022FF21FEF791
:1029F000D5FE294620680922FEF7D0FE2068002275
:102A00005421FEF7CBFE206804223121FEF7C6FEDA
:102A1000206803223221FEF7C1FE20688322402174
:102A2000FEF7BCFE206825224621FEF7B7FE20688F
:102A300000226021FEF7B2FE206800222721FEF767
:102A4000ADFE206806225021FEF7A8FE2068002275
:102A50005121FEF7A3FE206896225221FEF79EFE2A
:102A6000206808225621FEF799FE2A462068572141
:102A7000FEF794FE206800226121FEF78FFE206899
:102A800000226221FEF78AFE206800226421FEF700
:102A900085FE206800226521FEF780FE2068A022C6
:102AA000662107E0207200203810002028610020F5
:102AB000C42A0020FEF772FE20680122FF21FEF7E3
:102AC0006DFE206832222221FEF768FE2068142263
:102AD0004721FEF763FE2068FF224921FEF75EFED4
:102AE000206800224A21FEF759FE20680022FF21BB
:102AF000FEF754FE20680A227A21FEF74FFE206876
:102B000000227B21FEF74AFE206821227821FEF771
:102B100045FE20680122FF21FEF740FE2068342296
:102B20002321FEF73BFE206800224221FEF736FEFD
:102B30002068FF224421FEF731FE2068262245212D
:102B4000FEF72CFE206805224621FEF727FE4022D4
:102B500011462068FEF722FE206806220E21FEF7AD
:102B60001DFE20681A222021FEF718FE2068402250
:102B70004321FEF713FE20680022FF21FEF70EFE20
:102B8000206803223421FEF709FE20684422352103
:102B9000FEF704FE20680122FF21FEF7FFFD2068FA
:102BA00004223121FEF7FAFD206809224B21FEF7AD
:102BB000F5FD206805224C21FEF7F0FD2068042277
:102BC0004D21FEF7EBFD20680022FF21FEF7E6FD18
:102BD000206800224421FEF7E1FD206820224521E3
:102BE000FEF7DCFD206808224721FEF7D7FD2068AC
:102BF00028224821FEF7D2FD206800226721FEF737
:102C0000CDFD206804227021FEF7C8FD2068012256
:102C10007121FEF7C3FD2068FE227221FEF7BEFD82
:102C2000206800227621FEF7B9FD20680022772176
:102C3000FEF7B4FD20680122FF21FEF7AFFD2068FA
:102C400001220D21FEF7AAFD20680022FF21FEF7D8
:102C5000A5FD206801228021FEF7A0FD2068F82252
:102C60000121FEF79BFD20680122FF21FEF796FD62
:102C7000206801228E21FEF791FD206801220021AB
:102C8000FEF78CFD20680022FF21FEF787FD2068FB
:102C900000228021FEF782FD042220680A21FEF72F
:102CA0007DFD256884212846FFF784FC842100F0FF
:102CB000EF022846FEF772FD012220680B21FEF785
:102CC0006DFD2068019003A9FFF7B0FC019807AAE9
:102CD00003A9FFF7C0FC9DF80C30002B00F0288101
:102CE0000A9D05F684559DF80E30002B00F02381D7
:102CF0000A9B03F2B22305EB43059DF80F3023B185
:102D0000BDF82C3003F525731D449DF8103023B118
:102D1000BDF82E3003F226231D442068C7F8105C4E
:102D2000E8220121FEF73AFD44F61F639D4203D9D4
:102D30002068294643F0F3FF012220681146FEF780
:102D40002DFD20684021FFF743FC002800F0E780BC
:102D5000206801210222FEF721FD20680021FFF7F3
:102D600037FC002800F0DB802068DFF8E491E822DF
:102D70000121FEF713FD202220684421FEF75BFDB0
:102D8000256803A92846FFF751FC07AA03A928468E
:102D9000FFF761FC502257212846FEF7FFFC08226E
:102DA00056212846FEF7FAFC082250212846FEF755
:102DB000F5FCBDF82C004FF47A7A48F20E660AFB57
:102DC0000060B0FBF9F080B2FEF794FA51210246A0
:102DD0002846FEF730FD0A9A5C4B0AFB02669E42CB
:102DE0009DBFB6FBF9F202F1FF32D2B2FF224621BB
:102DF0002846FEF7D3FCD7F8101C44F61F6399420F
:102E000002D9284643F08BFF01212846FFF7D2FB69
:102E10000222064601212846FEF7C0FC0021284672
:102E2000FFF7D6FB324601212846FEF7B7FC24689F
:102E300003A92046FFF7FAFB07AA03A92046FFF7DC
:102E40000AFC482211462046FEF7A8FC082247212A
:102E50002046FEF7A3FC032232212046FEF79EFC0B
:102E6000072230212046FEF799FC0122FF2120464F
:102E7000FEF794FC202230212046FEF78FFC002232
:102E8000FF212046FEF78AFC062220467021FEF72D
:102E900085FCBDF82E304FF47A7246F6440002FBF2
:102EA00003004DF28803B0FBF3F09DF80F3080B2C1
:102EB0001BB1BDF82230184480B2FEF71BFA712115
:102EC00002462046FEF7B7FCD7F8101C44F61F63F5
:102ED000994202D9204643F022FF01212046FFF704
:102EE00069FB0222054601212046FEF757FC00211E
:102EF0002046FFF76DFB2A4601212046FEF74EFCD7
:102F00006423C7F8083C012388F8F03007E0D9F8BB
:102F100000309BB29B1BB3F5FA7F7FF69FAC0CB0E1
:102F2000BDE8F0870B41DB0744BF0132D2B20FE5A9
:102F300040F63635D7E69DF80D30002B3FF4DDAE78
:102F40000A9B03F525731D44D7E600BF1B280D011E
:102F50001C0C0100F8B53B4F97F8F0300446002BED
:102F600037D0394D95F8146C012E33D0022E4FD046
:102F70007EBB006801228021FEF710FC2068012240
:102F8000FF21FEF70BFC206832463146FEF706FCB7
:102F900095F80C2C20689121FEF700FC2068012296
:102FA0003146FEF7FBFB20683246FF21FEF7F6FBB9
:102FB000206832468021FEF7F1FB2068012231466D
:102FC000FEF7ECFB214B1B68C5F8043C012385F898
:102FD000143CF8BD00680021FFF7ECFAC20711D5D8
:102FE000D5F8082C002AF4D0184BD5F8041C1B681F
:102FF0009BB25B1A9A42ECD2154B4FF0FF325A60EB
:103000000023E4E7114B1B68C5F8043C0223DEE70C
:1030100000681321FFF7CEFA4307E1D01E21206894
:10302000FEF768FF012206460B212068FEF7B6FB7B
:10303000074B0A20B6FBF0F6B6B25E60012387F8B4
:10304000F130DDE72861002020720020C42A002032
:103050003810002010B5EFF31182102383F312888B
:103060004FF0E023D2B29C69196911F4803F0D49F9
:103070001EBF0120C1F8F00A9C690B4B1868D1F8FB
:10308000F03A82F31188094A11684FF47A720344C6
:1030900002FB01F0001BB0FBF1F00021E3FB020199
:1030A00010BD00BF20720020C42A0020F42B002095
:1030B000124B5B68C3F3080330B4EBB9EFF3118331
:1030C000D3B90F4B0F484FF0E0251968AC691A6867
:1030D0008A42FAD1D0F8EC1AA142F6D30A4B196809
:1030E0004FF47A7303FB01F0001BB0FBF1F00021F9
:1030F000E2FB030130BC704730BCABE700ED00E001
:10310000C42A002020720020F42B002010B5074CA8
:1031100094F8190C40B1FFF7CBFFD4F8203CC01A4B
:10312000C0F5FA5020EAE07010BD00BF2072002008
:10313000F8B506460D46FFF7BBFF04460F46FFF7FE
:10314000B7FF031B61EB0702B34272EB0503F6D333
:10315000F8BD38B50D460446FFF7D8FF011E02DD65
:10316000C917FFF7E5FF064B2068002283F8192CEA
:10317000492193F81A3C2A46FEF7CEFB012038BDC0
:10318000207200202DE9F341364CD4F8283CC0F8D9
:103190003630B4F82C3C438794F8183C012B054694
:1031A00000F1360704F628460AD0022B23D08BBB49
:1031B0000122022142F0A1FA012384F8183C02E026
:1031C000FFF7A4FF28B194F82E2C104602B0BDE8FA
:1031D000F08169462846FFF7BCFF18B19DF8003022
:1031E0009B0701D10023E8E707220321284642F08C
:1031F00084FA0223E1E7FFF789FF0028E3D169465B
:103200002846FFF7A6FF9DF80630024610B113F0DE
:10321000080805D0002284F8182C84F82E2CD4E756
:10322000B4F9301C6846FBF79DFE4042B4F9321CED
:10323000E8860DF10200FBF795FEB4F9341C2887EF
:1032400001A8FBF78FFED5F83630C4F8283C404281
:103250006887BB88B380012384F8188C84F82E3CDF
:10326000B3E700BF2072002010B50446013C00D235
:1032700010BD4FF47A700021FFF75AFFF6E710B542
:10328000044600210068FCF70FFBB62214212068D9
:10329000FEF746F96420FFF7E7FF8122102120683E
:1032A000FEF73EF90120FFF7DFFF1521206880229D
:1032B000FEF736F90120FFF7D7FF20680321BDE8AC
:1032C0001040FCF7F1BA10B5044600210068FCF785
:1032D000EBFAB6227E212068FEF722F96420FFF780
:1032E000C3FF00227C212068FEF71AF96420FFF753
:1032F000BBFF04227D212068FEF712F96420FFF74E
:10330000B3FF8C2240212068FEF70AF90120FFF765
:10331000ABFF022241212068FEF702F90120FFF7EE
:10332000A3FF20680221FCF7BFFA4FF40063A381DA
:1033300010BD10B504464069FCF76FFD0120FFF792
:1033400093FF6069FCF764FDBDE810400A208BE73D
:1033500073B50468B6227E2105462046FEF7E0F8E4
:103360006420FFF781FF02212046FCF79DFA2046EA
:10337000FFF7DFFF00227C212046FEF7D1F8012075
:10338000FFF772FF002259212046FEF7C9F80120FD
:10339000FFF76AFF5E238DF8073094F9103014228E
:1033A00053433D4AD658A3689A0702D4606943F054
:1033B000DDFF01230DF107020021304645F096F8AC
:1033C0004FF4A473354A0021304645F08FF8A368C6
:1033D0009B0702D42046FEF775F80A20FFF744FF4A
:1033E000012259212046FEF79BF80120FFF73CFF00
:1033F0008C2240212046FEF793F80120FFF734FF8E
:10340000032241212046FEF78BF80120FFF72CFF15
:10341000234EA96B234A95F83500B6FBF1F1092339
:1034200089B2FBF711FF4388B6FBF3F62E640279ED
:10343000422142F0C0022046FEF772F80120FFF759
:1034400013FF082243212046FEF76AF80120FFF708
:103450000BFF042258212046FEF762F80120FFF7F7
:1034600003FF0A2253212046FEF75AF80120FFF7F6
:10347000FBFE00227C212046FEF752F80120FFF7D8
:10348000F3FE06227D212046FEF74AF8012002B015
:10349000BDE87040E8E600BFB000002067170608EE
:1034A00040420F00B0180608F8B5816B0468294A3D
:1034B000294FB7FBF1F10546102389B290F835008A
:1034C000FBF7C2FE00214388B7FBF3F706462F64E3
:1034D0002046FCF7E9F980226B212046FEF720F810
:1034E0006420FFF7C1FE032268212046FEF718F88A
:1034F0006420FFF7B9FE01226B212046FEF710F889
:103500000F20FFF7B1FE18221B212046FEF708F816
:103510000F20FFF7A9FE18221C212046FEF700F815
:103520000F20FFF7A1FE32791A212046FDF7F8FFA0
:103530000F20FFF799FE727919212046FDF7F0FF61
:103540006420FFF791FE20460321BDE8F840FCF718
:10355000ABB900BFE618060840420F00F7B50F23CD
:103560000468816B3F4A404FB7FBF1F1064689B2D0
:1035700090F83500FBF768FE00214388B7FBF3F7AE
:10358000054637642046FCF78FF90F224E2120466E
:10359000FDF7C6FF0F20FFF767FE6A794F2102F0A3
:1035A0000F022046FDF7BCFF0F20FFF75DFE6A7992
:1035B000502102F00F022046FDF7B2FF0F20FFF767
:1035C00053FE6A7942EA0212D2B252212046FDF736
:1035D000A7FF0F20FFF748FE032214212046FDF726
:1035E0009FFF0F20FFF740FE002263212046FDF7DA
:1035F00097FF6420FFF738FE082265212046FDF77B
:103600008FFF0DF1070264212046FEF785FE9DF82D
:10361000072022F0100242F06002642120468DF85B
:103620000720FDF77DFF0F20FFF71EFE0DF10602BC
:103630004D212046FEF770FE9DF8062002F03F0265
:1036400042F040024D2120468DF80620FDF768FF2C
:103650000F20FFF709FE03212046FCF725F903B0F0
:10366000F0BD00BF4619060840420F00F8B5816B57
:1036700004682D4A2D4FB7FBF1F10546102389B29E
:1036800090F83500FBF7E0FD00214388B7FBF3F726
:1036900006462F642046FCF707F980226B2120465E
:1036A000FDF73EFF6420FFF7DFFD0722682120467B
:1036B000FDF736FF6420FFF7D7FD00226B2120467F
:1036C000FDF72EFF6420FFF7CFFD01226B2120467E
:1036D000FDF726FF0F20FFF7C7FD18221B2120460C
:1036E000FDF71EFF0F20FFF7BFFD18221C2120460B
:1036F000FDF716FF0F20FFF7B7FD32791A2120469C
:10370000FDF70EFF0F20FFF7AFFD7279192120465C
:10371000FDF706FF6420FFF7A7FD20460321BDE863
:10372000F840FCF7C1B800BFE618060840420F0099
:103730009CE710B57822044600210068FDF7F0FEF2
:103740000520FFF791FD202201212068FDF7E8FE0A
:103750000520FFF789FD002202212068FDF7E0FE29
:103760006420FFF781FD012010BD10B5072204463B
:103770000A210068FDF7D4FE0520FFF775FD24221D
:1037800041212068FDF7CCFE0520FFF76DFDC0222A
:1037900042212068FDF7C4FE0520FFF765FD0120EA
:1037A00010BD10B50122044610210068FDF7B8FED7
:1037B00048B11420FFF758FD2068A022BDE8104052
:1037C0001121FDF7ADBE10BD13B504460021006800
:1037D000FCF76AF80021204641F076FF1420FFF73D
:1037E00043FD0F21204641F06FFF0A20FFF73CFD0B
:1037F00001AA03231021204640F03FFD0A20FFF7D5
:1038000033FD9DF80420174B8032A3F8302C9DF82F
:1038100005208032A3F8322C9DF806208032A3F8D0
:10382000342C0021204641F04FFF0A20FFF71CFDF9
:103830000DF1030201230221204640F01EFD012369
:103840000DF103020921204640F017FD2046122108
:1038500041F03AFF20680321FCF726F8012002B06E
:1038600010BD00BF207200200023F7B51A46362194
:103870000120FCF7EFFC154E0446C6F8380C40B9A1
:1038800096F83C3C0C2B02D10123C6F8403C25465F
:1038900018E005279620FFF7E7FC0DF1070200214D
:1038A0002046FEF739FD054660B9013FF2D196F892
:1038B0003C3C0C2B08BF0223204608BFC6F8403C06
:1038C000FBF7C5FF284603B0F0BD00BF2072002003
:1038D00008B5006801220921FDF722FEBDE8084075
:1038E0006420C1E480B506460B25013D01D1FDF7FA
:1038F000A0FD01210846FCF72FFE00210846FCF739
:103900002BFE771C4FF0320805240120FCF712FE35
:103910000020FCF70FFE0120FDF732FD4046FFF7C7
:10392000A3FC0120FCF706FE0020FCF703FE0020AC
:10393000FDF726FD4046FFF797FC7CB1013C05D121
:103940004FF4FA70FFF790FC4FF0FA0854EA0703BF
:10395000DBD14FF47A70FFF787FCC6E7013FF5E74C
:1039600037B5044600210068FBF79EFF15227E2133
:103970002068FDF7D5FD6420FFF776FC11227E213B
:103980002068FDF7CDFD0520FFF76EFC20680DF1E6
:1039900007020321FEF7C0FC9DF8073003F03C034B
:1039A000142B02D00620FFF79DFF0C224021206837
:1039B000244DFDF7B5FD0120FFF756FCA16B224A0F
:1039C00094F83500B5FBF1F1092389B2FBF73CFC13
:1039D0004388B5FBF3F52564027920684221FDF7A1
:1039E0009FFD0120FFF740FC082241212068FDF7E0
:1039F00097FD0120FFF738FC002243212068FDF7E6
:103A00008FFD0120FFF730FC102251212068FDF7C7
:103A100087FD0120FFF728FC0A2253212068FDF7CB
:103A20007FFD0120FFF720FC802256212068FDF752
:103A300077FD0120FFF718FC20680321FBF734FF16
:103A400003B030BD40420F00A0190608F0B5816BED
:103A50000568514A514FB7FBF1F185B00446102378
:103A600089B290F83500FBF7EFFB00214388B7FBE4
:103A7000F3F7064627642846FBF716FF80226B21E2
:103A80002846FDF74DFD9620FFF7EEFB0322682147
:103A90002846FDF745FD9620FFF7E6FB03226B2144
:103AA0002846FDF73DFD0F200021FFF741FB1022C6
:103AB0006A212846FDF734FD0F200021FFF738FB6F
:103AC00000226C212846FDF72BFD0F200021FFF777
:103AD0002FFB727919212846FDF722FD0F200021C6
:103AE000FFF726FB18221B212846FDF719FD0F20A2
:103AF0000021FFF71DFB18221C212846FDF710FDB1
:103B00000F200021FFF714FB32791A212846FDF718
:103B100007FD01200021FFF70BFB03212846FBF7DF
:103B2000C3FE2068062302AA4321FDF7F5FED0B1AB
:103B3000BDF80830DBBA07EE903ABDF80A30F8EE6F
:103B4000E77ADBBAC4ED077A07EE903ABDF80C309D
:103B5000F8EEE77ADBBAC4ED087A07EE903AF8EEB1
:103B6000E77AC4ED097AD4ED087AFDEEE77ACDED77
:103B7000017A9DF9043001330CD1D4ED077AFDEEC2
:103B8000E77ACDED017A9DF90430013302D10620A8
:103B9000FFF7A8FE05B0F0BDE618060840420F008A
:103BA00018B103685B6803B11847FF20704718B16C
:103BB00003689B6803B118470020704770B450B188
:103BC00006798E4207D34579954204D30368DB68B2
:103BD0000BB170BC184770BC704710B440B1847909
:103BE0008C4205D303681B6913B15DF8044B184779
:103BF0005DF8044B704718B103685B6903B118475F
:103C0000704718B10368DB6903B11847002070479B
:103C100018B103681B6A03B118470020704730B51C
:103C200060B1041D0A4600F114032068616815465E
:103C300003C508349C422A46F7D1012030BD10B597
:103C40000C4670B92D23002023750A4B2061C4E96E
:103C50000000C4E90200C4E90633302384F82030B0
:103C600010BD0368DB6A002BECD098470028E9D030
:103C7000F6E700BF6DE8060838B5054D441E14F898
:103C8000011F01B938BDD5F8600CFBF7CFFDF6E791
:103C90002072002013B50C4C01900C480091FFF7E6
:103CA000EBFFDDE900320A49D4F8600C44F09FFCD8
:103CB000D4F8600CFBF7AEFD94F8643C13B101231B
:103CC00084F8653C02B010BD2072002013B20608D3
:103CD0004DF8000808B50648FFF7CEFF054BB3F8CE
:103CE000660C18B1BDE80840FFF7BEBA08BD00BFBA
:103CF000850C07082072002010B5074C02460B46C1
:103D0000D4F8600C054944F072FCD4F8600CFBF761
:103D100081FDBDE81040DDE7207200204DF800086D
:103D200008B5FFF7A9FFBDE80840D3E710B5044682
:103D30000648FFF7A1FF2046FFF79EFF044B93F8CC
:103D4000642C12B1012283F8652C10BD13B2060851
:103D50002072002010B504460348FFF78DFF20466F
:103D6000BDE81040DCE700BF1FB206080CB48306B4
:103D700007B500D551B9049805A90191FFF7BCFF1B
:103D8000012003B05DF804EB02B070470020F8E7B3
:103D9000024B0146D3F8600CFBF748BD20720020AF
:103DA0000CB407B510F0400009D069B92320FFF723
:103DB000EFFF049805A90191FFF79EFF012003B0D2
:103DC0005DF804EB02B070470020F8E70FB413B5BC
:103DD000094C0A49D4F8600C04AB53F8042B019346
:103DE00044F005FCD4F8600CFBF714FD02B0BDE80C
:103DF000104004B0704700BF207200204DF800084A
:103E00000FB407B504A951F8040B0191FFF774FF33
:103E100003B05DF804EB04B070470FB407B504A914
:103E200051F8040B0191FFF735FFFFF753FF03B083
:103E30005DF804EB04B0704770B58379164603F063
:103E400007028EB00446062A50D8DFE802F00414B8
:103E500017191C1E4A000D7813F0C00348D0402BE0
:103E60003DD12946204615F0B7FB00285BD00EB0A7
:103E7000BDE87040AAE791F90050EDE70D88EBE747
:103E8000B1F90050E8E70D68E6E791ED000A03A8F4
:103E9000FAF7B0FA01462948FFF798FFFEB1A37977
:103EA00013F0C00F1BD1204615F0E1FA00EE100A06
:103EB00003A8B8EEC00AFAF79DFA01462048FFF7BA
:103EC00085FF204615F0E4FA00EE100A03A8B8EECC
:103ED000400AFAF78FFA01461948FFF777FF0EB04C
:103EE00070BD16480EB0BDE870406FE70025B3E71F
:103EF000042A0CBF134814482946FFF767FF002E19
:103F0000EDD0A37913F0C00FE9D1204615F0AFFA38
:103F10000190204615F0BCFA019902460B480EB0FC
:103F2000BDE8704052E703A9204615F0B7F90848EC
:103F300003AA2946FFF771FFD1E700BFA1B7060822
:103F4000CEB9060875B20608C4E70608B10D070821
:103F500024B206082DE9F04F8FB001F020034D4C3C
:103F6000009381460F464FF000084B4BD3F8600C8E
:103F7000FBF750FC94F806B00BF038034B454BD1DF
:103F8000204615F005FAFAF793FC0646204615F090
:103F900021FAD6F808A005460AEB0006204615F0DF
:103FA00059FA0BF00702062A6CD8DFE802F0044049
:103FB00045494E525E001AF805200078111A4A420F
:103FC0004A41009B03B13ABB03A92046019215F078
:103FD00065F97B0615D5019A9AB9304803A9FFF710
:103FE000F5FE2F4903A844F0BBFC00284CD11AF879
:103FF0000530202B48D12B483146FFF7E7FEFFF76D
:1040000069FE294803A9FFF7E1FE00223146204658
:10401000FFF712FFFFF75EFE08F1010840F25A2396
:10402000984504F10B04A0D10FB0BDE8F08F1AF948
:10403000052090F90000C1E73AF805200088BDE7A7
:104040003AF90520B0F90000B8E75AF805200068F1
:10405000B4E796ED007AD0ED007AB4EE677AF1EE2F
:1040600010FA0CBF01220022ABE70190204615F0A8
:104070000FFA0199421C30464BF01AF8B0FA80F260
:1040800052099EE700229CE7002231462046FFF7B6
:10409000D3FEB4E7BE1B06082072002041B206081A
:1040A000830D07084CB2060842B2060813B5044651
:1040B000019115F0CFF9019A0146204602B0BDE802
:1040C0001040B9E6F7B5847914F0C003054603D073
:1040D000402B18D003B0F0BD04F0070415F0D8F958
:1040E000062C05D10146164803B0BDE8F04087E62E
:1040F0000190284615F0BBF9019A0146114803B01A
:10410000BDE8F0407CE615F057FA05460E480F4E24
:104110000F4FFFF7B1FD00242B79A34203D803B062
:10412000BDE8F040D6E514B13046FFF7A5FD2B6899
:10413000384653F82410FFF749FE0134ECE700BF7E
:1041400051B2060861B2060878B2060888B20608BD
:10415000CEB9060808B50548FFF78EFD044BD3F825
:10416000600CBDE80840FBF755BB00BF1FB2060856
:1041700020720020004850E68AB2060813460A461C
:104180000146014849E600BF96B2060820B1007812
:10419000B0FA80F040097047012070472DE9F04FD8
:1041A00087B00346FFF7F2FF064618B107B0BDE837
:1041B000F04FDFE74649DFF84091DFF840A1DFF834
:1041C00040B105AA184649F049FE34460546B046B6
:1041D0004FF0FF378DB97EB230461EF0A3FF10B10D
:1041E0004568002D5AD1B8F1000F36D1394839460B
:1041F000F9F7ADFB07B0BDE8F08F012E0ED0022E0F
:1042000011D01EB92846FAF7E5F90746304905AA44
:10421000002049F023FE01360546DBE72846FAF781
:10422000D9F98046F2E7494628464BF060FF20B9AD
:10423000294928464BF05BFF08B144F00104514680
:1042400028464BF054FF28B9594628464BF04FFFFB
:104250000028DBD044F00204D8E7002C08BF032478
:104260000023E4B2CDE9008402931A461946304691
:104270001FF01EF9054610B918483946B8E7184826
:1042800042463946F9F763FB39461648F9F75FFBB2
:10429000154B2946D3F8680C3FF03CFA13483946D1
:1042A000F9F755FB5CB16979A14208D01048224664
:1042B000F9F74DFB2B68E1B29B6928469847EB6AFA
:1042C000002BE1D00B48F9F742FB0023EB62DBE760
:1042D000B9050708B6B20608C9ED0608DEB2060839
:1042E000FDB2060868B30608207200201AB306085B
:1042F00032B3060852B3060812C50608B3B2060860
:104300000FCC06082DE9F04F85B00546FFF73EFFBC
:10431000044630B10021012005B0BDE8F04F3FF068
:1043200053BA85492846F9F729FD20B905B0BDE8FB
:10433000F04F39F091B981492846F9F71FFD28B9A6
:10434000012005B0BDE8F04F39F0F2BA7C492846AB
:10435000F9F714FD034688BB7A4A92F9231E82F8C6
:104360001C0E104692F8CE54012D08D0033D052DA9
:1043700005D9002C00F0D28080F8231ECEE092F800
:10438000CF54A52D03F1010313D101290ED16E4A9B
:1043900080F81D3E002380F81C1E82F86C3C80F8DB
:1043A000233E05B0BDE8F04F39F00EBB013949B2EC
:1043B0000124782B02F11402D4D1DAE72846FAF767
:1043C00009F9614B93F96C3C009303FA80F6772E60
:1043D000834600F2A7802846FBF786F907460028A7
:1043E00000F08980FAF7F6F80124C5B23846FBF7E9
:1043F0007BF90746002800F08180FAF7EBF80134DA
:104400000190E4B23846FBF76FF98046002877D078
:10441000FAF7E0F801340746E4B24046FBF764F9E6
:10442000814600286ED0FAF7D5F801340290E4B244
:104430004846FBF759F98246002865D0FAF7CAF8D2
:1044400001340FFA80F9E4B25046FBF74DF9824689
:1044500000285BD0FAF7BEF801340FFA80F8E4B216
:104460005046FBF741F9002852D00390FAF7B2F812
:1044700003990FFA80FA0846FBF736F9034600283D
:1044800057D004F0FD04FAF7A5F8042C46D1C3B2C6
:10449000012D02D9E91E052940D81BB1A52B01D059
:1044A000482B3BD1274C0EB984F8236E142101FB15
:1044B0000646019AC6F8BC24A52B029A86F8CE546B
:1044C000C6F8C074C6F8C424A6F8C894A6F8CA846E
:1044D000A6F8CCA486F8CF340AD100981A4B013044
:1044E000584483F86C0C94F8233E013384F8233E3F
:1044F00005B0BDE8F08F0446054677E7019081E7F7
:1045000007468AE7029093E781469DE78046A7E742
:104510005FFA88F382468046062CB9D005B0BDE824
:10452000F04F27E609487722214605B0BDE8F04F55
:1045300024E60134E4B2EFE796B306089CB306081C
:1045400002C30608849C002020720020A1B3060844
:1045500010B50346FFF71AFE30B1FCF76FF9BDE85E
:1045600010400748FFF7DCBB1846FAF733F804465B
:1045700080B2FCF737F921460248BDE810403FE41D
:10458000AAB30608B6B3060808B50346FFF7FEFD52
:1045900040B10C4B0C480022A3F8662CBDE8084043
:1045A000FFF7BEBB1846FAF715F8014630B1054BC8
:1045B000A3F8660CBDE80840044821E4BDE80840C3
:1045C000D8E500BF20720020C8B30608DEB3060895
:1045D0002DE9F04FDFF8B8A087B0074616460C4625
:1045E00015464FF0000B4FF019094FF46178002E7B
:1045F0004BD0237828788342EB7844D161786A786D
:10460000914240D1A178AA7891423CD1E178CA1A6E
:1046100051425141CDE9041313F07EFF059B0499EB
:1046200019FB03830393AB7819FB038302936B7825
:1046300001934379009352465B463846FFF7B0FB3F
:1046400004992078049113F067FFE378049919FB2B
:1046500003830393A37819FB038302936378019385
:104660004379009352465B4638460BF1010BFFF746
:104670007DFBBBF1280F04F1040405F10405B6D15C
:1046800007B0BDE8F08F0021C4E73146D9E700BF8D
:10469000F5B30608F7B50746FFF778FD044630B1D5
:1046A0002E490022012003B0BDE8F04090E73846D3
:1046B000F9F790FF272806463DDC8500781C8DF829
:1046C0000740FBF711F8074690B1F9F783FF031E87
:1046D0000EDB234A2146DBB202F5C26404EBC10CB7
:1046E000C8009CF805C09C452CD001313829F5D173
:1046F0003846FAF7F9FF044660B1F9F76BFF0D2869
:1047000008D8184B2B4483F86E0C9DF80730013302
:104710008DF80730114FA91C0DF1070239442046CE
:10472000FAF7EFFF9DF80730042B02D0002347F87B
:10473000263003B0F0BD0C482722214603B0BDE867
:10474000F0401BE5074B02442B4492F8142683F8F3
:104750006D2C01238DF80730CAE700BF8D7E002045
:10476000C813060820720020DAB406082DE9F04FBD
:1047700089B0374EDFF8E090069280460C46154629
:1047800002F1300B94F9041000230C22314F02FB8C
:1047900003F0C057884255D00133042BF6D10C35B5
:1047A0005D4504F10C04EDD109B0BDE8F08F95F939
:1047B00004302A68687995F806C095F808E095F8FD
:1047C00007A099423CD12168914239D16179814257
:1047D00036D1A179614533D1217A714530D1E17962
:1047E000A1EB0A077942794156F82A7056F8200061
:1047F000049756F82E70039756F82C700297CDE95F
:1048000000204A4640460791FFF7CAFA0799E27925
:1048100094F9043056F822200492227A56F8222085
:104820000392A27956F822200292627956F8222049
:1048300001922268009240464A46FFF797FAAEE797
:104840000021D1E7069B002BB1D11946DFE700BF5D
:1048500080130608307F002008B40608F0B585B044
:104860000346FFF793FC30B13F490022012005B019
:10487000BDE8F0407AE718465E1CF9F7ABFE044647
:1048800040B21EF0CFFD054630B93848214605B08C
:10489000BDE8F040FFF7C1BA0068696801AB03C327
:1048A000A86818603046FAF71FFF044600284BD06E
:1048B00003782B2B05D02D2B3BD0F9F78BFE0190E5
:1048C00009E001342046F9F785FE019B012202FA36
:1048D00000F003430193022600272046FAF704FF65
:1048E000044600B3F9F776FE214900228C4651F8C0
:1048F00004EB7045D3B203D00132112AF7D1002363
:104900005CF8232090420ED1022F1FD0032F20D01D
:10491000012F14BF8DF809308DF80A3001370136A8
:10492000042FF6B2D9D1012E16D805B0BDE8F0405B
:1049300020E401342046F9F74DFE019B012202FAE2
:1049400000F023EA0003C5E70126C5E78DF80C3027
:10495000E4E78DF80B30E1E701AB03CB2860186882
:104960006960A86005B0F0BD607F002025B406082E
:10497000801306082DE9F04FDFF8C0B089B08046FB
:1049800017460C46154600264FF0190A4FF4617978
:10499000002F51D06979A8780791A1782B786A788F
:1049A00095F803C095F804E00693814242D121783E
:1049B00099423FD1617891423CD1E178614539D14A
:1049C0002179714536D16179079BCB1A59425941FA
:1049D000069B06911AFB0393CDE901031AFB029291
:1049E000079B03920093CDE904CE33465A464046D6
:1049F000FFF7D6F9069923790593E3780493637852
:104A00001AFB0393039323781AFB03930293A3786F
:104A10000193637900935A46334640460136FFF7C7
:104A2000A5F9142E04F1060405F10605B0D109B06C
:104A3000BDE8F08F0021CBE73946DCE738B4060843
:104A40002DE9F3478246FFF7A1FB064630B13C490A
:104A50000022012002B0BDE8F0478BE75046F9F78D
:104A6000B9FD1328054663DC062747430AF1010018
:104A70008DF80760334CFAF737FE04F6745909EBEA
:104A80000708064648B1F9F7A5FD03289FBFE319BB
:104A900083F8790D01238DF807303046FAF724FEAC
:104AA000064668B1F9F796FD0D2809D8062303FBE1
:104AB000054383F8760D9DF8073001338DF80730F4
:104AC0000DF1070241463046FAF71BFEFAF70CFEDD
:104AD000064668B1F9F77EFD3B2809D89DF80730F6
:104AE000062202FB0542013382F8770D8DF807306C
:104AF0003046FAF7F9FD68B1F9F76CFD0D2809D8D1
:104B00009DF80730062202FB0544013384F8780D36
:104B10008DF807309DF80730062B06D0002349F8A2
:104B20000730A8F80430FFF725FB02B0BDE8F08796
:104B300005481322314602B0BDE8F047FFF71EBB1F
:104B4000947F002020720020DAB406082DE9F04F8F
:104B50002DED088BDFF814A197B0074690460C4660
:104B60001546002694ED008AB5EE408AF1EE10FA63
:104B700073D0D4ED019A94ED029AD4ED038AB8F182
:104B8000000F40D095ED000A95ED01BAD5ED02AACF
:104B900095ED03AAB4EE408AF1EE10FA62D1F4EE7C
:104BA0004B9AF1EE10FA5DD1B4EE6A9AF1EE10FA7A
:104BB00058D1F4EE4A8AF1EE10FA0CBF4FF0010919
:104BC0004FF0000912A8F9F715FCB0EE4B0A834626
:104BD0000EA8F9F70FFCB0EE6A0A05900AA8F9F7DB
:104BE00009FCB0EE4A0A049006A8F9F703FC059BFD
:104BF000049A0390CDE900B30292334652464946E7
:104C00003846FFF7CDF8B0EE480A12A8F9F7F2FBE4
:104C1000B0EE690A81460EA8F9F7ECFBB0EE490A3E
:104C200083460AA8F9F7E6FBB0EE680A049006A8E6
:104C3000F9F7E0FB049B0390CDE901B3CDF80090B8
:104C400033465246002138460136FFF78FF80C2EC6
:104C500004F1100405F1100584D117B0BDEC088BE8
:104C6000BDE8F08F4FF00009ACE700BF56B406086E
:104C7000F8B50546FFF78AFA064668B1494991F842
:104C80007A3F4FF4C67202FB031101F6F85100227D
:104C9000BDE8F840012059E7434905222846F9F7C5
:104CA00051F880B93F4A02F6EC5392F87A2F4FF44C
:104CB000C67101FB0233002201300C28DA6003F1D7
:104CC0001003F9D1F8BD2846F9F784FC0B280446F7
:104CD00060D82846FAF708FD0546002842D0F9F7C3
:104CE000EDFB304B03F6EC5293F87A3F4FF4C6716C
:104CF0004B4303EB0413134483ED030A01262846B8
:104D0000FAF7F2FC054678B1F9F7D8FB254B03F624
:104D1000EC5293F87A3F4FF4C6714B4303EB041304
:104D2000134483ED040A01362846FAF7DDFC0546F4
:104D300080B1F9F7C3FB1B4A02F6EC5192F87A2FC7
:104D40004FF4C670631C424302EB03130B4483ED24
:104D5000010A01362846FAF7C7FC28B9BDE8F84031
:104D6000FFF708BA0646CAE70E4F97F87A5FF9F7D9
:104D7000A5FB4FF4C67301346B4307F6EC5103EB0C
:104D800004140C44032E84ED020AE7D10C330022F4
:104D900019447DE731460548BDE8F8400B22FFF78E
:104DA000EDB900BF2072002096B30608DAB40608F9
:104DB0002DE9F043DFF8649085B080460D46164635
:104DC0000227002446B336F8242035F82430F05B5F
:104DD00093421FD1EB5B191A4B424B411946CDE967
:104DE000002023464A4640460391FEF7D9FF039927
:104DF000EB5B019335F8243000934A462346404646
:104E00000134FEF7B3FF042C07F10407DAD105B033
:104E1000BDE8F0830023E1E73146E9E76AB406081C
:104E2000F8B50446FFF7B2F9054628B1BDE8F840E9
:104E3000294900220120BBE728492046F8F79EFFB8
:104E4000A8B9274B4FF47A714FF4FA62A3F8A01F68
:104E5000A3F8A22FA3F8A41FA3F8A62FA3F8A81FB6
:104E6000A3F8AA2FA3F8AC1FA3F8AE2FF8BD2046D5
:104E7000F9F7B0FB0328074627D82046FAF734FC99
:104E8000044670B1F9F7A6FB012506462046FAF75D
:104E90002BFC10B1F9F79EFB2DB9BDE8F840FFF7E8
:104EA00069B90546F2E7A6F2EE2240F2DC539A42D7
:104EB000F3D8A0F2EE229A42EFD8094B03EB870316
:104EC000A3F8A06FA3F8A20FD0E729460548BDE8D4
:104ED000F8400322FFF752B9C081002096B30608BC
:104EE000207200207BB406082DE9F04FDFF800A106
:104EF00091B0834691460C461546002604F11508EC
:104F00000422414609A84BF0CFF800238DF8283041
:104F1000D4E90232082B72F100010BAF56D23049AE
:104F20001A463846F8F730FDB9F1000F55D02B7806
:104F30000793079A237893424DD1D4E90202D5E929
:104F400002139A4208BF884245D1227D2B7D9A42A6
:104F500041D1042205F1150140464BF04FF80028DD
:104F600039D121692B69CB1A594259411D4B0593FF
:104F700000230493B5F912300393B5F9103002936E
:104F8000194B0193079B00935246334658460791AD
:104F9000FEF706FF079909AB0593237D0493B4F947
:104FA00012300393B4F91030CDE9017314F8203BAB
:104FB00000935246334658460136FEF7D7FE082E78
:104FC00005F120059AD111B0BDE8F08F07493846A8
:104FD000F8F7DAFCA8E70021C8E74946DBE700BF9D
:104FE000C4E70608F3D00608F9F1060883B40608FA
:104FF0008EB406082DE9F74F0446FFF7C7F80746B9
:1050000030B170490022012003B0BDE8F04F6BE7DA
:105010006D492046F8F7B2FE014638B969484FF4A9
:10502000807203B0BDE8F04F4AF0A8B82046F9F707
:10503000D1FA83B2072B054600F2BB802046FAF76F
:1050400053FB804600284CD0F9F7C4FA01240FFA2C
:1050500080FB4046FAF748FB68B14FF0000A411E5A
:1050600000F1100C564611F8013F13F0DF0F3BD151
:1050700001270134E4B2FAF737FB804600284CD010
:10508000F9F7A8FA01340FFA80F9E4B24046FAF7CA
:105090002BFB0346002842D00190F9F79BFA01341C
:1050A000019B0FFA80F8E4B21846FAF71DFB03469D
:1050B000002836D00190F9F78DFA0134019B41B2F6
:1050C000E4B218460191FAF70FFB0199024650B37A
:1050D0000134E4B2032C28D803B0BDE8F04FFFF749
:1050E00049B804468346B4E76145C2D0A3F1300213
:1050F000D2B2092A05D9A3F16102052A07D8573B84
:10510000DAB2360146EA1A7642EA0A1AABE7A3F1A6
:105110004102052AADD8373BF2E78146B6E7804623
:10512000C2E70146CDE7294AD4E71FFA8BF3022BE9
:10513000D2D809F226239BB2B3F5E16FCCD808F29E
:1051400026239BB2B3F5E16FC6D8CCB2062CC3D8E8
:105150001046019243F00EFC0428BDD8002FBBD0AE
:105160001B4B019A2DB203EB451103F57B6303EB57
:105170004510C0E902A60346164D81F8B0BFA1F85C
:10518000C09FA1F8C28F81F8C44F1533511E03325E
:1051900011F8010F445D04F00304022C08BF20380D
:1051A00003F8010B087808B18A42F1D103B0BDE8D9
:1051B000F08F09480722394603B0BDE8F04FFEF7EB
:1051C000DDBF00BFD081002096B30608F3D00608EB
:1051D00020720020C1120708AFB406082DE9F0477D
:1051E000DFF874A086B0814690460D46174600262B
:1051F000B8F1000F2ED03B782A789A42D7E9010CFB
:1052000026D16A68824223D1AC68A4EB0C025442D6
:105210005441CDE9010C214600935246334648469D
:105220000594FEF7BDFD0599AB6802936B68019389
:1052300015F80C3B00935246334648460136FEF7BC
:1052400095FD082E07F10C07D2D106B0BDE8F08716
:105250000024DEE74146E7E7BCB406082DE9F84341
:105260000446FEF793FF054628B1BDE8F8432D49F3
:1052700000220120B2E72C492046F8F77FFD0146C5
:1052800028B9BDE8F8432748602249F077BF204697
:10529000F9F7A0F9C3B2072B064606D929462348D9
:1052A000BDE8F8430722FEF769BF2046FAF71CFA6B
:1052B000074628B3F9F78EF9051E18BF012501240A
:1052C0003846FAF711FA0746E0B1F9F783F90134E5
:1052D0008046E4B23846FAF707FA0746A0B1F9F774
:1052E00079F901348146E4B23846FAF7FDF908B19C
:1052F0000134E4B2032C09D0BDE8F843FEF73ABF0D
:105300000446DDE78046E5E78146EDE7084B76B2E7
:105310000C2000FB063646E9118906F8485CBDE81A
:10532000F88300BFD082002096B30608D1B40608E7
:10533000188300202DE9F04FDFF8849091B00746E4
:105340008846164600240DF12C0A04EB840508EB70
:10535000050358F805001B790290514602A88DF804
:105360000C303EF085F94EB3731970591B790490D7
:10537000052204A902A88DF814304AF03FFE0DF171
:10538000180BB0FA80F5594604A86D093EF070F983
:10539000CDF800B023464A4629463846FEF700FDC0
:1053A0002346CDF800A04A46294638460134FEF788
:1053B000DDFC202CC9D111B0BDE8F08F3546EFE7F8
:1053C000E0B406082DE9F04F89B00546FEF7DEFE91
:1053D000044630B167490022012009B0BDE8F04F12
:1053E000A8E72846F9F7F6F81F28074600F3B98022
:1053F0002846FAF779F95F4A0194BB00039307EB5B
:105400008703D118D4505C4B0C7106460293254695
:10541000A246A346A046A146029B05AA13F801CBCB
:10542000029396460023304616F8011B19B18C45AD
:1054300001D00A2B0CD120336B444FF000068C4571
:1054400003F80C6C08D009B0BDE8F04FFEF792BE2F
:105450000EF8011B0133E6E709F1FF33461C032B6D
:1054600003D8DFE803F02C436C7505A8F9F7B2F810
:10547000019009F101095FFA89F9B9F1050FCBD162
:10548000039A3E4B01993A4417469A1818331F4421
:1054900005F00F0004F00F0444EA081440EA01107C
:1054A0004FEA2818107682F819B082F81AA0FC701A
:1054B00087F8048009B0BDE8F04F2CF0F9B805A8D2
:1054C000F9F788F80546D4E74E2B14D0452B14D0B5
:1054D000532B14D0572B14D0552B14D0442B05D15B
:1054E0000523012101FA03F348EA030812F8013BFE
:1054F000002BE9D1BDE70023F3E70123F1E7022305
:10550000EFE70323EDE70423EBE7DFF878C00023A0
:1055100019461CF8013B834204D0072901F101031D
:10552000F6D15946DFF860C000231CF801EB704546
:105530000AD1012000FA03F34AEA030A8B4612F863
:10554000010B0028E1D194E70133072BEDD1F5E7FA
:1055500005A8F9F73FF810280446B4BF0446002414
:1055600087E707481F22214609B0BDE8F04FFEF744
:1055700005BE00BF30830020981B0608188300205A
:10558000DAB406089D1B0608A51B06082DE9F0479E
:10559000DFF870A086B0814690460D46164600277B
:1055A000B8F1000F2BD033882A889A4225D16C8815
:1055B0007188621A54425441F2780292B27805948A
:1055C000CDE9003221463B4652464846FEF7E8FB0D
:1055D0000599EB780293AB78019335F8043B00937F
:1055E00052463B4648460137FEF7C0FB102F06F1F6
:1055F0000406D5D106B0BDE8F0870024DCE74146BB
:10560000E7E700BFEAB406082DE9F8430546FEF7D0
:10561000BDFD044628B1BDE8F8432349002201201E
:10562000B4E72846F8F7D6FF0F2806462DDC2846B3
:10563000FAF75AF828361D4FDFF87C8005464FEA06
:1056400086092846F8F7C6FF37F8023B984223DC64
:10565000012C08EB090310D0022C10D01883284627
:105660002C214AF0EAFC054658B1013501230134EA
:1056700093B1032CE5D1BDE8F8839876EFE7D876AF
:10568000EDE7A21E53425341F1E721460848BDE829
:10569000F8430F22FEF772BD064B002243F8262086
:1056A000BDE8F843FEF766BDD0830020AC1B0608BA
:1056B000DAB4060830830020188300202DE9F04F6B
:1056C00014462C4A85B00646894600274FF0060B43
:1056D0000BFB07F5E0354FF0000819F805A0002C8A
:1056E00043D0635DAAEB030041424141CDE9008311
:1056F00030463B460391FEF753FB03991D4ACDE923
:10570000008A3B46304608F10108FEF72FFBB8F14E
:10571000060F184A05F10105DFD10137062FD7D151
:10572000144F4FF4827519F805A0A5F58278F4B1ED
:10573000635DAAEB030251425141CDE900833A4631
:10574000062330460391FEF72BFB03990623CDE990
:10575000008A3A463046FEF709FB013540F20D1348
:105760009D42E0D105B0BDE8F08F2146C7E7214654
:10577000ECE700BFFCB4060870B586B00346FEF740
:1057800005FD044630B11A490022012006B0BDE8EB
:10579000704093E71749174E02AA184648F05EFB7F
:1057A00003AD80B1032C03D1FEF7E4FC06B070BD5D
:1057B000F8F710FF02AA45F8040B31460020013427
:1057C00048F04CFBEDE7032CEED1DDE90345059BEA
:1057D00001931A462946E0B22CF0C8F80028E3D01D
:1057E000019B05482A462146FEF70AFBDEE700BF7B
:1057F00030830020B9050708FCB406082DE9F04302
:10580000DFF8989087B0804617460C46154600266C
:10581000002F41D0B5F90030B4F90010B5F90220DD
:10582000B5F9040095F906C0994233D1B4F90210D4
:1058300091422FD1B4F9041081422BD194F9061072
:10584000A1EB0C0EDEF1000141EB0E01CDE90032BF
:10585000CDE9020C33464A4640460591FEF7A0FAD0
:10586000059994F906300393B4F904300293B4F91E
:105870000230019334F9083B00934A4633464046D0
:105880000136FEF773FA102E05F10805C0D107B0F6
:10589000BDE8F0830021D9E73946E2E710B50608F4
:1058A0007FB50546FEF772FC00285ED03049002225
:1058B000012004B0BDE87040A0E72D2B03D0A3F178
:1058C0003002092A4CD8042C04DD04B0BDE8704035
:1058D000FEF750BC2846F8F77DFE04AB621C03EBD4
:1058E000440424F80C0C15F8013F303B092BFAD97D
:1058F00014462B78002BE0D1052CE6D1BDF80430FE
:10590000BDF904600F2BE0D8BDF90610A1F5FA72BD
:1059100092B2B2F5FA6FD8D8BDF90820A2F5FA70A4
:1059200080B2B0F5FA6FD0D8BDF90A008142CCDC64
:105930008242CADB9142C8DCBDF90C5005F17D04FE
:10594000A4B2FA2CC1D80B4B03EBC603A3F8261163
:10595000A3F82821A3F82A0183F82C5104B070BDC4
:10596000202BB2D101352246C2E70446C1E700BF71
:105970003E840020188300202DE9F04FDFF8B8B0F6
:105980008FB0804617460C4615460026A388ADF812
:105990002C3023780893B4F902906378206806933A
:1059A000237994F905A00A900793B9F1000F3CD030
:1059B000002F3FD02868BDF828100C9080B2AB882B
:1059C000ADF8343081422A7895F801C0B5F902303B
:1059D00095F804E02CD14B452AD1BDF82C10BDF828
:1059E0003400081A41424141CDE901C30092CDE99A
:1059F00003EA33465A4640460991FEF7D1F9099920
:105A0000079BCDF810A0CDE90293069B0193089B5C
:105A100000935A46334640460136FEF7A7F9202E3A
:105A200004F1060405F10605B0D10FB0BDE8F08F12
:105A30000021D9E73946E3E725B50608F0B589B076
:105A4000044642F097FF10F0FF020DD13C4991F857
:105A50007A3F4FF4C67000FB031101F6B8610120D4
:105A600009B0BDE8F04087E7364905222046F8F73F
:105A700069F9B0B9324B93F87A2F4FF4C67101FB34
:105A80000233314A1568948803F6B863062606FB8C
:105A900000F29918013020289D508C80F7D109B070
:105AA000F0BD20462949294E01AA48F0D7F94FF008
:105AB000FF33079302AD002478B1062C02D1FEF724
:105AC00059FBECE7F8F786FD01AA45F8040B3146CF
:105AD0000020013448F0C2F9EEE7042CEFDD029F0C
:105AE0001F2FECD8039E0F2EE9D8049D262DE6D853
:105AF000059C04F57A73B3F5FA6FE0D80698FF2891
:105B0000DDD807994B1C402BD9D80D4B93F87A2F31
:105B10004FF4C67C0CFB02F24FF0060C0CFB072284
:105B2000134483F8BC0E83F8B86E094883F8B95E55
:105B3000A3F8BA4E83F8BD1EFFF780FFAFE700BFA2
:105B40002072002096B30608B21B0608B9050708A4
:105B5000F3D006082DE9F04F9BB0DFF814A10E93A7
:105B6000074693460C46154600260E9B5A1C01D04C
:105B7000B3426FD1A646BEE80F000DF1400CACE871
:105B80000F00DEF80030CCF80030237B0A93237C32
:105B90000B9394F911300C93A37C94F8048094F83F
:105BA0001390089009920D93BBF1000F5ED0AE46A2
:105BB000BEE80F000DF1540CACE80F00DEF8003029
:105BC000149ACCF8003022F07F4223F07F439A42AF
:105BD0000F9095F804E0A86895F80CC0E97C43D1D3
:105BE000F04541D1089B0F9A93423DD10A9B6345F2
:105BF0003AD1099B834237D1A9EB0103594259415C
:105C0000099B06930A9B0593089BCDF81C90CDE950
:105C100003830D9B02930C9B01930B9B00935246B5
:105C2000334638460F91FEF7BBF80F99099B069350
:105C30000A9B0593089BCDF81C90CDE903830D9B2F
:105C400002930C9B01930B9B0093524633463846BC
:105C5000FEF78CF80136402E04F1140405F114050A
:105C600083D11BB0BDE8F08F0021C9E75946DDE7BD
:105C70003CB506082DE9F0418AB004460D4642F0D5
:105C800079FE10F0FF0210D13F4B93F8641C41B92C
:105C90004FF0FF330A463D4901200AB0BDE8F0410C
:105CA00058E76B1C6CD02B46F5E739490522204696
:105CB000F8F748F838B935484FF47E710AB0BDE8B6
:105CC000F04141F07DBB20463249324E6A4648F0F1
:105CD000C5F801AD002478B1092C02D1FEF74AFACB
:105CE0004EE0F8F777FC6A4645F8040B3146002091
:105CF000013448F0B3F8EEE7092CEFD101993F29C0
:105D0000ECD8DDF808E0BEF1010FE7D8DDF80CC0F3
:105D10000CF10103402BE1D8049F342FDED8059EFF
:105D2000072EDBD8069D1C4A05F5742303F5107376
:105D30009342D3D8079C072CD0D8089800F5742339
:105D400003F510739342C9D8099AFF2AC6D8134B9A
:105D50004FF0140808FB013309B2C3F8B00183F80F
:105D6000B8E10F4883F8B9C183F8BA7183F8AC6120
:105D7000C3F8A85183F8B44183F8BB21FFF77AFF39
:105D80000AB0BDE8F08100BF20720020C08400206E
:105D900096B30608B905070880841E001883002002
:105DA000F3D006084FF0FF3164E72DE9F04F1646B7
:105DB00015461D4A87B007460C464FF0000BD4E944
:105DC000009AD4F8088066B3AB689845D5E900011D
:105DD00025D1814523D1AAEB010359425941CDE98F
:105DE000019ACDF800805B4638460591FDF7D8FF53
:105DF00005990D4ACDF800805B46CDE9019A3846F9
:105E00000BF1010BFDF7B2FFBBF1080F064A04F1DD
:105E10000C0405F10C05D2D107B0BDE8F08F0021CC
:105E2000DDE73146E6E700BF5DB5060870B586B030
:105E3000044642F09FFD10F0FF0205D121490120E8
:105E400006B0BDE87040B0E71F4905222046F7F7CD
:105E500079FF38B91B4840F2FF3106B0BDE8704009
:105E600041F0AEBA20461949184E01AA47F0F6FF94
:105E700002AD002478B1042C02D1FEF77BF91FE0BB
:105E8000F8F7A8FB01AA45F8040B314600200134BD
:105E900047F0E4FFEEE7042CEFD1029A072AECD892
:105EA0000B4B0C480C2101FB0233039AC3F8B026BC
:105EB000049AC3F8A826059AC3F8AC26FFF7B6FFE4
:105EC00006B070BDC089002096B30608B905070862
:105ED00018830020F3D006082DE9F04FDFF808B151
:105EE000A1B0804617460C4615460026A646BEE8D9
:105EF0000F000DF1480CACE80F0023680C932379D8
:105F00000A93A3680B939EE80700238A0D93638A84
:105F10000E93A38A0F93E38A94F80C9094F818A038
:105F200010938CE80700002F5CD0AE46BEE80F004F
:105F30000DF1640CACE80F009EE807002B7E534582
:105F40008CE807004CD12B790A9A934248D12B68F0
:105F50000C9A9A4244D12B7B4B4541D1AB680B9AAA
:105F60009A423DD1169A82423AD117991E9BCB1A7A
:105F700059425941109B08930F9B07930E9B069320
:105F80000D9B05930B9B1191CDE903930C9B029301
:105F90000A9B5A46CDE900A340463346FDF700FF71
:105FA0001199109B08930F9B07930E9B06930D9BD3
:105FB00005930B9BCDE903930C9B02930A9B5A46D6
:105FC000CDE900A3404633460136FDF7CFFE042E4F
:105FD00004F11C0405F11C0588D121B0BDE8F08F47
:105FE0000021C7E73946DCE76EB50608034B9A780F
:105FF0000021101A997018BF012070479881002065
:1060000010B5114B014603F1180253F8044B41F847
:10601000044B9342F9D11B880B800B4900F11A0302
:1060200051F8044B43F8044B9142F9D1118819807F
:10603000054B343053F8041B40F8041B9342F9D14C
:106040001B88038010BD00BFA0350608104A117AD6
:10605000537A0B43D17C0B4351780B4391780B431C
:10606000D1780B4311790B43917B0B43917E0B430A
:1060700092F823100B4392F82F100B4305D192F89E
:106080003D00013818BF012070470120704700BF54
:1060900048AD002070B5244C94F84C3005460E46AF
:1060A00043B1D4E91423904271EB030324BF0023CE
:1060B00084F84C30E36E1D48984710F0010321D05E
:1060C00080F00203C3F3400384F84C30D4E9183164
:1060D0005B1946EB0106C4E91436012384F88030CD
:1060E0004307D4F8880048BF0123A5EB000548BF4B
:1060F00084F88130002D0EDD012084F8800000F04E
:10610000010070BD8207EBD594F84C20002AE7D03F
:1061100084F84C30E4E794F8803013B994F88100A7
:10612000EDE70120EBE700BF48AD0020A0AD002067
:106130002DE9F0438DB0044642F01CFC10F0FF0244
:1061400006D13F4901200DB0BDE8F043FFF7C4BEC2
:106150003C4905222046F7F7F5FD38B938484FF499
:106160007E710DB0BDE8F04341F02AB920463649B2
:10617000354E01AA47F072FE02AD002478B10A2C18
:1061800002D1FDF7F7FF57E0F8F724FA01AA45F826
:10619000040B31460020013447F060FEEEE70A2C84
:1061A000EFD1DDF80880B8F1030FEAD8DDF80CE094
:1061B000BEF1010FE5D8DDF810C0BCF1070FE0D843
:1061C000059F224B07F5742202F510729A42D8D827
:1061D000069E072ED5D8079D05F5742202F510728C
:1061E0009A42CED8089CB4F5004FCAD20998B0F5AF
:1061F000004FC6D20A99B1F5004FC2D20B9AB2F540
:10620000004FBED2124B4FF01C0909FB0833A3F814
:10621000A20083F8A8E00F4883F894C0C3F89070F8
:1062200083F89C60C3F89850A3F8A040A3F8A4108A
:10623000A3F8A620FFF77CFF0DB0BDE8F08300BFF8
:10624000D8AD002096B30608B905070880841E0063
:1062500048AD0020F3D0060837B505460846019141
:1062600042F088FB0199044602462846F7F76AFD8A
:1062700068B92B5DA3F13002092A06D923F0200367
:10628000413B192B01D90134281903B030BD00203E
:10629000FBE7F8B50B4C0C4E0C4F31252068FDF791
:1062A000EBFC616811B13046FDF790FDA16811B1BA
:1062B0003846FDF78BFDFDF70DFD013D04F110049F
:1062C000ECD1F8BDBC35060881D206089EB7060899
:1062D00030B5274885B0FDF7CFFCF5F71FFA28B990
:1062E000244805B0BDE83040FDF71ABDF5F71AFDAA
:1062F00008B92148F5E7F5F71FFD0268037D8179AC
:106300000446407C0290207C0190608A00905208F4
:106310001A48FDF75BFDE51D0C3415F8010BFDF780
:1063200037FDA542F9D1164C1648FDF7A5FC637858
:10633000022B06D007D9032B10D11348FDF79CFC84
:106340000CE01248FAE704F580541148FDF794FC7C
:1063500094F8B431022B06D0032B06D005B0BDE86B
:106360003040FDF7B7BC0B48E8E70B48E6E700BF55
:10637000A4B70608AEB70608BCB70608CBB7060830
:10638000044F0020F9B7060809B806080FB8060838
:106390001CB8060822B806083BB806082DE9F347E2
:1063A0003649DFF8D89001AA47F058FD4FF0000AAF
:1063B0004FF0FF3557465446D0462E4668B9BAF1DD
:1063C000040F50D03ADCBAF1020F13DC2C492B46F3
:1063D000324601203DF082FA0EE0BAF1040F09D8EE
:1063E000DFE80AF0030D12171C00F8F7F3F8064671
:1063F00003281BD9FDF7BEFE02B0BDE8F087F8F711
:10640000E9F805469228F4E7F8F7E4F880463F28D3
:10641000EFE7F8F7DFF804463F28EAE70378482B70
:1064200003D0562BE6D1012700E0002701AA4946F8
:1064300000200AF1010A47F011FDBFE7BAF1050F8C
:10644000D8D1932303FB0655A4010E4E04F47C64BB
:1064500008F03F0844EA080406EB450544EA4734DF
:10646000A5F80041C8E7932303FB0652054B03EB55
:106470004203B3F80071C7F34037E2E7B9050708F4
:1064800048AE002048AD00202DE9F04FDFF864A0B1
:10649000DFF864B085B00646894615461F460024DD
:1064A000002F01DBA7421DD119F8048005B32B5D35
:1064B000A8EB03020AEB83035142D3F82C33009379
:1064C000514123465A4630460391FDF769FC039932
:1064D0000AEB88085A46D8F82C33009330462346F6
:1064E000FDF744FC01340E2CDAD105B0BDE8F08F85
:1064F0002946EDE7A03506084DB806082DE9F0431A
:1065000085B003AA2549264E264FDFF8A08047F024
:10651000A5FC0024024625464FF0FF3942B9012D63
:1065200035DD022D07D120494B4601F8094030E006
:1065300035B1012D12D0FDF71DFE05B0BDE8F08389
:106540001046F8F747F80D288146F4D803AA1349F6
:10655000002047F083FC01350246DFE71146304654
:106560000192F7F70BFC019A04460028EED0114681
:106570003846F7F703FC019A38B111464046F7F761
:10658000FDFB0028D7D10224E0E72C46DEE70649D0
:106590004B460120FFF778FFCFE700BFB90507089A
:1065A00065B8060864D00608D87900209BFA06086A
:1065B0002DE9F04F2DED028B4D484E4D9FED4E8A4B
:1065C0008BB0FDF71DFC0027B946BA464B4B4C4A31
:1065D000196800238B4227DB01371A2F05F1480584
:1065E000F4D14849484BD1E90021520942EAC1623D
:1065F0004649186809684FF47A73B0FBF3F34448CE
:10660000FDF7FEFB0A2299FBF2F302FB13900090C8
:106610009AFBF2F13F4802FB11A2FDF7F1FB0BB030
:10662000BDEC028BBDE8F08F52F8040BA84201D0FC
:106630000133CFE7AC6A4CB107EE904AB8EEE77A87
:10664000C8EE077AFDEEE77A17EE904AD5E90C61BD
:10665000AB6B08934A09EB6B0992089A4FEAE47B0B
:1066600063437609A4FB020C46EAC16602FB0B31C8
:1066700041F28833C01841EB0C014FF47A720023C9
:1066800043F090F8099A04FB02F1804606FB0B1BCD
:1066900041F28833A4FB0601C0184BEB01014FF413
:1066A0007A72002343F07EF8042F2B6C01964FF48E
:1066B0007A72B3FBF2F306934FF00A0318BF8144DA
:1066C00090FBF3F203FB1200CDE9042098FBF3F2F8
:1066D00003FB1283CDE90223089B00932A680E482E
:1066E0002346394618BFC244FDF78AFB74E700BF52
:1066F0006AB80608E8080020002474490028012030
:1067000060270120CC270120D4270120DC2701208D
:10671000E6B8060808B90608B1B806081FB5094B5F
:106720000293094B0193094B0093094A094B0A490B
:106730000A48FDF765FB0A490A4805B05DF804EB15
:10674000FDF75EBB8BAE060894AE06089DAE06084C
:10675000E8AD0608A9AE0608FBAD060836B906087E
:106760004EB9060868B90608F8B50C480C4D0D4E30
:106770000D4FFDF745FB00246CB93268C2F500727D
:10678000920022B157F824100848FDF739FB013474
:10679000222CF1D1F8BD55F82420F2E771B9060892
:1067A000B03C0020AC340020DC38060887B906086D
:1067B0002DE9F84F054642F0DDF8DFF8EC8004469D
:1067C000D8F80090C0B93048304D314FFDF754FA39
:1067D000012655F8041B59B10B783BB106FA04F3B6
:1067E00013EA090F02D03846FDF7F0FA0134F0E75A
:1067F000BDE8F84FFDF76EBA024626492846F7F77E
:10680000A1FA78B92448214C214DFDF735FA54F806
:10681000041B0029ECD00B78002BF8D02846FDF79C
:10682000D5FAF4E72B78DFF864B02D2B03BF0135E0
:1068300004F1FF344FF0010A4FF0000A00265BF824
:10684000047B1FB9BDE8F84F3CF0A8BF224639468B
:106850002846F7F777FAA8B90120B040BAF1000F3F
:106860000AD0F8F71BF80D48FDF706FA39460C4830
:10687000BDE8F84FFDF7C4BA40EA0900C8F80000C7
:106880000848F1E70136DAE795B9060864390608E1
:106890007F09070840C806089FB90608ABB9060873
:1068A000CEB90608B4B90608E03E00202DE9F84F3D
:1068B000054642F05FF8354F0446D7F8A065C8B9E1
:1068C0003348344DDFF8DC80FDF7D6F90127E3B219
:1068D00005EB8302D2F8481441B107FA03F33342BF
:1068E00002D04046FDF772FA0134F0E7BDE8F84FF8
:1068F000FDF7F0B9024628492846F7F723FA60B9B0
:106900002648274C274DFDF7B7F954F8041B0029FA
:10691000ECD02846FDF75AFAF7E72B78DFF880B07D
:106920002D2B03BF013504F1FF344FF0010A4FF066
:10693000000A4FF000095BF8048BB8F1000F03D197
:10694000BDE8F84F3CF02ABF224641462846F7F7FB
:10695000F9F9B8B9012303FA09F3BAF1000F0CD021
:1069600026EA03031048C7F8A035FDF785F941462C
:106970000E48BDE8F84FFDF743BA33430C48C7F85B
:10698000A035F2E709F10109D5E700BF48AD0020C5
:1069900095B90608A035060840C806089FB906083C
:1069A000E83906087F090708ABB90608CEB906081A
:1069B000B4B906082DE9F047814641F0DBFF4D4EA2
:1069C0000446376800BB4C484C4D4D4EFDF7FEF970
:1069D0004FF00C0808FB04F35B5D5A1E0123934043
:1069E0003B4206D020461CF0DDF901463046FDF75B
:1069F000EDF90134182CEDD117B94248FDF73CF9F7
:106A0000BDE8F047FDF766B902463F494846F7F74B
:106A100099F9054678B93D48FDF72EF92C46384DD1
:106A200020461CF0BFF9013401462846FDF7CEF997
:106A30001A2CF5D1E4E799F800302D2B03BF09F1AA
:106A4000010904F1FF344FF0010A4FF0000A4FF042
:106A5000000840461CF0A6F9224605460146484675
:106A6000F7F770F900283BD1BAF1000F1FD0B8F149
:106A7000180F0BD16FF07F4333602548FDF7FCF80A
:106A800029462448BDE8F047FDF7BAB9B8F1190F17
:106A900001D17368F0E7204B0C2202FB083898F80C
:106AA00080345A1E012393401F433760E5E7B8F155
:106AB000180F03D1C6F800A01848DFE7B8F1190F86
:106AC00001D17760F8E7144B0C2202FB083898F8E4
:106AD00080345A1E0123934027EA03073760EBE70F
:106AE00008F10108B8F11A0FB3D1BDE8F0473CF046
:106AF00055BE00BFF07C0020BCB90608203A06084D
:106B0000CDB90608C6B9060840C80608D2B90608B5
:106B1000ABB90608CEB90608A0350608B4B9060810
:106B2000F0B585B0044641F025FF04283DD1631E31
:106B30002546E11C13F8012FA2F16100192898BF26
:106B4000203A8B421A70F5D11A4F261D15F8011BF9
:106B50000191384649F071FA20B10199284649F06F
:106B60006CFA20B105B0BDE8F040FDF703BBB542BB
:106B7000ECD1204620F0C0FE0F48104CFDF77CF809
:106B80000C4901231A5D11F8010B10326A440133DC
:106B9000052B02F8080CF5D1002309488DF80C30BC
:106BA00002A9FDF72DF905B0F0BD0028E4D0FDF7EE
:106BB000E1FAE1E7583B0608DDB90608ECB200202F
:106BC000A1B7060808B504460648FDF755F8064B78
:106BD0001868F8F71FFE054B18681CF0B3FD204637
:106BE00007F05AF8E3B90608807E0020887E00206E
:106BF000034808B5FDF740F80120FFF7E3FF00BFA9
:106C0000EFB906087FB5194B93F8A425012A29D1BD
:106C100093F8A9350A2B05D0154807B05DF804EBA9
:106C2000FDF72AB81122002101A848F0A7FAA623EF
:106C30008DF8003041238DF80130EB238DF80330BF
:106C40000C4B1B788DF80430B22315218DF80530DC
:106C5000684603238DF802108DF8063021F073F892
:106C60000548DAE707B05DF804FB00BF48AD002037
:106C700008BA06089410002017BA060808B50A4892
:106C8000FDF74EF8094B1868F8F7C4FD084B0024CF
:106C900083F8C645C3F8084683F80C4613F060FD38
:106CA0002046FFF78FFF00BF31BA0608807E002024
:106CB00048AD002008B5214B214C1D68D4F81806BA
:106CC0001CF040FD28461CF03DFDD4F81806417923
:106CD0008B0704D4036841F002019B6998470021A7
:106CE0000846F9F739FC00210120F9F735FCD4F802
:106CF0001806FAF711FB78B101210020F9F72CFCF6
:106D0000D4F81806FAF729FB01462846FAF701FBE2
:106D100000210846F9F720FC2846FAF7FDFA00287A
:106D2000E5D001210846F9F717FC2846FAF715FBCC
:106D30000146D4F81806FAF7ECFAD4E7887E00206A
:106D400048AD0020F7B50546FDF720FA044620B10E
:106D500003B0BDE8F040FDF70DBA28461E491E4FAE
:106D600001AA47F07BF82646254640B90B2D18D9D5
:106D700001461A480B22FDF701FA03B0F0BD44B1F9
:106D8000012C0AD001AA39460020013447F066F8E8
:106D9000EBE7F7F71FFC0546F4E7F7F71BFC0646A1
:106DA000F0E7022C0ED1A6F57A73B3F57A7F05D9F8
:106DB0000B484FF4FA624FF47A71DCE7094B03EBAE
:106DC00045039E80074B084803EB45032946B3F96A
:106DD0000420FDF715F8D0E7B9050708DAB406086E
:106DE0005ED40608002801205BBA060870B5044688
:106DF000FDF7CCF9C0B11F4B5E68013630461BF081
:106E0000D1FF34460546E8B901341A2CA8BF002446
:106E100020461BF0C7FF0546A0B9B442F4D1BDE837
:106E200070401548FCF77CBF2046F7F7D3FB0446BB
:106E30001BF0B8FF054628B921461048BDE8704050
:106E4000FCF7DEBF0B4B5C601CF030FF0C482146AA
:106E50002A46FCF7D5FF192C9DBF0A480C2101FBDF
:106E600004000020BDE8704098BF90F880041CF03A
:106E700035BF00BF9410002068BA06087CBA060827
:106E800092BA0608A035060838B517490522044607
:106E900049F0E8F858B9154A13781BB90121117067
:106EA000134A1370BDE838401248FCF739BF124945
:106EB0000322204649F0D6F880B90C4D0C4C2B78B3
:106EC00043B1237833B10D48FCF7A7FF00232B70A3
:106ED000237038BD0A48FCF723FFF7E7BDE83840C8
:106EE0000848FCF79ABF00BF05C10608847E002051
:106EF000857E0020A7BA060823C30608BDBA060887
:106F0000F4BA060808BB060838B50E4D2B7863B1F5
:106F10000D4C23784BB10D48FCF77FFF0C48FCF774
:106F20007CFF00232B70237038BD0A48FCF7A4FEB9
:106F300020F0C6FCF7F7B0FB20F0CCFC0020FFF7F8
:106F400041FE00BF847E0020857E0020BDBA060879
:106F500017BB060835BB06082DE9F0478CB007467D
:106F600010F8013B202BFAD00025204CDFF884805C
:106F7000DFF88490DFF884A02E4601A9204612F0A5
:106F80008DF9394601A849F0B2F8E0B101A94046AF
:106F9000FCF71CFF494601A841F0E2FC00BB20467B
:106FA00012F058FA124B0146007820280CBF5046C8
:106FB0001846FCF70BFFFCF78DFE2046FDF782F824
:106FC000FCF788FE0136013540F25A239D4204F158
:106FD0000B04D2D10EB93CF0E1FB0CB0BDE8F08758
:106FE00000212046FDF762F8E5E700BFBE1B06085A
:106FF000A1B7060846B20608830D07084CB206087A
:107000002DE9F04F2DED028B8FB00578202D06462F
:1070100000F10100F9D0304641F0ACFC044618B153
:10702000012822D12A2D20D19448954DDFF868827D
:10703000FCF776FE002640F25A27284603A912F0F4
:107040002DF903A94046FCF7C1FE0136284621462A
:10705000FDF72CF8FCF73EFEBE4205F10B05ECD126
:107060000FB0BDEC028BBDE8F08F3D21304648F0FB
:10707000E4FF002800F0FA800346994613F8012D3A
:10708000202AFAD0A9EB060901308046074610F8FD
:10709000013B202BF9D07A4D4FF0000A5FFA89F9B5
:1070A00040F25A2B03A9284612F0F8F803A841F041
:1070B00061FC03A9024601903046F6F743FE704B8F
:1070C000044658BB019A4A4528D10B2202FB0A33D9
:1070D0009B7903F00706062E37D1404641F04AFC63
:1070E0008442064623D3674903A841F039FC20B106
:1070F000654903A841F034FC20BB98F80030222BEE
:1071000020D108EB060313F8013C222B1AD1B21E42
:1071100008F10101284612F06BFAA1E70AF1010A11
:10712000DA4505F10B05BDD13CF038FB98E718F8BE
:107130000430A3F16102192A9CBF203B08F80430F7
:107140000134CAE732464146E4E713F0C0030AD0EF
:10715000402B5BD04D48FCF7E9FD2846FCF7B2FF19
:10716000FCF7B8FD7CE798F80030002BF2D04849D6
:10717000404648F0ACFF0446404641F0FBFB8442E9
:10718000E8D14046F7F79AF92846B0EE408A12F067
:107190006EF907EE900AF8EEE77AF4EEC87AF1EEAF
:1071A00010FAD7D8284612F073F907EE900AF8EED5
:1071B000677AF4EEC87AF1EE10FACBDB052E0BD12C
:1071C00018EE104A284612F045F9052E3FD8DFE8A0
:1071D00006F03D3D4747494B042E12D13A4617F879
:1071E000013B202BFAD0092BF8D0013A00240A21C8
:1071F00012F8013F303BDBB2092BE3D801FB04342A
:10720000F6E74046F7F7E6F90446DBE7284612F0D2
:10721000D3F990F804B0814627462346A246BB45E1
:1072200000D91BB1BAF1000F94D0CBE7D9F80030E8
:10723000414653F82700F6F7A1FD002805BF3C465C
:10724000012300234FF0010A0137E8E7047003A986
:107250001048FCF7BBFD00212846FCF727FFFFE69E
:107260000480F4E70460F2E70460F0E730460FB012
:10727000BDEC028BBDE8F04F6EE600BF3CBB0608DC
:10728000BE1B0608830D07084EBB060872BB060826
:1072900059BB060867BB060846B206082DE9F04F41
:1072A000A5B0C04B0293C04B0193C04BC04AC1492B
:1072B000C1480093C14BC24CC24DC34FFCF7A0FD67
:1072C000C249C348FCF79CFDC24BC34819684FF440
:1072D0007A73B1FBF3F1FCF793FD09A8F6F74EFEC4
:1072E000BE4B09A9B3F9002019A83EF081F919A9EC
:1072F000BB48FCF785FD21F051F894F8453605EBC5
:1073000083036422D3F8C035B0FBF2F102FB110213
:107310000093B44894F8443692B289B2FCF770FDF9
:10732000B14BB2481968B24BB1FBF3F1FCF74EFD1B
:10733000D7F81C80002605F5BA6904F2466A05F202
:10734000EC5B0123B34013EA080F0BD059F8263049
:1073500043B11AF806205BF8261053F82220A548FE
:10736000FCF734FD0136072EEBD1FCF7B3FCA24845
:107370009F4EFCF7D5FC0CA8F2F7DCFF0C999F4858
:10738000B1FBF6F1FCF73CFD0D999D48B1FBF6F120
:10739000FCF736FD0E999B48B1FBF6F1FCF730FD8A
:1073A0000F999948B1FBF6F1FCF72AFD21F0F4FBA7
:1073B00005EB8000D0F81416079121F0F7FB05EBE0
:1073C0008000D0F81426069221F000FC05EB800026
:1073D000D0F81436059321F01DFC05EB8000D0F8A1
:1073E000149621F039FC064621F080FC804621F0FD
:1073F00065FC05EB800005EB8808D0F814060390C7
:1074000005EB8606D8F814060290D6F814060799FC
:10741000CDE90090DDE905327C48FCF7F1FC7C4BBE
:107420001B68DB031CD57B4B93F80080B8F1000F81
:1074300016D07948DFF83892DFF838A24146FCF7D9
:10744000DFFC0026B9F90220314650460136FCF730
:10745000BDFCF3B2434509F11009F3D3FCF73AFC44
:107460000020FEF735FF6D4B6D4A1E886D4B6E494F
:107470001B686E48DFF800A2DFF80092DFF8008298
:10748000DFF800B2C3F500739B00FCF7B9FC684A53
:10749000684B6948D31A694AB6B231461288FCF77C
:1074A000AFFC6748FCF73CFC04265AF8041B65480F
:1074B000FCF78CFC6448FCF7DFFB19F8011B002982
:1074C00040F097816148FCF7D7FB6148FCF7D4FB9B
:1074D00058F8041B002940F090815C48FCF720FC20
:1074E000013EE2D1398C5B48FCF770FC5A490A6FC7
:1074F0005AB107EE902ADFED596AF8EEE77A86EE88
:10750000A77AFDEEC77A17EE902AD1F800315BB169
:1075100007EE903ADFED516AF8EEE77A86EEA77A49
:10752000FDEEC77A17EE903A896A59B107EE901AC4
:10753000DFED4A6AF8EEE77A86EEA77AFDEEC77AC3
:1075400017EE901A46480091464FB4F85416DFF8EB
:107550003891FCF755FC4448FCF78EFB3E6826F05A
:10756000004626F07F064FF00108002E40F04981CA
:10757000FCF7B0FB3B685F0140F18C8010A811F074
:107580009FFF002840F08680109B40F259229342D2
:107590009DBF36480B2606FB0300304619A911F0A3
:1075A0007DFE73E08BAE060894AE06089DAE06081D
:1075B000E8AD0608FBAD060838B90608A9AE06080E
:1075C00048AD0020A0350608002801204EB9060865
:1075D0006AB90608C42A0020B5BB0608403D002051
:1075E000CFBB0608E0BB06086006002005BC060805
:1075F00040420F0015BC06081DBC060832BC060838
:1076000044BC060856BC060868BC06087ABC0608D6
:10761000F4270120F0270120CDBC0608F02B002024
:1076200000000220AC3400200018000001BD060854
:10763000008000080040000839BD0608DC3E00203C
:1076400073BD060886BD06088EBD0608C8B90608C3
:10765000A4BD0608AEBD0608E80800200024744951
:10766000BEBD060858270120FBBD0608BE1B060844
:10767000043E0020F2BC0608C43B060895B3002077
:10768000286100209DBD0608CEB90608734819A9D7
:10769000FCF7C3FB7248FCF7EFFAD4F85816002940
:1076A00000F0C2800B7B4A7B6E488968FCF78EFB3A
:1076B000FCF710FB6C48FCF7DFFAD4F85C06FCF72B
:1076C00076FA002800F0B48010A9D4F85C06FCF724
:1076D000B6FA9DF854109DF86030179A6348FCF78D
:1076E00075FB149911B16248FCF770FB129911B146
:1076F0006048FCF76BFBFCF7EDFA5F4B1B68180664
:107700006AD594F86036012B66D85C48FCF7B4FA69
:10771000D4F81C36B3F5487F00F0988000F28C80D6
:10772000B3F5167F00F09480B3F52F7F00F09280C0
:107730005349544AB3F5FA7F08BF114694F823061B
:1077400094F8213694F82026072896BF05EB800090
:107750000020D0F8940600904B48FCF737FBFCF76C
:10776000B9FA4A48FCF74CFB4948FCF7D9FA4948B2
:10777000FCF7D6FA94F86C3619070AD594F87426F3
:1077800094F875164448C2F3C002C1F3C001FCF777
:1077900037FB94F86C365A070AD594F8742694F897
:1077A00075163E48C2F38002C1F38001FCF728FB46
:1077B00094F86C369B070AD594F8742694F87516DD
:1077C0003748C2F34002C1F34001FCF719FB94F8BB
:1077D00070163448FCF714FB334B1B7833B105EBC0
:1077E00083053248D5F8B416FCF70AFB25B0BDE88E
:1077F000F08F5846FCF7EAFA67E65846FCF700FBBC
:107800006EE696FAA6F3B3FA83F308FA03F2062BB0
:1078100026EA02067FF7A9AE05EB83034846D3F8B4
:107820001816FCF7D3FAA0E62148FCF725FA3FE743
:107830002048FCF721FA5EE7B3F5617F0CD01049D0
:107840001D4AB3F57A7F08BF114677E71B4975E7F4
:107850001B4973E71B4971E71B496FE712BE060816
:1078600026BE06082CBE060845BE06084BBE060806
:1078700069BE060872BE0608E03E00208EBE0608FD
:1078800082BB060898BB060894BE0608BBBE060865
:10789000D0BE0608F1BE0608FDBE06080FBF0608EA
:1078A00020BF060832BF0608CB7C002049BF06086F
:1078B00039BE060881BE0608ADBB06088ABB0608AD
:1078C00091BB0608A6BB06089FBB06082DE9F3413D
:1078D0001A481B4C1B4E1C4FDFF87080FCF790FAC7
:1078E0000025E2792168A37994F808C006EB8202AA
:1078F00001F13F41D2F8CC06A28806EB830301F5E3
:107900007E01B2FA82F2890AD3F83C33C2F11F0237
:107910004131BCF1000F0CD0CDE900C04046FCF76E
:107920006FFA0135312D04F10C04DAD102B0BDE853
:10793000F08100903846FCF763FAF2E763BF06086F
:1079400038730020A03506088FBF06087FBF0608E1
:1079500010B5F4F7DEF9124CD0B11248FCF7FAF981
:107960001148FCF789F92068F7F754FF4FF47A7053
:10797000FBF77AFC0D4B18681BF0E4FE0C4B1878F3
:10798000F9F74CFB02210120F3F7C4FAF9F73EFDA9
:107990000848FCF771F92068BDE81040F7F73ABFD6
:1079A000807E00209DBF0608E3B90608887E00207F
:1079B000F0270120BDBF06082DE9F0410446254E01
:1079C000254DDFF8B0800020FEF710FB2348FCF7C0
:1079D000C1F9B17822480131FCF712FA2146202082
:1079E000FCF7B8FA1F48FCF7B5F9B3781E4A4FF414
:1079F000C67707FB0353D3ED037AF5EE407AF1EE39
:107A000010FA0CBF012100212046FCF7AFF9B17834
:107A100079430C3108EB010220462944FDF796F822
:107A20001248FCF797F9B378114A07FB0353204635
:107A3000B3F9CE10B1FA81F14909FCF797F9B178A1
:107A40007943CC3108EB010220462944BDE8F041DE
:107A5000FDF792BF9881002080920020ECBF0608BD
:107A6000FABF06080DC0060820C006082FC0060889
:107A700042C006080C800020A0F2DC50164BB0F586
:107A8000FA7FA8BF4FF4FA70984210B5B8BF1846F5
:107A90000C4611463BF089FF00B207EE900A9FEDBD
:107AA0000F7AF8EEE77AE4B287EE870AFBEE096A0E
:107AB000E0EE006A07EE904A9FED097AF8EE677AE9
:107AC000A7EEA67AF3EE097A20EE070A80EE270ADF
:107AD00042F0A8FB00B210BD0CFEFFFF0000C84240
:107AE00000401C452DE9F843884D95F87D062DEDA5
:107AF000028BB0EE408A80B3854E864FDFF8289225
:107B0000002405F5CF6895F8A436062202FB03731E
:107B1000234493F84A3753B1012B0DD00134042C80
:107B200006F10206EFD1BDEC028BBDE8F88308EB4D
:107B300044031B8E3380F1E7032C01D00023F9E7C7
:107B4000D9F80030DA0405D412F09EFD00B2724B71
:107B50005885E3E740F2DC50F9E76F4C1FF0ECFE8C
:107B6000E76AD5F8B06695F8B42617F4807714BFA5
:107B7000717B317AFFF780FFA08401201FF0DCFECB
:107B8000002F00F08480717B95F8B426FFF774FF16
:107B9000E08402201FF0D0FE002F7AD0B17B95F850
:107BA000B526FFF769FF404200B22085002F72D052
:107BB000A28CF37BE18C13FB02F3642293FBF2F3C0
:107BC000A384337C13FB01F393FBF2F3E384737C14
:107BD00013FB00F090FBF2F0208511F0C5F895F84A
:107BE0007C36608543B9B4F92830626AC5F8A826A6
:107BF000A5F8AC36A5F8AE06E36A5B0693D5B4F9F2
:107C0000343007EE103AB8EEC77AF2EE046AC7EEE7
:107C1000267AB5F9C03608EE103AB8EEC88A37EEC3
:107C2000C88ADFED3E7ABDEEC88A18EE103A1BB264
:107C300008EE103AB8EEC88A28EE278AB0EE480A55
:107C4000F5F7FAF9F0EE408AB0EE480AF5F792F946
:107C5000B4F9263007EE903AB4F9243006EE903AA3
:107C6000F8EEE66AF8EEE77A26EE807AA7EEA87AD2
:107C700060EE677ABDEEC77AE6EEA87AFDEEE77AA7
:107C800017EE903AA38417EE103AE3844BE7317A6B
:107C90007AE7717A83E7224EB4F924003378122B05
:107CA00008BF204BB0EE480A08BF1860002112F050
:107CB00041FC3378122B02BF1A4BB4F926209A608C
:107CC00000B208BF5860A084B0EE480A0121B4F9A0
:107CD000260012F02FFC3378122B02BF114BB4F99F
:107CE00028201A6100B208BFD860E084B0EE480ACC
:107CF000B4F92800022112F01DFC3378122B08BFC2
:107D0000084B00B2208508BF586166E748AD0020E7
:107D100024280120A03506080028012035FA8E3CD1
:107D20005C7E0020607E0020F82701202DE9F043D2
:107D3000DFF8F891774CD9F80030D3F82880764BEB
:107D40001B6813F0100F87B040F0A68094F838300D
:107D5000002B00F0A180714E06F2C465D6F8CC3637
:107D600028469847002800F0978096F82937002B7E
:107D700043D1022384F85830B6F92A3707EE903AF7
:107D8000B6F92C37F8EEE77AC5ED0A7A07EE903AA5
:107D9000B6F92E37F8EEE77AC5ED0B7A07EE903A92
:107DA000F8EEE77AC5ED0C7A5D4903AAA1F10C0063
:107DB0003CF0E2FD03A996F80827084620F07AFC7B
:107DC00003A820F043FC95ED060A5649554D03A83B
:107DD0003CF0DFFD05F178070026B5EC010AD4F888
:107DE000243185ED020A384698470136032E05ED09
:107DF000010A07F12407F0D14EE094F85830012B26
:107E0000D2D1EB6903932B6A049303A96B6A0593A0
:107E100004F15800F5F742FC94F85830012B4FF06C
:107E2000000772D0022B67D0039704970597DDED0A
:107E3000037A9DED047ADDED056AC5ED0A7A85EDDC
:107E40000B7AC5ED0C6AFDEEE77ABDEEC77AFDEE62
:107E5000E66A17EE903A17EE102A16EE901A1BB249
:107E600012B209B2A6F82A37A6F82C27A6F82E17C0
:107E70000120CDE9002104212B4AF5F79BFDD9F81B
:107E8000003000200021C3E90C01C3E91001C3E95F
:107E90000E0127646764A764E3695B0629D51F4D5B
:107EA00095F860372BB34FEAE8763146404641F00B
:107EB000E3FB05F5E76307EE900AD4ED106A93ED56
:107EC0000F7AD5F88027D5F88417A7EEA67A12EB9B
:107ED000080246EB0106D4ED116A83ED0F7A93EDAB
:107EE000107AC5F88027A7EEA67AC5F8846783EDD7
:107EF000107A07B0BDE8F083236F0393D4F888307D
:107F00000493D4F8A030059391E7AF62EF622F633A
:107F1000BFE700BF002801205827012048AD0020FE
:107F200034B40020402801204FC00608EC2701206F
:107F300038B52D4B1B68580350D5D90609D42B4BA7
:107F40001A782B4B302101FB0233D3F87037DA0556
:107F500045D4284B5D79002D40D0274AD26A93073B
:107F60003CD02DB212F090FB044611F08BFC9FED3B
:107F7000237AB4EEC70AF1EE10FAF7EE007A30D4A5
:107F8000B4EE670AF1EE10FAC8BFB0EE670A07EE6A
:107F9000105AC7EE806A184DB5F92A301B1B002114
:107FA000B8EEC77ADFED165A87EE256A76EEE76AF5
:107FB000E6EE867AB0EE677A07EE903AF8EEE76A78
:107FC00007EE904AF8EEE77AE6EE877AFCEEE77A7B
:107FD00017EE903A98B212F05DFD688538BD6425C1
:107FE000C0E7B0EE470AD2E7F4270120849C0020C6
:107FF000A035060898810020002801209A99193F91
:108000000000C842034B012283F89027022283F824
:108010009127704748AD002070B50D4E35782D1A68
:1080200018BF01250328044634BF04460024204617
:10803000F6F786FC074B347003F292701A2204FBA9
:108040000200C3F8B0061AF051FD284670BD00BF0B
:108050009881002048AD0020022810B50C4614D8A5
:10806000FFF7DAFF0948FBF775FE094B0948197855
:108070000131FBF7C5FE21460820FBF76BFF2146C7
:108080001020BDE81040FBF765BF10BDB5C706085E
:108090009881002000C0060838B5154C154DAC423B
:1080A00013D30020F6F74CFC13481FF025FC134AAD
:1080B000136843F48003136000BF114B1878FFF777
:1080C000ABFFBDE8384029F0F3BAB4F90230002B19
:1080D0004FF00001204607DAF6F722FC0121204686
:1080E000F6F71EFC02212046F6F71AFC1434D6E7F8
:1080F000F8160708E41B070876C00608E03E0020D3
:108100009881002010B504460A48FBF7B5FDFFF73B
:10811000C3FF1FF0D5FBF6F7BFFA1FF0DBFB064BE2
:108120000649002220461A70FEF796F808B9FEF7B5
:1081300049FD10BD7FC00608857E00203DC10608B0
:1081400010B5064B5C78241A18BF0124032828BFF9
:108150000020587020F0E4F8204610BD98810020DF
:10816000022810B50C4610D8FFF7EAFF0748FBF7C6
:10817000F1FD074B074859780131FBF741FE2146D5
:108180001820BDE81040FBF7E5BE10BD95C00608FD
:1081900098810020A5C006082DE9F04F0D468DB04E
:1081A000B0490446FEF758F80646002840F0AD8076
:1081B000AD492046FEF750F80646002840F0A7805B
:1081C000AA492046FEF748F80646002840F0A1805C
:1081D000A7492046FEF740F80646002840F09B805D
:1081E0002046A449FEF738F80028064612BF10249E
:1081F000264601240DB144F020049F4D9F4F95F871
:1082000000A095F8019095F80280DFF8D8B25F459C
:10821000C0F08380FFF740FF5046FFF7FDFE484661
:10822000FFF78EFF4046FDF7E1FE95493046FEF729
:1082300013F808B144F0400414F01103009300F067
:1082400083829048FBF786FD0020FEF767FA8E4890
:10825000FBF780FD8D48FBF763FD04F03003302B06
:1082600002D18B48FBF776FD8A48DFF87C92FBF75A
:1082700071FD8948FBF76EFD4FF0FF33874A88494F
:108280002046FEF701F98748FBF764FD864A8749D7
:108290002046FDF7B3FA8648FBF75CFD854A864920
:1082A0002046FCF79BFF8548FBF754FD844B854A2D
:1082B0001E68854B1F6867EA0603CB464FF0000A2D
:1082C00001935BF8043B002B34D01978D1B10199AC
:1082D00002934FF0010808FA0AF811EA080F14BFD8
:1082E000012100212046FBF75BFD66EA070111EA48
:1082F000080F744A029B14BF012100212046FBF79E
:1083000035FD704A0AF1010ADBE7012472E7022415
:1083100070E704246EE708246CE77B88C3F30B0244
:108320001B04D7E9011048BF02EB420244F088FD6C
:1083300014376CE79846654A67EA0603019359F8D3
:1083400004BBBBF1000F27D09BF8001009B34FF01E
:10835000010A0AFA08FA17EA0A0F0BD066EA0701BF
:1083600011EA0A0F5B4614BF012100212046FBF7EA
:1083700017FD564A16EA0A0F0BD0019B13EA0A0FA3
:1083800018BF01215B4608BF00212046FBF7EEFC29
:108390004E4A08F10108D2E74D48DFF850A1FBF73B
:1083A000D9FC4C4AD2F800904B4A12685E4689EAE2
:1083B0000208DFF83CB16FEA08080127B74018EA65
:1083C000070F14BF0121002119EA070714BF524605
:1083D0005A463046039101921AF0E4FC019A03993F
:1083E00002900346204601910136FBF7D9FC002F8D
:1083F00014BF5A465246029B01992046FBF7B6FC31
:10840000182EDAD13548DFF8ECA0DFF8EC80DFF881
:10841000EC90FBF79FFC324BD3F8E8770026F3B2E1
:108420000AEB8302D2F848B4BBF1000F68D00121F7
:10843000994039405B460CD04A4600212046FBF764
:1084400095FC5B464A4600212046FBF7A9FC013615
:10845000E5E7424620460191FBF788FC01995B461F
:108460004246F1E7CFC00608B5C7060895C0060822
:10847000ECBF0608D6C0060898810020F816070849
:10848000DAC0060826CB0608E7C00608FFC00608C3
:108490000BC1060810C8060846C10608D879002096
:1084A0009895002056C106083E840020808F002049
:1084B00066C10608D08200201091002057C6060829
:1084C000E43E00206FC10608E03E00207BC10608A4
:1084D000F3C4060880950020F07C002086C10608C1
:1084E00048AD0020E41B070864390608BAC0060836
:1084F000C4C00608A03506089BC106088FC106083F
:1085000099489A4EFBF726FC012399488DF820B034
:108510008DF810B08DF821B08DF811B08DF822B023
:108520008DF812B08DF823B08DF813B01F46A6F564
:10853000127E9A5D10F801CB02F13001694401F816
:1085400020CC13F80E1001F13008E84408F810CCE4
:108550002FB1A2EB010CDCF1000747EB0C07013354
:10856000052BE6D13946834A002608AB20468DF814
:108570001460FBF715FC04AB39467E4A2046FBF736
:10858000F5FB7D48FBF7E6FB7C4A7D492046FCF77E
:10859000EDF87C48FBF7DEFB7B4A7C492046FCF784
:1085A000C9FE7B48FBF7D6FB7A4A7B492046FCF79D
:1085B000EDFF7A48FBF7CEFB734A74492046FDF77E
:1085C0007DF87748FBF7C6FB764A77492046FBF7EC
:1085D000FFFF7648FBF7BEFB754A76492046FCF75D
:1085E000C9F97548FBF7B6FB744A75492046FCF794
:1085F000DFFB7448FBF7AEFB734A74492046FCF777
:1086000073FC7348FBF7A6FB724920463BF0DCF88D
:108610007148FBF79FFB4FF0FF331A466F49204626
:108620003BF05CF96E48FBF795FB4FF0FF336D4A6A
:108630006D492046FDF78EFA6C48FBF78BFB6C4AC0
:108640006C492046FDF7B1FB6B48FBF783FB6B4A97
:108650006B492046FDF740FC6A48FBF77BFB21464F
:108660003046FBF777FCE7065FD5204695F800809B
:108670006F7895F80290FFF79FF921463046FFF793
:10868000EBFC21460120FFF7E7FC21460220FFF723
:10869000E3FC21463046FFF763FD21460120FFF74A
:1086A0005FFD21460220FFF75BFD4046FFF7B4FC6B
:1086B0003846FFF745FD4846FDF798FC5248FBF762
:1086C00049FB524809F10101FBF79AFB504808F1B8
:1086D0000101FBF795FB4F48791CFBF791FB200745
:1086E00004D5AB7813B92046FFF766F9A10703D587
:1086F00028782146FFF7B0FC620703D56878214649
:10870000FFF72EFD009B13B14348FBF723FB2EB16F
:108710004248FBF71FFB4248FBF702FB414C424D2E
:10872000AC4213D30DB0BDE8F08FAB7813B920463F
:10873000FFF742F928782146FFF78EFC687821463A
:10874000FFF70EFD0126CAE7009EC8E76388C3F362
:108750000B021B04D4E9010148BF02EB420244F0C2
:108760006FFB1434DCE700BFA8C1060834B5002055
:10877000583B0608BEC10608C5C10608607F002038
:10878000AC940020CBC1060830830020009000206C
:10879000D0C10608D0830020A0900020DAC10608CE
:1087A000E9C106088D7E0020E0940020F5C106088E
:1087B000947F0020349400200CC20608C081002061
:1087C000709200201DC20608D08100207091002008
:1087D00029C2060858B5002048C20608B8BE0020C5
:1087E00059C20608C0840020808A00206CC2060896
:1087F000C0890020208A00208AC20608D8AD002047
:1088000050C30020CFC00608A7C20608CAC2060887
:10881000D0C20608DBC20608EEC2060807C3060877
:108820001DC30608F8160708E41B07080021B3E477
:108830000121B1E42DE9F74FC04CC14B9C42C0F07F
:108840006981C04C2078FFF7E7FB6078FFF778FC80
:10885000A078BD4CFDF7CAFB94F8903594F89125AB
:10886000BA489A4224BF002384F89035F6F716F8E8
:10887000B74B1A68B74B934312D100212520F1F76B
:108880006BF9054660B100212720F1F765F938B191
:1088900002682B689A4203D14FF48030F5F7FEFF4F
:1088A0000026AD4F35464FF0FF0848F2B83957F86B
:1088B00026004308810801F0333103F077330B447D
:1088C000C10801F01131C31A5B1A03EB131310F046
:1088D000010203F00F33B3FBF8F1C1EB012118BF24
:1088E0000135A3EB010318BFEDB2012B08D9022B10
:1088F0000CD112B110EA090F02D13DF08DF828B168
:1089000003360C2ED3D1013D022D03D992480D21FF
:108910003EF056FDB4F8BE35B4F8BC25643B934236
:10892000A8BF1346A4F8BC3500BF94F8283613B985
:10893000082384F82836002010F0C2FD874D2B68EC
:10894000002800F0398123F080632B60844BDFF82E
:108950002882D3F8B07611F097FE824B39781E88C2
:1089600083B2361A6422009306FB01F393FBF2F301
:1089700013FA80F0A4F83E0697F80190C1F16E0357
:1089800001EB810CA2EB090B9BB24A42C1F1640ED0
:108990004FEA4C0C92B201935FFA8EFE4FF00A0A36
:1089A00017B2002F40F30B81704607FB07F309FB5A
:1089B00003F310FB00F093FBF0F0584407FB00F3C7
:1089C00093FBFAF363441BB24FF47A70734393FB47
:1089D000F0F30098034428F8023B0A32019B92B25C
:1089E0009342DDD11FF0B6FC19F018FE30220021B1
:1089F0005D4846F0C3FB10F097FB594B93F87C267B
:108A00004ABB93F83A00C3F888266421C82611FBB4
:108A10000060C3F8800693F83B00C3F88C2611FB76
:108A20000061C3F88416C3F8902693F83D10C3F88C
:108A30009426C3F89826C3F89C2683F8A52683F8C5
:108A4000A62683F87D26C3F8A8264FF07A7283F80D
:108A5000A416C3F8AC262B6844499B060A6800F1AB
:108A6000B280B4F88605B4F884350343B4F88805B9
:108A700003431BB2002B40F0A680B4F98A35B3F54E
:108A8000805F40F0A080B4F98C35B3F5805F40F092
:108A90009A80B4F98E35B3F5805F40F0948022F46B
:108AA00000720A601FF07CFBB4F87026DFED307AAC
:108AB000304B07EE102AB8EEC77AB4F87226C7EE2C
:108AC000276A07EE102AB8EEC77AC3ED506AC7EEE0
:108AD000276AB4F8742607EE102AB8EEC77AC3EDF9
:108AE000516AC7EE276AB4F8762607EE102AB8EE68
:108AF000C77AC3ED526AC7EE276A94F8782683F8DE
:108B00005021C3ED536A18F08FFE03B0BDE8F04F5B
:108B100035F09CBAB4F90230DFF86090002BADBF9D
:108B2000002703274FF00108B846002608EB06018E
:108B3000C9B28F4224D214347FE600BFF81607086A
:108B4000E41B07089881002040BE00202063140623
:108B5000E03E002040000100607F002058270120F7
:108B600048AD0020D03E002080C40020F427012022
:108B700000401C4600280120282901200080000810
:108B8000234A02F1060ACA453DD21588DDB35019C1
:108B9000484538D2052D36D9B4F800C0B2F802E005
:108BA000CCF30B0CE64505D192F805C00CF0030C94
:108BB0008C450BD00246E4E743F08063C5E614BF62
:108BC00008460120F1E642F400726AE73146204689
:108BD00092F804B0F5F7A4FE2188BBEB113F10D149
:108BE000B4F802C06068CCF30B01AA1F8A42A8BF88
:108BF0000A461CF4004F18BF01FB0600514644F022
:108C00001FF9013692E731462046F5F789FEF8E76D
:108C10000140000810B5154C94F89137022B18D17B
:108C20001EF04EFEF5F738FDFFF704FE1EF052FE73
:108C300001201BF091F80E4B0E491B6803F59C5365
:108C40000022083384F89027C1F8803684F89127F1
:108C500010BD012BFCD11EF033FEF5F71DFD1EF0FB
:108C600039FE002384F89137F2E700BF48AD0020B9
:108C7000C42A002040BE002010B50446FFF7CCF9FE
:108C800038B11EF01DFEF5F707FDFFF7D3FD1EF00E
:108C900021FE601CC0B2BDE810401BF05DB838B5C5
:108CA0000C4D04462046FBF771FA38B10A4B0B48CD
:108CB0001978BDE838400131FBF7A2B82046F5F736
:108CC00089FC0138022804D8C0B2FFF7D5FF2C4632
:108CD000E8E738BDF3D0060898810020D0C2060826
:108CE00010B50446FFF72CFA38B11EF0E9FDF5F790
:108CF000D3FCFFF79FFD1EF0EDFD601CC0B2BDE888
:108D000010401BF029B838B50C4D04462046FBF73F
:108D10003DFA38B10A4B0B485978BDE8384001316B
:108D2000FBF76EB82046F5F755FC0138022804D849
:108D3000C0B2FFF7D5FF2C46E8E738BDF3D00608F0
:108D400098810020DBC2060810B50446FDF74EF9F5
:108D500038B11EF0B5FDF5F79FFCFFF76BFD1EF077
:108D6000B9FD601CC0B2BDE810401AF0F5BF70B587
:108D70000C4E04462046FBF709FA054638B10A4B6B
:108D80000A489978BDE870400131FBF739B82046B0
:108D9000F5F720FC012804D12846FFF7D5FF34461B
:108DA000E8E770BDF3D0060898810020CAC2060823
:108DB00038B5144DEC69630702D538F00DFCF8B1F5
:108DC000200703D5104B1B68D90519D5A20602D57B
:108DD00038F0A2FCA0B138F055FB10B9FDF736F918
:108DE00068B995F85431012B04D1A30702D5FDF7DA
:108DF0002DF920B91FF0FAFF80F00100C0B238BD94
:108E00000120FCE700280120F42701202DE9F84388
:108E1000924C256815F0040705D0BDE8F843012100
:108E20000020F7F799BBFFF7C3FF8D4E002800F035
:108E3000B58045F40075256086F88476894F2568ED
:108E400097F8A636012B96F8863614BF45F4802590
:108E500025F4802525603BB90FF05EFF002800F067
:108E6000AB8025F40025256036F0BAF950B197F8AB
:108E7000B70625680FF038FF002800F0A08045F401
:108E800000052560DFF8FC81DFF8FC91D8F80020B0
:108E900023681507B9F8202054BF43F4807323F4E6
:108EA0008073632A8CBF43F4806323F480630020C3
:108EB000236035F01FF82568002800F0838045F412
:108EC0000065D9F81C3018077FD5D8F80020D105E7
:108ED0007BD445F480559A07256079D5D8F80030C1
:108EE0009B0575D4FDF7B2F8002871D045F4005504
:108EF00025601FF013FF256800286CD145F400455C
:108F0000122025600FF09CFF002867D045F48035C3
:108F1000172025600FF094FF002862D045F400353B
:108F20001B2025600FF08CFF00285DD045F0807578
:108F30002560FAF7BDF8D6F890364B4AC01A526849
:108F40004A4B61EB02015A7A022A50D8484B494DEC
:108F5000002A18BF2B462568984271F1000397F844
:108F60002A3034BF45F0005525F00055256093B1F7
:108F70002A200FF065FF002840D096F89836002B85
:108F800043D0B6F88A2632B13B4BD6F89C161B6804
:108F90005B1A934239D225F0805538E096F8843632
:108FA00025F400752560002B7FF448AF012086F87A
:108FB00084061AF093FE41E745F4002553E725F4B3
:108FC00000055EE725F400657BE725F4805582E720
:108FD00025F400558CE725F4004591E725F480350C
:108FE00096E725F400359BE725F08075A0E7234B35
:108FF0001F4D033A012A88BF2B46ACE7012386F8B0
:1090000098361D4B1B68C6F89C3645F08055256088
:1090100000200FF015FF2568194A15EA020315D044
:10902000B0B145F4804525602368134214BF022384
:10903000002386F8A036FAF73BF8D6F8A436C01A13
:10904000002808DBBDE8F8431AF014BE0028F0D170
:1090500025F48045E7E7BDE8F88300BF58270120E5
:1090600040BE002048AD0020D0C40020F07C00208D
:1090700000171100407E0500C42A002060CC0500C6
:1090800080FFFF7FF42701200028012038B5454DDF
:109090002B685C0775D5444C84F8A806FAF708F8E5
:1090A00004F5D663C3E900012B68404A23F00403AA
:1090B0002B6013683E4D23F0006313602B68190387
:1090C00007D594F8B8360A2B5CD8082B64D8012B46
:1090D0005AD8384BDB6A1A0406D51420F7F7AEFFCE
:1090E0004FF400403DF051FD94F8D036ABB3324B15
:1090F000D4F8D4261B689B1A42F20F7293422CD9E3
:109100004FF47A72B3FBF2F3D4F8C4261344C4F8D4
:10911000C43633F01BFFD4F8D836C01A6423B0FB32
:10912000F3F0D4F8C83618442B68C4F8C8069B0777
:1091300011D51FF07FF970B1D4F8E026D4F8DC36F1
:109140009B1AD4F8CC261A44C4F8CC26D4F8E426CA
:109150001344C4F8E436FEF755FF1BF08BFE1748A6
:10916000F3F7CFFE1648F3F7CCFE1648F3F7C9FE27
:109170001548F3F7C6FE05201AF0B0FD002384F869
:10918000983638BD0B2BA4D00B4B1B68C4F8C036E7
:109190000B2384F8B8369CE70021FF2021F046FF1E
:1091A000F2E700BF5827012040BE0020F42701202D
:1091B000F827012000280120C42A0020B42901201A
:1091C000142A0120742A0120D42A01201D4B1B6877
:1091D0002DE9F04FD3F828801B4C1C4B1C4F1D4E23
:1091E00007EE908A2DED0C8BF8EEE77A9FED1A9A38
:1091F000C3F85486236867EE897A13F0040F0DEEE6
:10920000100A0DEE901A93B0C7EDCD7A06F5DE6523
:1092100028D10022002345E902231DEE101AD6F8BA
:10922000B0360E4ACB1A52681DEE901A61EB02025C
:109230000B4999424FF0000393416ED2FFF7EAFCCD
:109240005DE000BFEC2701205827012048AD002039
:109250000028012040BE0020BD378635F0C4002024
:1092600020A10700C24B1B68D90606D535F0B8FF10
:1092700018B197F84033032B41D9D6F8F0366A6815
:10928000BC4913EB080342EBE872C6F8F0366A609B
:1092900055E9023213EB080342EBE87245E902326A
:1092A000A1F124030322F1EC017A93ED117AF4EE9B
:1092B000C77A93ED127AF1EE10FAF4EEC77A48BF4E
:1092C000C3ED117AF1EE10FAC8BFC3ED127A013A7C
:1092D00003F10803E7D197EDDD1AD7EDDC0A97ED2E
:1092E000DB0AF4F7E2FAD7EDE97A2368B4EEE70A8D
:1092F000F1EE10FAC8BF87EDE90A5A0789D555E99A
:1093000002239D4991424FF0000272EB03033FBFDD
:10931000974A136823F00063136097F838300BB155
:109320001FF0D8FDFB699B070CD52368DD0606D42A
:10933000D7F850339148984708B11FF0FEF9012340
:1093400087F8A8331DEE100A1DEE901A10F0AEFA41
:1093500097EDCD0AFEF7C6FBFFF758FD884B93F853
:10936000BC353BB11DEE102A1DEE903A96F8F8067A
:109370000FF01AFB96F8F836824D002B00F017819B
:1093800033F042FBDFF810A22268DAF80030D6F89A
:10939000FC16C6F8FC36540714D55B1A07EE903A53
:1093A0009FED797AF8EEE77A05F5805305F580624E
:1093B00067EE877AD2ED006A93ED2F7AA6EEA77A50
:1093C00083ED2F7A34F08AFD40B196F800372BB93F
:1093D0000E201AF083FC012386F80037EB7B2BB1BB
:1093E00016200FF02DFD08B901232B7416200FF065
:1093F00027FDE87335F008FF32F02CFE2A78634B26
:10940000302101FB0233D3F87047FB6A980540F125
:10941000DA84574B1B68590303D5E20401D536F0B3
:109420003DFF0023AB81AB732A78584BDFF8549192
:10943000302101FB023341F6B800D3F8744720EA2B
:1094400004003DF0A2FB20463DF0ACFB2E200FF0C7
:10945000F7FC4F4C8046002800F02A874D4BDB6A12
:109460001A0500F1258734F089FF002840F0208795
:10947000EA8840F202239A4208BF3D4BD4F81827ED
:1094800008BF18684FF0010389F81530424B1B687C
:10949000A3EB020308BFC0F34000B3F57A7F09D203
:1094A00094F8A13533B1002389F8223EA9F81C3E77
:1094B00089F8213E99F921AE002800F0F086BAF132
:1094C000030F00F0F186DFF8D4B09BF80A30002BD0
:1094D00000F0D88640464FF0010A89F821AE0028F6
:1094E0005ED013200FF0ACFC002859D099F9223E31
:1094F0000BB934F0B1F832F033FE014605A83CF068
:1095000037F895F9223E0599142000FB0352B2F872
:10951000CCC4C2F8BC140699C2F8C0144CF0010CBB
:109520000799C2F8C414A2F8CCC400214AF2015C25
:10953000C2F8C814A2F8CEC4012285F81C2E23B1AB
:109540005A1E00FB025282F8CF1401335BB2782B13
:1095500089F8223E89F81F3E89F81D3E0CBF03237F
:10956000022389F8213E0D4B00229A7218E000BFB9
:10957000F42701206C2B012040420F00482B0120D2
:1095800048AD0020849C00206F12833AA035060865
:1095900040BE002000280120C42A00209410002092
:1095A000002033F05FFB99F80130A4F81C37E24B40
:1095B000002283F8F82693F81E2703F5E46B03F5E1
:1095C000ED6403F5EE6A002A49D100230022CAE9BE
:1095D0002823CAE90023CAE90A23CAE91423DBEDD8
:1095E0000F7A9FEDD67AD64B77EE877A93F82937A4
:1095F000C4ED487A4FF00008C4ED497AC4F83081D0
:10960000C4F83481C4F83881C4F83C81C4F8CC80F3
:109610000BB137F07BFFCB4BE36363660123C4F8E8
:10962000BC80C4F80881C4F81481C4F8C080C4F8B0
:109630000C81C4F81881C4F8C480C4F81081C4F83F
:109640001C81C4F83880C4F84080C4F84480C4F851
:109650006080C4F86880C4F86C8086F81E37F9F71B
:1096600027FDDAF8A030019380468946DAF8A41085
:109670000091CAE9288910F0D7F8DDE90013002825
:1096800040F034860023C4F8B030C4F8B430C4F8D5
:10969000B830AB4B93F829370BB137F037FFAA4AF4
:1096A0009FEDAAAADFEDAA9AD2E93E01B8EB00002D
:1096B00069EB01013FF0E0FF07EE900AA24A27EEB6
:1096C000898AC2E93E898DED058A10F0ADF89BEDDF
:1096D0000F7A9D4A8246002840F0E686DFED977AB1
:1096E000C6F8680737EE277A84ED487A84ED497A20
:1096F00026F0A0FD974BB3F93440002801F0E48434
